 psipred

 Timestamp is 5dee3612 (Mon Dec 09 18:54:58 2019)

 Preferred load address is 10000000

 Start         Length     Name                   Class
 0001:00000000 000011a4H .text$di                CODE
 0001:000011b0 00005af8H .text$mn                CODE
 0001:00006cb0 00000bd4H .text$x                 CODE
 0001:00007890 000005aaH .text$yd                CODE
 0002:00000000 000002c0H .idata$5                DATA
 0002:000002c0 00000004H .CRT$XCA                DATA
 0002:000002c4 00000124H .CRT$XCU                DATA
 0002:000003e8 00000004H .CRT$XCZ                DATA
 0002:000003ec 00000004H .CRT$XIA                DATA
 0002:000003f0 00000004H .CRT$XIAA               DATA
 0002:000003f4 00000004H .CRT$XIC                DATA
 0002:000003f8 00000004H .CRT$XIZ                DATA
 0002:00000400 000d8f48H .rdata                  DATA
 0002:000d9348 00000070H .rdata$debug            DATA
 0002:000d93b8 00000464H .rdata$r                DATA
 0002:000d9820 000000ccH .rdata$sxdata           DATA
 0002:000d98ec 00000004H .rtc$IAA                DATA
 0002:000d98f0 00000004H .rtc$IZZ                DATA
 0002:000d98f4 00000004H .rtc$TAA                DATA
 0002:000d98f8 00000004H .rtc$TZZ                DATA
 0002:000d9900 00000f2cH .xdata$x                DATA
 0002:000da830 00000050H .edata                  DATA
 0002:000da880 000000a0H .idata$2                DATA
 0002:000da920 00000014H .idata$3                DATA
 0002:000da934 000002c0H .idata$4                DATA
 0002:000dabf4 000016ceH .idata$6                DATA
 0003:00000000 000001e4H .data                   DATA
 0003:000001e4 0000024cH .data$r                 DATA
 0003:00000430 00000474H .bss                    DATA
 0004:00000000 00000058H .rsrc$01                DATA
 0004:00000060 00000180H .rsrc$02                DATA

  Address         Publics by Value              Rva+Base       Lib:Object

 0000:00000000       __except_list              00000000     <absolute>
 0000:00000000       ___guard_fids_table        00000000     <absolute>
 0000:00000000       ___guard_fids_count        00000000     <absolute>
 0000:00000000       ___guard_flags             00000000     <absolute>
 0000:00000033       ___safe_se_handler_count   00000033     <absolute>
 0000:00009876       __fltused                  00009876     <absolute>
 0000:00009876       __ldused                   00009876     <absolute>
 0000:00000000       ___ImageBase               10000000     <linker-defined>
 0001:000011b0       ??$_Allocate@D@std@@YAPADIPAD@Z 100021b0 f i PsipredAlgTask.obj
 0001:000011e0       ??$_Move@AAPAUData@QListData@@@std@@YA$$QAPAUData@QListData@@AAPAU12@@Z 100021e0 f i PsipredAlgTask.obj
 0001:000011f0       ??$addressof@D@std@@YAPADAAD@Z 100021f0 f i PsipredAlgTask.obj
 0001:00001200       ??$atomic@H@?$QAtomicOpsBySize@$03@@CAPAJPAH@Z 10002200 f i PsipredAlgTask.obj
 0001:00001210       ??$construct@PADAAPAD@?$_Wrap_alloc@V?$allocator@D@std@@@std@@QAEXPAPADAAPAD@Z 10002210 f i PsipredAlgTask.obj
 0001:00001230       ??$construct@PADAAPAD@?$allocator@D@std@@QAEXPAPADAAPAD@Z 10002230 f i PsipredAlgTask.obj
 0001:00001250       ??$construct@PADAAPAD@?$allocator_traits@V?$allocator@D@std@@@std@@SAXAAV?$allocator@D@1@PAPADAAPAD@Z 10002250 f i PsipredAlgTask.obj
 0001:00001270       ??$deref@H@?$QAtomicOpsBySize@$03@@SA_NAAH@Z 10002270 f i PsipredAlgTask.obj
 0001:00001290       ??$destroy@PAD@?$_Wrap_alloc@V?$allocator@D@std@@@std@@QAEXPAPAD@Z 10002290 f i PsipredAlgTask.obj
 0001:000012a0       ??$destroy@PAD@?$allocator@D@std@@QAEXPAPAD@Z 100022a0 f i PsipredAlgTask.obj
 0001:000012b0       ??$destroy@PAD@?$allocator_traits@V?$allocator@D@std@@@std@@SAXAAV?$allocator@D@1@PAPAD@Z 100022b0 f i PsipredAlgTask.obj
 0001:000012c0       ??$forward@AAPAD@std@@YAAAPADAAPAD@Z 100022c0 f i PsipredAlgTask.obj
 0001:000012d0       ??$load@H@?$QGenericAtomicOps@U?$QAtomicOpsBySize@$03@@@@SAHABH@Z 100022d0 f i PsipredAlgTask.obj
 0001:000012e0       ??$qSwap@PAUData@QListData@@@@YAXAAPAUData@QListData@@0@Z 100022e0 f i PsipredAlgTask.obj
 0001:00001300       ??$swap@PAUData@QListData@@@std@@YAXAAPAUData@QListData@@0@Z 10002300 f i PsipredAlgTask.obj
 0001:00001320       ??0?$AbstractId@H@U2@@IAE@ABH@Z 10002320 f i PsipredAlgTask.obj
 0001:00001340       ??0?$QList@VQString@@@@QAE@XZ 10002340 f i PsipredAlgTask.obj
 0001:00001350       ??0?$_String_alloc@$0A@U?$_String_base_types@DV?$allocator@D@std@@@std@@@std@@QAE@ABV?$allocator@D@1@@Z 10002350 f i PsipredAlgTask.obj
 0001:00001370       ??0?$_String_val@U?$_Simple_types@D@std@@@std@@QAE@XZ 10002370 f i PsipredAlgTask.obj
 0001:00001390       ??0?$_Wrap_alloc@V?$allocator@D@std@@@std@@QAE@XZ 10002390 f i PsipredAlgTask.obj
 0001:000013a0       ??0?$allocator@D@std@@QAE@XZ 100023a0 f i PsipredAlgTask.obj
 0001:000013b0       ??0?$basic_string@DU?$char_traits@D@std@@V?$allocator@D@2@@std@@QAE@PBD@Z 100023b0 f i PsipredAlgTask.obj
 0001:00001410       ??0AbstractInt32Id@U2@@IAE@H@Z 10002410 f i PsipredAlgTask.obj
 0001:00001430       ??0PsipredAlgTask@U2@@QAE@ABVQByteArray@@@Z 10002430 f   PsipredAlgTask.obj
 0001:00001520       ??0QLatin1Char@@QAE@D@Z    10002520 f i PsipredAlgTask.obj
 0001:00001530       ??0QStringList@@QAE@XZ     10002530 f i PsipredAlgTask.obj
 0001:00001540       ??0ServiceType@U2@@QAE@H@Z 10002540 f i PsipredAlgTask.obj
 0001:00001560       ??0_Generic_error_category@std@@QAE@XZ 10002560 f i PsipredAlgTask.obj
 0001:00001570       ??0_Ignore@std@@QAE@XZ     10002570 f i PsipredAlgTask.obj
 0001:00001580       ??0_Iostream_error_category@std@@QAE@XZ 10002580 f i PsipredAlgTask.obj
 0001:00001590       ??0_System_error_category@std@@QAE@XZ 10002590 f i PsipredAlgTask.obj
 0001:000015a0       ??0error_category@std@@QAE@XZ 100025a0 f i PsipredAlgTask.obj
 0001:000015b0       ??0error_condition@std@@QAE@HABVerror_category@1@@Z 100025b0 f i PsipredAlgTask.obj
 0001:000015d0       ??1?$AbstractId@H@U2@@MAE@XZ 100025d0 f i PsipredAlgTask.obj
 0001:000015e0       ??1?$QList@V?$QSharedDataPointer@VAnnotationData@U2@@@@@@QAE@XZ 100025e0 f i PsipredAlgTask.obj
 0001:00001630       ??1?$QList@VQString@@@@QAE@XZ 10002630 f i PsipredAlgTask.obj
 0001:00001690       ??1?$QSharedDataPointer@VAnnotationData@U2@@@@QAE@XZ 10002690 f i PsipredAlgTask.obj
 0001:000016c0       ??1?$basic_string@DU?$char_traits@D@std@@V?$allocator@D@2@@std@@QAE@XZ 100026c0 f i PsipredAlgTask.obj
 0001:000016f0       ??1AbstractInt32Id@U2@@UAE@XZ 100026f0 f i PsipredAlgTask.obj
 0001:00001700       ??1PsipredAlgTask@U2@@UAE@XZ 10002700 f i PsipredAlgTask.obj
 0001:00001710       ??1QStringList@@QAE@XZ     10002710 f i PsipredAlgTask.obj
 0001:00001720       ??1ServiceType@U2@@UAE@XZ  10002720 f i PsipredAlgTask.obj
 0001:00001730       ??1_Generic_error_category@std@@UAE@XZ 10002730 f i PsipredAlgTask.obj
 0001:00001740       ??1_Iostream_error_category@std@@UAE@XZ 10002740 f i PsipredAlgTask.obj
 0001:00001750       ??1_System_error_category@std@@UAE@XZ 10002750 f i PsipredAlgTask.obj
 0001:00001760       ??1error_category@std@@UAE@XZ 10002760 f i PsipredAlgTask.obj
 0001:00001770       ??2@YAPAXIPAX@Z            10002770 f i PsipredAlgTask.obj
 0001:00001780       ??3@YAXPAX0@Z              10002780 f i PsipredAlgTask.obj
 0001:00001790       ??4?$QList@V?$QSharedDataPointer@VAnnotationData@U2@@@@@@QAEAAV0@$$QAV0@@Z 10002790 f i PsipredAlgTask.obj
 0001:000017b0       ??6QStringList@@QAEAAV0@ABVQString@@@Z 100027b0 f i PsipredAlgTask.obj
 0001:000017d0       ??8error_category@std@@QBE_NABV01@@Z 100027d0 f i PsipredAlgTask.obj
 0001:000017e0       ??8error_condition@std@@QBE_NABV01@@Z 100027e0 f i PsipredAlgTask.obj
 0001:00001800       ??H@YA?BVQString@@ABV0@PBD@Z 10002800 f i PsipredAlgTask.obj
 0001:000018a0       ??H@YA?BVQString@@ABV0@VQChar@@@Z 100028a0 f i PsipredAlgTask.obj
 0001:00001910       ??_E?$AbstractId@H@U2@@MAEPAXI@Z 10002910 f i PsipredAlgTask.obj
 0001:00001910       ??_G?$AbstractId@H@U2@@MAEPAXI@Z 10002910 f i PsipredAlgTask.obj
 0001:00001940       ??_G?$QSharedDataPointer@VAnnotationData@U2@@@@QAEPAXI@Z 10002940 f i PsipredAlgTask.obj
 0001:00001990       ??_GAbstractInt32Id@U2@@UAEPAXI@Z 10002990 f i PsipredAlgTask.obj
 0001:00001990       ??_EAbstractInt32Id@U2@@UAEPAXI@Z 10002990 f i PsipredAlgTask.obj
 0001:000019c0       ??_GAnnotationData@U2@@QAEPAXI@Z 100029c0 f i PsipredAlgTask.obj
 0001:000019f0       ??_EPsipredAlgTask@U2@@UAEPAXI@Z 100029f0 f i PsipredAlgTask.obj
 0001:000019f0       ??_GPsipredAlgTask@U2@@UAEPAXI@Z 100029f0 f i PsipredAlgTask.obj
 0001:00001a20       ??_GQString@@QAEPAXI@Z     10002a20 f i PsipredAlgTask.obj
 0001:00001a50       ??_EServiceType@U2@@UAEPAXI@Z 10002a50 f i PsipredAlgTask.obj
 0001:00001a50       ??_GServiceType@U2@@UAEPAXI@Z 10002a50 f i PsipredAlgTask.obj
 0001:00001a80       ??_G_Generic_error_category@std@@UAEPAXI@Z 10002a80 f i PsipredAlgTask.obj
 0001:00001a80       ??_E_Generic_error_category@std@@UAEPAXI@Z 10002a80 f i PsipredAlgTask.obj
 0001:00001ab0       ??_G_Iostream_error_category@std@@UAEPAXI@Z 10002ab0 f i PsipredAlgTask.obj
 0001:00001ab0       ??_E_Iostream_error_category@std@@UAEPAXI@Z 10002ab0 f i PsipredAlgTask.obj
 0001:00001ae0       ??_E_System_error_category@std@@UAEPAXI@Z 10002ae0 f i PsipredAlgTask.obj
 0001:00001ae0       ??_G_System_error_category@std@@UAEPAXI@Z 10002ae0 f i PsipredAlgTask.obj
 0001:00001b10       ??_Gerror_category@std@@UAEPAXI@Z 10002b10 f i PsipredAlgTask.obj
 0001:00001b10       ??_Eerror_category@std@@UAEPAXI@Z 10002b10 f i PsipredAlgTask.obj
 0001:00001b40       ?_Copy@?$basic_string@DU?$char_traits@D@std@@V?$allocator@D@2@@std@@QAEXII@Z 10002b40 f i PsipredAlgTask.obj
 0001:00001c90       ?_Eos@?$basic_string@DU?$char_traits@D@std@@V?$allocator@D@2@@std@@QAEXI@Z 10002c90 f i PsipredAlgTask.obj
 0001:00001cc0       ?_Getal@?$_String_alloc@$0A@U?$_String_base_types@DV?$allocator@D@std@@@std@@@std@@QBE?AU?$_Wrap_alloc@V?$allocator@D@std@@@2@XZ 10002cc0 f i PsipredAlgTask.obj
 0001:00001cd0       ?_Grow@?$basic_string@DU?$char_traits@D@std@@V?$allocator@D@2@@std@@QAE_NI_N@Z 10002cd0 f i PsipredAlgTask.obj
 0001:00001d80       ?_Inside@?$basic_string@DU?$char_traits@D@std@@V?$allocator@D@2@@std@@QAE_NPBD@Z 10002d80 f i PsipredAlgTask.obj
 0001:00001dc0       ?_Myptr@?$_String_val@U?$_Simple_types@D@std@@@std@@QAEPADXZ 10002dc0 f i PsipredAlgTask.obj
 0001:00001dd0       ?_Myptr@?$_String_val@U?$_Simple_types@D@std@@@std@@QBEPBDXZ 10002dd0 f i PsipredAlgTask.obj
 0001:00001de0       ?_Tidy@?$basic_string@DU?$char_traits@D@std@@V?$allocator@D@2@@std@@QAEX_NI@Z 10002de0 f i PsipredAlgTask.obj
 0001:00001e30       ?_Xlen@?$basic_string@DU?$char_traits@D@std@@V?$allocator@D@2@@std@@QBEXXZ 10002e30 f i PsipredAlgTask.obj
 0001:00001e40       ?_Xran@?$basic_string@DU?$char_traits@D@std@@V?$allocator@D@2@@std@@QBEXXZ 10002e40 f i PsipredAlgTask.obj
 0001:00001e50       ?allocate@?$_Wrap_alloc@V?$allocator@D@std@@@std@@QAEPADI@Z 10002e50 f i PsipredAlgTask.obj
 0001:00001e80       ?allocate@?$allocator@D@std@@QAEPADI@Z 10002e80 f i PsipredAlgTask.obj
 0001:00001eb0       ?append@?$QList@VQString@@@@QAEXABVQString@@@Z 10002eb0 f i PsipredAlgTask.obj
 0001:00001fa0       ?assign@?$basic_string@DU?$char_traits@D@std@@V?$allocator@D@2@@std@@QAEAAV12@ABV12@II@Z 10002fa0 f i PsipredAlgTask.obj
 0001:000020c0       ?assign@?$basic_string@DU?$char_traits@D@std@@V?$allocator@D@2@@std@@QAEAAV12@PBD@Z 100030c0 f i PsipredAlgTask.obj
 0001:00002100       ?assign@?$basic_string@DU?$char_traits@D@std@@V?$allocator@D@2@@std@@QAEAAV12@PBDI@Z 10003100 f i PsipredAlgTask.obj
 0001:00002200       ?assign@?$char_traits@D@std@@SAXAADABD@Z 10003200 f i PsipredAlgTask.obj
 0001:00002210       ?category@error_code@std@@QBEABVerror_category@2@XZ 10003210 f i PsipredAlgTask.obj
 0001:00002220       ?category@error_condition@std@@QBEABVerror_category@2@XZ 10003220 f i PsipredAlgTask.obj
 0001:00002230       ?copy@?$char_traits@D@std@@SAPADPADPBDI@Z 10003230 f i PsipredAlgTask.obj
 0001:00002250       ?dealloc@?$QList@V?$QSharedDataPointer@VAnnotationData@U2@@@@@@AAEXPAUData@QListData@@@Z 10003250 f i PsipredAlgTask.obj
 0001:00002280       ?dealloc@?$QList@VQString@@@@AAEXPAUData@QListData@@@Z 10003280 f i PsipredAlgTask.obj
 0001:000022c0       ?deallocate@?$_Wrap_alloc@V?$allocator@D@std@@@std@@QAEXPADI@Z 100032c0 f i PsipredAlgTask.obj
 0001:000022e0       ?deallocate@?$allocator@D@std@@QAEXPADI@Z 100032e0 f i PsipredAlgTask.obj
 0001:00002300       ?default_error_condition@_System_error_category@std@@UBE?AVerror_condition@2@H@Z 10003300 f i PsipredAlgTask.obj
 0001:00002340       ?default_error_condition@error_category@std@@UBE?AVerror_condition@2@H@Z 10003340 f i PsipredAlgTask.obj
 0001:00002360       ?deref@?$QBasicAtomicInteger@H@@QAE_NXZ 10003360 f i PsipredAlgTask.obj
 0001:00002370       ?deref@RefCount@QtPrivate@@QAE_NXZ 10003370 f i PsipredAlgTask.obj
 0001:00002390       ?detach_helper_grow@?$QList@VQString@@@@AAEPAUNode@1@HH@Z 10003390 f i PsipredAlgTask.obj
 0001:00002510       ?equivalent@error_category@std@@UBE_NABVerror_code@2@H@Z 10003510 f i PsipredAlgTask.obj
 0001:00002530       ?equivalent@error_category@std@@UBE_NHABVerror_condition@2@@Z 10003530 f i PsipredAlgTask.obj
 0001:00002570       ?erase@?$basic_string@DU?$char_traits@D@std@@V?$allocator@D@2@@std@@QAEAAV12@I@Z 10003570 f i PsipredAlgTask.obj
 0001:000025b0       ?erase@?$basic_string@DU?$char_traits@D@std@@V?$allocator@D@2@@std@@QAEAAV12@II@Z 100035b0 f i PsipredAlgTask.obj
 0001:00002650       ?generic_category@std@@YAABVerror_category@1@XZ 10003650 f i PsipredAlgTask.obj
 0001:00002660       ?isShared@RefCount@QtPrivate@@QBE_NXZ 10003660 f i PsipredAlgTask.obj
 0001:00002680       ?isValid@AbstractInt32Id@U2@@UBE_NXZ 10003680 f i PsipredAlgTask.obj
 0001:00002690       ?length@?$char_traits@D@std@@SAIPBD@Z 10003690 f i PsipredAlgTask.obj
 0001:000026b0       ?load@?$QBasicAtomicInteger@H@@QBEHXZ 100036b0 f i PsipredAlgTask.obj
 0001:000026c0       ?max_size@?$_Wrap_alloc@V?$allocator@D@std@@@std@@QBEIXZ 100036c0 f i PsipredAlgTask.obj
 0001:000026d0       ?max_size@?$allocator@D@std@@QBEIXZ 100036d0 f i PsipredAlgTask.obj
 0001:000026e0       ?max_size@?$allocator_traits@V?$allocator@D@std@@@std@@SAIABV?$allocator@D@2@@Z 100036e0 f i PsipredAlgTask.obj
 0001:000026f0       ?max_size@?$basic_string@DU?$char_traits@D@std@@V?$allocator@D@2@@std@@QBEIXZ 100036f0 f i PsipredAlgTask.obj
 0001:00002700       ?message@_Generic_error_category@std@@UBE?AV?$basic_string@DU?$char_traits@D@std@@V?$allocator@D@2@@2@H@Z 10003700 f i PsipredAlgTask.obj
 0001:00002780       ?message@_Iostream_error_category@std@@UBE?AV?$basic_string@DU?$char_traits@D@std@@V?$allocator@D@2@@2@H@Z 10003780 f i PsipredAlgTask.obj
 0001:000027d0       ?message@_System_error_category@std@@UBE?AV?$basic_string@DU?$char_traits@D@std@@V?$allocator@D@2@@2@H@Z 100037d0 f i PsipredAlgTask.obj
 0001:00002850       ?move@?$char_traits@D@std@@SAPADPADPBDI@Z 10003850 f i PsipredAlgTask.obj
 0001:00002870       ?name@_Generic_error_category@std@@UBEPBDXZ 10003870 f i PsipredAlgTask.obj
 0001:00002880       ?name@_Iostream_error_category@std@@UBEPBDXZ 10003880 f i PsipredAlgTask.obj
 0001:00002890       ?name@_System_error_category@std@@UBEPBDXZ 10003890 f i PsipredAlgTask.obj
 0001:000028a0       ?node_construct@?$QList@VQString@@@@AAEXPAUNode@1@ABVQString@@@Z 100038a0 f i PsipredAlgTask.obj
 0001:000028f0       ?node_copy@?$QList@VQString@@@@AAEXPAUNode@1@00@Z 100038f0 f i PsipredAlgTask.obj
 0001:00002990       ?node_destruct@?$QList@V?$QSharedDataPointer@VAnnotationData@U2@@@@@@AAEXPAUNode@1@0@Z 10003990 f i PsipredAlgTask.obj
 0001:000029e0       ?node_destruct@?$QList@VQString@@@@AAEXPAUNode@1@0@Z 100039e0 f i PsipredAlgTask.obj
 0001:00002a10       ?node_destruct@?$QList@VQString@@@@AAEXPAUNode@1@@Z 10003a10 f i PsipredAlgTask.obj
 0001:00002a20       ?run@PsipredAlgTask@U2@@UAEXXZ 10003a20 f   PsipredAlgTask.obj
 0001:00003120       ?size@?$basic_string@DU?$char_traits@D@std@@V?$allocator@D@2@@std@@QBEIXZ 10004120 f i PsipredAlgTask.obj
 0001:00003130       ?system_category@std@@YAABVerror_category@1@XZ 10004130 f i PsipredAlgTask.obj
 0001:00003140       ?value@error_code@std@@QBEHXZ 10004140 f i PsipredAlgTask.obj
 0001:00003150       ?value@error_condition@std@@QBEHXZ 10004150 f i PsipredAlgTask.obj
 0001:00003160       _hypot                     10004160 f i PsipredAlgTask.obj
 0001:00003190       ??0?$QList@PAVAnnotationSettings@U2@@@@QAE@XZ 10004190 f i PsipredPlugin.obj
 0001:000031a0       ??0Factory@PsipredAlgTask@U2@@QAE@XZ 100041a0 f i PsipredPlugin.obj
 0001:000031b0       ??0PsipredPlugin@U2@@QAE@XZ 100041b0 f   PsipredPlugin.obj
 0001:000033a0       ??1?$QList@PAVAnnotationSettings@U2@@@@QAE@XZ 100043a0 f i PsipredPlugin.obj
 0001:000033d0       ??1Factory@PsipredAlgTask@U2@@UAE@XZ 100043d0 f i PsipredPlugin.obj
 0001:000033e0       ??1PsipredPlugin@U2@@UAE@XZ 100043e0 f   PsipredPlugin.obj
 0001:000033f0       ??6?$QList@PAVAnnotationSettings@U2@@@@QAEAAV0@ABQAVAnnotationSettings@U2@@@Z 100043f0 f i PsipredPlugin.obj
 0001:00003410       ??_GFactory@PsipredAlgTask@U2@@UAEPAXI@Z 10004410 f i PsipredPlugin.obj
 0001:00003410       ??_EFactory@PsipredAlgTask@U2@@UAEPAXI@Z 10004410 f i PsipredPlugin.obj
 0001:00003440       ??_GPsipredPlugin@U2@@UAEPAXI@Z 10004440 f i PsipredPlugin.obj
 0001:00003440       ??_EPsipredPlugin@U2@@UAEPAXI@Z 10004440 f i PsipredPlugin.obj
 0001:00003470       ?append@?$QList@PAVAnnotationSettings@U2@@@@QAEXABQAVAnnotationSettings@U2@@@Z 10004470 f i PsipredPlugin.obj
 0001:00003500       ?createTaskInstance@Factory@PsipredAlgTask@U2@@UAEPAVSecStructPredictTask@3@ABVQByteArray@@@Z 10004500 f i PsipredPlugin.obj
 0001:00003570       ?dealloc@?$QList@PAVAnnotationSettings@U2@@@@AAEXPAUData@QListData@@@Z 10004570 f i PsipredPlugin.obj
 0001:00003590       ?detach_helper_grow@?$QList@PAVAnnotationSettings@U2@@@@AAEPAUNode@1@HH@Z 10004590 f i PsipredPlugin.obj
 0001:000036a0       ?node_construct@?$QList@PAVAnnotationSettings@U2@@@@AAEXPAUNode@1@ABQAVAnnotationSettings@U2@@@Z 100046a0 f i PsipredPlugin.obj
 0001:000036c0       ?node_copy@?$QList@PAVAnnotationSettings@U2@@@@AAEXPAUNode@1@00@Z 100046c0 f i PsipredPlugin.obj
 0001:000036f0       ?node_destruct@?$QList@PAVAnnotationSettings@U2@@@@AAEXPAUNode@1@0@Z 100046f0 f i PsipredPlugin.obj
 0001:00003700       ?node_destruct@?$QList@PAVAnnotationSettings@U2@@@@AAEXPAUNode@1@@Z 10004700 f i PsipredPlugin.obj
 0001:00003710       ?tr@PsipredPlugin@U2@@SA?AVQString@@PBD0H@Z 10004710 f i PsipredPlugin.obj
 0001:00003740       _ugene_plugin_init         10004740 f   PsipredPlugin.obj
 0001:00003760       ?seq2mtx@@YAHPBDH0@Z       10004760 f   seq2mtx.obj
 0001:00003880       ?seq2mtx@@YAHPBDHPAVQTemporaryFile@@@Z 10004880 f   seq2mtx.obj
 0001:000039d0       ??$ref@H@?$QAtomicOpsBySize@$03@@SA_NAAH@Z 100049d0 f i sspred_avpred.obj
 0001:000039f0       ??0?$QFlags@W4OpenModeFlag@QIODevice@@@@QAE@W4OpenModeFlag@QIODevice@@@Z 100049f0 f i sspred_avpred.obj
 0001:00003a00       ??0?$QForeachContainer@VQStringList@@@@QAE@ABVQStringList@@@Z 10004a00 f i sspred_avpred.obj
 0001:00003a40       ??0?$QList@VQString@@@@QAE@ABV0@@Z 10004a40 f i sspred_avpred.obj
 0001:00003b00       ??0PsiPassOne@@QAE@PAVQTemporaryFile@@ABVQStringList@@@Z 10004b00 f   sspred_avpred.obj
 0001:00003bc0       ??0QStringList@@QAE@ABV0@@Z 10004bc0 f i sspred_avpred.obj
 0001:00003be0       ??0const_iterator@?$QList@VQString@@@@QAE@PAUNode@1@@Z 10004be0 f i sspred_avpred.obj
 0001:00003bf0       ??1?$QForeachContainer@VQStringList@@@@QAE@XZ 10004bf0 f i sspred_avpred.obj
 0001:00003c00       ??1PsiPassOne@@QAE@XZ      10004c00 f   sspred_avpred.obj
 0001:00003d00       ??9const_iterator@?$QList@VQString@@@@QBE_NABV01@@Z 10004d00 f i sspred_avpred.obj
 0001:00003d20       ??Dconst_iterator@?$QList@VQString@@@@QBEABVQString@@XZ 10004d20 f i sspred_avpred.obj
 0001:00003d30       ??Econst_iterator@?$QList@VQString@@@@QAEAAV01@XZ 10004d30 f i sspred_avpred.obj
 0001:00003d40       ?begin@?$QList@VQString@@@@QBE?AVconst_iterator@1@XZ 10004d40 f i sspred_avpred.obj
 0001:00003d60       ?compute_output@PsiPassOne@@QAEXXZ 10004d60 f   sspred_avpred.obj
 0001:00003ed0       ?end@?$QList@VQString@@@@QBE?AVconst_iterator@1@XZ 10004ed0 f i sspred_avpred.obj
 0001:00003ef0       ?exp@@YAMM@Z               10004ef0 f i sspred_avpred.obj
 0001:00003f20       ?getmtx@PsiPassOne@@QAEHXZ 10004f20 f   sspred_avpred.obj
 0001:000041e0       ?init@PsiPassOne@@QAEXXZ   100051e0 f   sspred_avpred.obj
 0001:00004290       ?load_wts@PsiPassOne@@QAEXPBD@Z 10005290 f   sspred_avpred.obj
 0001:00004440       ?predict@PsiPassOne@@QAEXXZ 10005440 f   sspred_avpred.obj
 0001:00004a40       ?ref@?$QBasicAtomicInteger@H@@QAE_NXZ 10005a40 f i sspred_avpred.obj
 0001:00004a60       ?ref@RefCount@QtPrivate@@QAE_NXZ 10005a60 f i sspred_avpred.obj
 0001:00004a80       ?runPsiPass@PsiPassOne@@QAEHXZ 10005a80 f   sspred_avpred.obj
 0001:00004aa0       ?t@Node@?$QList@VQString@@@@QAEAAVQString@@XZ 10005aa0 f i sspred_avpred.obj
 0001:00004ab0       _expf                      10005ab0 f i sspred_avpred.obj
 0001:00004ad0       ??0PsiPassTwo@@QAE@XZ      10005ad0 f   sspred_hmulti.obj
 0001:00004b20       ??1PsiPassTwo@@QAE@XZ      10005b20 f   sspred_hmulti.obj
 0001:00004b50       ?compute_output@PsiPassTwo@@QAEXXZ 10005b50 f   sspred_hmulti.obj
 0001:00004cc0       ?getss@PsiPassTwo@@QAEHPAU_iobuf@@@Z 10005cc0 f   sspred_hmulti.obj
 0001:00004e10       ?init@PsiPassTwo@@QAEXXZ   10005e10 f   sspred_hmulti.obj
 0001:00004ec0       ?load_wts@PsiPassTwo@@QAEXPBD@Z 10005ec0 f   sspred_hmulti.obj
 0001:00005040       ?predict@PsiPassTwo@@QAE?AVQByteArray@@HMMPBD@Z 10006040 f   sspred_hmulti.obj
 0001:000057b0       ?runPsiPass@PsiPassTwo@@QAEHHQAPBDAAVQByteArray@@@Z 100067b0 f   sspred_hmulti.obj
 0001:00005a50       ?aanum@@YAHH@Z             10006a50 f   sspred_utils.obj
 0001:00005a80       ?err@@YAXPBD@Z             10006a80 f   sspred_utils.obj
 0001:00005aa0       ?fail@@YAXPBD@Z            10006aa0 f   sspred_utils.obj
 0001:00005ae0       ??C?$QScopedPointer@VQObjectData@@U?$QScopedPointerDeleter@VQObjectData@@@@@@QBEPAVQObjectData@@XZ 10006ae0 f i moc_PsipredAlgTask.obj
 0001:00005af0       ?metaObject@PsipredAlgTask@U2@@UBEPBUQMetaObject@@XZ 10006af0 f   moc_PsipredAlgTask.obj
 0001:00005b10       ?qt_metacall@PsipredAlgTask@U2@@UAEHW4Call@QMetaObject@@HPAPAX@Z 10006b10 f   moc_PsipredAlgTask.obj
 0001:00005b20       ?qt_metacast@PsipredAlgTask@U2@@UAEPAXPBD@Z 10006b20 f   moc_PsipredAlgTask.obj
 0001:00005b80       ?qt_noop@@YAXXZ            10006b80 f i moc_PsipredAlgTask.obj
 0001:00005b90       ?qt_static_metacall@PsipredAlgTask@U2@@CAXPAVQObject@@W4Call@QMetaObject@@HPAPAX@Z 10006b90 f   moc_PsipredAlgTask.obj
 0001:00005ba0       ?metaObject@PsipredPlugin@U2@@UBEPBUQMetaObject@@XZ 10006ba0 f   moc_PsipredPlugin.obj
 0001:00005bc0       ?qt_metacall@PsipredPlugin@U2@@UAEHW4Call@QMetaObject@@HPAPAX@Z 10006bc0 f   moc_PsipredPlugin.obj
 0001:00005bd0       ?qt_metacast@PsipredPlugin@U2@@UAEPAXPBD@Z 10006bd0 f   moc_PsipredPlugin.obj
 0001:00005c30       ?qt_static_metacall@PsipredPlugin@U2@@CAXPAVQObject@@W4Call@QMetaObject@@HPAPAX@Z 10006c30 f   moc_PsipredPlugin.obj
 0001:00005c40       ??0initializer@?A0x86132f99@@QAE@XZ 10006c40 f i qrc_psipred.obj
 0001:00005c60       ??1initializer@?A0x86132f99@@QAE@XZ 10006c60 f i qrc_psipred.obj
 0001:00005c80       ?qCleanupResources_psipred@@YAHXZ 10006c80 f   qrc_psipred.obj
 0001:00005ca0       ?qInitResources_psipred@@YAHXZ 10006ca0 f   qrc_psipred.obj
 0001:00005cc0       ??1AnnotationData@U2@@QAE@XZ 10006cc0 f   U2Core:U2Core.dll
 0001:00005cc6       ??1GCounter@U2@@UAE@XZ     10006cc6 f   U2Core:U2Core.dll
 0001:00005ccc       ??0GReportableCounter@U2@@QAE@ABVQString@@0N@Z 10006ccc f   U2Core:U2Core.dll
 0001:00005cd2       ?getAppSettings@AppContext@U2@@SAPAVAppSettings@2@XZ 10006cd2 f   U2Core:U2Core.dll
 0001:00005cd8       ?getUserTemporaryDirPath@UserAppsSettings@U2@@QBE?AVQString@@XZ 10006cd8 f   U2Core:U2Core.dll
 0001:00005cde       ??0Logger@U2@@QAE@ABVQString@@@Z 10006cde f   U2Core:U2Core.dll
 0001:00005ce4       ??1Logger@U2@@UAE@XZ       10006ce4 f   U2Core:U2Core.dll
 0001:00005cea       ?cleanup@Task@U2@@UAEXXZ   10006cea f   U2Core:U2Core.dll
 0001:00005cf0       ?generateReport@Task@U2@@UBE?AVQString@@XZ 10006cf0 f   U2Core:U2Core.dll
 0001:00005cf6       ?getNumParallelSubtasks@Task@U2@@UBEHXZ 10006cf6 f   U2Core:U2Core.dll
 0001:00005cfc       ?getParentTask@Task@U2@@UBEPAV12@XZ 10006cfc f   U2Core:U2Core.dll
 0001:00005d02       ?getSubtaskWithErrors@Task@U2@@UBEPAV12@XZ 10006d02 f   U2Core:U2Core.dll
 0001:00005d08       ?getTaskId@Task@U2@@UBE_JXZ 10006d08 f   U2Core:U2Core.dll
 0001:00005d0e       ?getTopLevelParentTask@Task@U2@@UAEPAV12@XZ 10006d0e f   U2Core:U2Core.dll
 0001:00005d14       ?getWarnings@Task@U2@@UBE?AVQStringList@@XZ 10006d14 f   U2Core:U2Core.dll
 0001:00005d1a       ?hasSubtasksWithErrors@Task@U2@@UBE_NXZ 10006d1a f   U2Core:U2Core.dll
 0001:00005d20       ?hasWarning@Task@U2@@UBE_NXZ 10006d20 f   U2Core:U2Core.dll
 0001:00005d26       ?isNotificationReport@Task@U2@@UBE_NXZ 10006d26 f   U2Core:U2Core.dll
 0001:00005d2c       ?isReportingEnabled@Task@U2@@UBE_NXZ 10006d2c f   U2Core:U2Core.dll
 0001:00005d32       ?isReportingSupported@Task@U2@@UBE_NXZ 10006d32 f   U2Core:U2Core.dll
 0001:00005d38       ?isTopLevelTask@Task@U2@@UBE_NXZ 10006d38 f   U2Core:U2Core.dll
 0001:00005d3e       ?onSubTaskFinished@Task@U2@@MAE?AV?$QList@PAVTask@U2@@@@PAV12@@Z 10006d3e f   U2Core:U2Core.dll
 0001:00005d44       ?propagateSubtaskError@Task@U2@@UAE_NXZ 10006d44 f   U2Core:U2Core.dll
 0001:00005d4a       ?report@Task@U2@@UAE?AW4ReportResult@12@XZ 10006d4a f   U2Core:U2Core.dll
 0001:00005d50       ?setCollectChildrensWarningsFlag@Task@U2@@UAEX_N@Z 10006d50 f   U2Core:U2Core.dll
 0001:00005d56       ?setNoAutoDelete@Task@U2@@UAEX_N@Z 10006d56 f   U2Core:U2Core.dll
 0001:00005d5c       ?setNotificationReport@Task@U2@@UAEX_N@Z 10006d5c f   U2Core:U2Core.dll
 0001:00005d62       ?setReportingEnabled@Task@U2@@UAEX_N@Z 10006d62 f   U2Core:U2Core.dll
 0001:00005d68       ?setReportingSupported@Task@U2@@UAEX_N@Z 10006d68 f   U2Core:U2Core.dll
 0001:00005d6e       ??0Plugin@U2@@QAE@ABVQString@@0_NW4PluginState@1@@Z 10006d6e f   U2Core:U2Core.dll
 0001:00005d74       ??1Plugin@U2@@UAE@XZ       10006d74 f   U2Core:U2Core.dll
 0001:00005d7a       ?getAnnotationsSettingsRegistry@AppContext@U2@@SAPAVAnnotationSettingsRegistry@2@XZ 10006d7a f   U2Core:U2Core.dll
 0001:00005d80       ?getSecStructPredictAlgRegistry@AppContext@U2@@SAPAVSecStructPredictAlgRegistry@2@XZ 10006d80 f   U2Core:U2Core.dll
 0001:00005d86       ??0AnnotationSettings@U2@@QAE@ABVQString@@_NABVQColor@@1@Z 10006d86 f   U2Core:U2Core.dll
 0001:00005d8c       ?changeSettings@AnnotationSettingsRegistry@U2@@QAEXABV?$QList@PAVAnnotationSettings@U2@@@@_N@Z 10006d8c f   U2Core:U2Core.dll
 0001:00005d92       ?qt_metacast@Plugin@U2@@UAEPAXPBD@Z 10006d92 f   U2Core:U2Core.dll
 0001:00005d98       ?qt_metacall@Plugin@U2@@UAEHW4Call@QMetaObject@@HPAPAX@Z 10006d98 f   U2Core:U2Core.dll
 0001:00005d9e       ?tr@SecStructPredictTask@U2@@SA?AVQString@@PBD0H@Z 10006d9e f   U2Algorithm:U2Algorithm.dll
 0001:00005da4       ??0SecStructPredictTask@U2@@QAE@ABVQByteArray@@@Z 10006da4 f   U2Algorithm:U2Algorithm.dll
 0001:00005daa       ??1SecStructPredictTask@U2@@UAE@XZ 10006daa f   U2Algorithm:U2Algorithm.dll
 0001:00005db0       ?prepare@SecStructPredictTask@U2@@UAEXXZ 10006db0 f   U2Algorithm:U2Algorithm.dll
 0001:00005db6       ?registerAlgorithm@SecStructPredictAlgRegistry@U2@@QAE_NPAVSecStructPredictTaskFactory@2@ABVQString@@@Z 10006db6 f   U2Algorithm:U2Algorithm.dll
 0001:00005dbc       ?qt_metacast@SecStructPredictTask@U2@@UAEPAXPBD@Z 10006dbc f   U2Algorithm:U2Algorithm.dll
 0001:00005dc2       ?qt_metacall@SecStructPredictTask@U2@@UAEHW4Call@QMetaObject@@HPAPAX@Z 10006dc2 f   U2Algorithm:U2Algorithm.dll
 0001:00005dc8       ?saveAlgorithmResultsAsAnnotations@SecStructPredictUtils@U2@@SA?AV?$QList@V?$QSharedDataPointer@VAnnotationData@U2@@@@@@ABVQByteArray@@ABVQString@@@Z 10006dc8 f   U2View:U2View.dll
 0001:00005dce       ?setRgb@QColor@@QAEXHHHH@Z 10006dce f   Qt5Gui:Qt5Gui.dll
 0001:00005dd4       ??0QMutex@@QAE@W4RecursionMode@0@@Z 10006dd4 f   Qt5Core:Qt5Core.dll
 0001:00005dda       ??1QMutex@@QAE@XZ          10006dda f   Qt5Core:Qt5Core.dll
 0001:00005de0       ??0QMutexLocker@@QAE@PAVQBasicMutex@@@Z 10006de0 f   Qt5Core:Qt5Core.dll
 0001:00005de6       ??1QMutexLocker@@QAE@XZ    10006de6 f   Qt5Core:Qt5Core.dll
 0001:00005dec       ?unlock@QMutexLocker@@QAEXXZ 10006dec f   Qt5Core:Qt5Core.dll
 0001:00005df2       ??0QChar@@QAE@UQLatin1Char@@@Z 10006df2 f   Qt5Core:Qt5Core.dll
 0001:00005df8       ?constData@QByteArray@@QBEPBDXZ 10006df8 f   Qt5Core:Qt5Core.dll
 0001:00005dfe       ??0QString@@QAE@XZ         10006dfe f   Qt5Core:Qt5Core.dll
 0001:00005e04       ??0QString@@QAE@ABV0@@Z    10006e04 f   Qt5Core:Qt5Core.dll
 0001:00005e0a       ??1QString@@QAE@XZ         10006e0a f   Qt5Core:Qt5Core.dll
 0001:00005e10       ?arg@QString@@QBE?AV1@ABV1@HVQChar@@@Z 10006e10 f   Qt5Core:Qt5Core.dll
 0001:00005e16       ?append@QString@@QAEAAV1@ABV1@@Z 10006e16 f   Qt5Core:Qt5Core.dll
 0001:00005e1c       ??YQString@@QAEAAV0@VQChar@@@Z 10006e1c f   Qt5Core:Qt5Core.dll
 0001:00005e22       ?fromUtf8@QString@@SA?AV1@PBDH@Z 10006e22 f   Qt5Core:Qt5Core.dll
 0001:00005e28       ?fromAscii_helper@QString@@CAPAU?$QTypedArrayData@G@@PBDH@Z 10006e28 f   Qt5Core:Qt5Core.dll
 0001:00005e2e       ?detach_grow@QListData@@QAEPAUData@1@PAHH@Z 10006e2e f   Qt5Core:Qt5Core.dll
 0001:00005e34       ?dispose@QListData@@SAXPAUData@1@@Z 10006e34 f   Qt5Core:Qt5Core.dll
 0001:00005e3a       ?append@QListData@@QAEPAPAXXZ 10006e3a f   Qt5Core:Qt5Core.dll
 0001:00005e40       ?reset@QIODevice@@UAE_NXZ  10006e40 f   Qt5Core:Qt5Core.dll
 0001:00005e46       ??0QDir@@QAE@ABVQString@@@Z 10006e46 f   Qt5Core:Qt5Core.dll
 0001:00005e4c       ??1QDir@@QAE@XZ            10006e4c f   Qt5Core:Qt5Core.dll
 0001:00005e52       ?remove@QDir@@QAE_NABVQString@@@Z 10006e52 f   Qt5Core:Qt5Core.dll
 0001:00005e58       ?separator@QDir@@SA?AVQChar@@XZ 10006e58 f   Qt5Core:Qt5Core.dll
 0001:00005e5e       ??0QTemporaryFile@@QAE@XZ  10006e5e f   Qt5Core:Qt5Core.dll
 0001:00005e64       ??1QTemporaryFile@@UAE@XZ  10006e64 f   Qt5Core:Qt5Core.dll
 0001:00005e6a       ?childEvent@QObject@@MAEXPAVQChildEvent@@@Z 10006e6a f   Qt5Core:Qt5Core.dll
 0001:00005e70       ?connectNotify@QObject@@MAEXABVQMetaMethod@@@Z 10006e70 f   Qt5Core:Qt5Core.dll
 0001:00005e76       ?customEvent@QObject@@MAEXPAVQEvent@@@Z 10006e76 f   Qt5Core:Qt5Core.dll
 0001:00005e7c       ?disconnectNotify@QObject@@MAEXABVQMetaMethod@@@Z 10006e7c f   Qt5Core:Qt5Core.dll
 0001:00005e82       ?event@QObject@@UAE_NPAVQEvent@@@Z 10006e82 f   Qt5Core:Qt5Core.dll
 0001:00005e88       ?eventFilter@QObject@@UAE_NPAV1@PAVQEvent@@@Z 10006e88 f   Qt5Core:Qt5Core.dll
 0001:00005e8e       ?timerEvent@QObject@@MAEXPAVQTimerEvent@@@Z 10006e8e f   Qt5Core:Qt5Core.dll
 0001:00005e94       ?tr@QMetaObject@@QBE?AVQString@@PBD0H@Z 10006e94 f   Qt5Core:Qt5Core.dll
 0001:00005e9a       ?open@QTemporaryFile@@QAE_NXZ 10006e9a f   Qt5Core:Qt5Core.dll
 0001:00005ea0       ??0QTextStream@@QAE@PAVQIODevice@@@Z 10006ea0 f   Qt5Core:Qt5Core.dll
 0001:00005ea6       ??1QTextStream@@UAE@XZ     10006ea6 f   Qt5Core:Qt5Core.dll
 0001:00005eac       ??6QTextStream@@QAEAAV0@D@Z 10006eac f   Qt5Core:Qt5Core.dll
 0001:00005eb2       ??6QTextStream@@QAEAAV0@H@Z 10006eb2 f   Qt5Core:Qt5Core.dll
 0001:00005eb8       ??6QTextStream@@QAEAAV0@PBD@Z 10006eb8 f   Qt5Core:Qt5Core.dll
 0001:00005ebe       ??0QMessageLogger@@QAE@PBDH0@Z 10006ebe f   Qt5Core:Qt5Core.dll
 0001:00005ec4       ?debug@QMessageLogger@@QBAXPBDZZ 10006ec4 f   Qt5Core:Qt5Core.dll
 0001:00005eca       ??0QByteArray@@QAE@XZ      10006eca f   Qt5Core:Qt5Core.dll
 0001:00005ed0       ??1QByteArray@@QAE@XZ      10006ed0 f   Qt5Core:Qt5Core.dll
 0001:00005ed6       ??4QByteArray@@QAEAAV0@$$QAV0@@Z 10006ed6 f   Qt5Core:Qt5Core.dll
 0001:00005edc       ?data@QByteArray@@QAEPADXZ 10006edc f   Qt5Core:Qt5Core.dll
 0001:00005ee2       ?toLatin1@QString@@QBE?AVQByteArray@@XZ 10006ee2 f   Qt5Core:Qt5Core.dll
 0001:00005ee8       ?toLocal8Bit@QString@@QBE?AVQByteArray@@XZ 10006ee8 f   Qt5Core:Qt5Core.dll
 0001:00005eee       ?detach@QListData@@QAEPAUData@1@H@Z 10006eee f   Qt5Core:Qt5Core.dll
 0001:00005ef4       ??0QFile@@QAE@ABVQString@@@Z 10006ef4 f   Qt5Core:Qt5Core.dll
 0001:00005efa       ??1QFile@@UAE@XZ           10006efa f   Qt5Core:Qt5Core.dll
 0001:00005f00       ?open@QFile@@UAE_NV?$QFlags@W4OpenModeFlag@QIODevice@@@@@Z 10006f00 f   Qt5Core:Qt5Core.dll
 0001:00005f06       ?atEnd@QTextStream@@QBE_NXZ 10006f06 f   Qt5Core:Qt5Core.dll
 0001:00005f0c       ?readLine@QTextStream@@QAE?AVQString@@_J@Z 10006f0c f   Qt5Core:Qt5Core.dll
 0001:00005f12       ??5QTextStream@@QAEAAV0@AAH@Z 10006f12 f   Qt5Core:Qt5Core.dll
 0001:00005f18       ??5QTextStream@@QAEAAV0@AAN@Z 10006f18 f   Qt5Core:Qt5Core.dll
 0001:00005f1e       ??5QTextStream@@QAEAAV0@AAVQByteArray@@@Z 10006f1e f   Qt5Core:Qt5Core.dll
 0001:00005f24       ?append@QByteArray@@QAEAAV1@D@Z 10006f24 f   Qt5Core:Qt5Core.dll
 0001:00005f2a       ??5QTextStream@@QAEAAV0@AAM@Z 10006f2a f   Qt5Core:Qt5Core.dll
 0001:00005f30       ?dynamicMetaObject@QObjectData@@QBEPAUQMetaObject@@XZ 10006f30 f   Qt5Core:Qt5Core.dll
 0001:00005f36       ?qRegisterResourceData@@YA_NHPBE00@Z 10006f36 f   Qt5Core:Qt5Core.dll
 0001:00005f3c       ?qUnregisterResourceData@@YA_NHPBE00@Z 10006f3c f   Qt5Core:Qt5Core.dll
 0001:00005f42       ?_Xbad_alloc@std@@YAXXZ    10006f42 f   msvcprt:MSVCP120.dll
 0001:00005f48       ?_Xlength_error@std@@YAXPBD@Z 10006f48 f   msvcprt:MSVCP120.dll
 0001:00005f4e       ?_Xout_of_range@std@@YAXPBD@Z 10006f4e f   msvcprt:MSVCP120.dll
 0001:00005f54       ?_Syserror_map@std@@YAPBDH@Z 10006f54 f   msvcprt:MSVCP120.dll
 0001:00005f5a       ?_Winerror_map@std@@YAPBDH@Z 10006f5a f   msvcprt:MSVCP120.dll
 0001:00005f60       __purecall                 10006f60 f   MSVCRT:MSVCR120.dll
 0001:00005f66       ??2@YAPAXI@Z               10006f66 f   MSVCRT:MSVCR120.dll
 0001:00005f6c       ??3@YAXPAX@Z               10006f6c f   MSVCRT:MSVCR120.dll
 0001:00005f72       ___atonexitinit            10006f72 f   MSVCRT:atonexit.obj
 0001:00005fae       __onexit                   10006fae f   MSVCRT:atonexit.obj
 0001:00006057       _atexit                    10007057 f   MSVCRT:atonexit.obj
 0001:0000606c       _memmove                   1000706c f   MSVCRT:MSVCR120.dll
 0001:00006072       __hypot                    10007072 f   MSVCRT:MSVCR120.dll
 0001:00006078       @__security_check_cookie@4 10007078 f   MSVCRT:secchk.obj
 0001:00006088       __CxxThrowException@8      10007088 f   MSVCRT:MSVCR120.dll
 0001:0000608e       ___CxxFrameHandler3        1000708e f   MSVCRT:MSVCR120.dll
 0001:000060a0       __alloca_probe             100070a0 f   MSVCRT:chkstk.obj
 0001:000060a0       __chkstk                   100070a0 f   MSVCRT:chkstk.obj
 0001:000060cc       _memcpy                    100070cc f   MSVCRT:MSVCR120.dll
 0001:000060d2       ??0type_info@@AAE@ABV0@@Z  100070d2 f   MSVCRT:ti_inst.obj
 0001:000060dd       ??4type_info@@AAEAAV0@ABV0@@Z 100070dd f   MSVCRT:ti_inst.obj
 0001:000060e2       ??_Etype_info@@UAEPAXI@Z   100070e2 f i MSVCRT:ti_inst.obj
 0001:00006130       _fclose                    10007130 f   MSVCRT:MSVCR120.dll
 0001:00006136       _fopen                     10007136 f   MSVCRT:MSVCR120.dll
 0001:0000613c       _fprintf                   1000713c f   MSVCRT:MSVCR120.dll
 0001:00006142       _putc                      10007142 f   MSVCRT:MSVCR120.dll
 0001:00006148       _calloc                    10007148 f   MSVCRT:MSVCR120.dll
 0001:0000614e       _free                      1000714e f   MSVCRT:MSVCR120.dll
 0001:00006154       _malloc                    10007154 f   MSVCRT:MSVCR120.dll
 0001:0000615a       _sscanf                    1000715a f   MSVCRT:MSVCR120.dll
 0001:00006160       _strncmp                   10007160 f   MSVCRT:MSVCR120.dll
 0001:00006166       __libm_sse2_exp_precise    10007166 f   MSVCRT:MSVCR120.dll
 0001:0000616c       _atof                      1000716c f   MSVCRT:MSVCR120.dll
 0001:00006172       _atoi                      10007172 f   MSVCRT:MSVCR120.dll
 0001:00006178       _feof                      10007178 f   MSVCRT:MSVCR120.dll
 0001:0000617e       _fgets                     1000717e f   MSVCRT:MSVCR120.dll
 0001:00006184       _fputs                     10007184 f   MSVCRT:MSVCR120.dll
 0001:0000618a       ___iob_func                1000718a f   MSVCRT:MSVCR120.dll
 0001:00006190       _isalpha                   10007190 f   MSVCRT:MSVCR120.dll
 0001:000061e2       _NtCurrentTeb              100071e2 f i MSVCRT:crtdll.obj
 0001:000061e9       __CRT_INIT@12              100071e9 f   MSVCRT:crtdll.obj
 0001:000063e0       __DllMainCRTStartup@12     100073e0 f   MSVCRT:crtdll.obj
 0001:00006536       __lock                     10007536 f   MSVCRT:MSVCR120.dll
 0001:0000653c       __unlock                   1000753c f   MSVCRT:MSVCR120.dll
 0001:00006542       __calloc_crt               10007542 f   MSVCRT:MSVCR120.dll
 0001:00006548       ___dllonexit               10007548 f   MSVCRT:MSVCR120.dll
 0001:00006550       __SEH_prolog4              10007550 f   MSVCRT:sehprolg4.obj
 0001:00006595       __SEH_epilog4              10007595 f   MSVCRT:sehprolg4.obj
 0001:000065a9       __except_handler4          100075a9 f   MSVCRT:chandler4gs.obj
 0001:000065cc       ___raise_securityfailure   100075cc f   MSVCRT:gs_report.obj
 0001:00006609       ___report_gsfailure        10007609 f   MSVCRT:gs_report.obj
 0001:00006704       ___report_rangecheckfailure 10007704 f   MSVCRT:gs_report.obj
 0001:00006710       ___report_securityfailure  10007710 f   MSVCRT:gs_report.obj
 0001:000067e0       ___report_securityfailureEx 100077e0 f   MSVCRT:gs_report.obj
 0001:000068f6       ??_M@YGXPAXIHP6EX0@Z@Z     100078f6 f   MSVCRT:ehvecdtr.obj
 0001:0000697e       ?__ArrayUnwind@@YGXPAXIHP6EX0@Z@Z 1000797e f   MSVCRT:ehvecdtr.obj
 0001:000069dc       ??1type_info@@UAE@XZ       100079dc f   MSVCRT:MSVCR120.dll
 0001:000069e2       ___CppXcptFilter           100079e2 f   MSVCRT:MSVCR120.dll
 0001:000069e8       __amsg_exit                100079e8 f   MSVCRT:MSVCR120.dll
 0001:000069f0       __FindPESection            100079f0 f   MSVCRT:pesect.obj
 0001:00006a40       __IsNonwritableInCurrentImage 10007a40 f   MSVCRT:pesect.obj
 0001:00006b00       __ValidateImageBase        10007b00 f   MSVCRT:pesect.obj
 0001:00006b31       ___security_init_cookie    10007b31 f   MSVCRT:gs_support.obj
 0001:00006bcd       _DllMain@12                10007bcd f   MSVCRT:dllmain.obj
 0001:00006bf0       __malloc_crt               10007bf0 f   MSVCRT:MSVCR120.dll
 0001:00006bf6       __RTC_Initialize           10007bf6 f   MSVCRT:initsect.obj
 0001:00006c16       __RTC_Terminate            10007c16 f   MSVCRT:initsect.obj
 0001:00006c36       __initterm                 10007c36 f   MSVCRT:MSVCR120.dll
 0001:00006c3c       __initterm_e               10007c3c f   MSVCRT:MSVCR120.dll
 0001:00006c42       ___clean_type_info_names   10007c42 f   MSVCRT:tncleanup.obj
 0001:00006c4e       __except_handler4_common   10007c4e f   MSVCRT:MSVCR120.dll
 0001:00006c54       __crt_debugger_hook        10007c54 f   MSVCRT:MSVCR120.dll
 0001:00006c5a       ___crtUnhandledException   10007c5a f   MSVCRT:MSVCR120.dll
 0001:00006c60       ___crtTerminateProcess     10007c60 f   MSVCRT:MSVCR120.dll
 0001:00006c66       ?terminate@@YAXXZ          10007c66 f   MSVCRT:MSVCR120.dll
 0001:00006c6c       ___clean_type_info_names_internal 10007c6c f   MSVCRT:MSVCR120.dll
 0001:00006c72       _EncodePointer@4           10007c72 f   kernel32:KERNEL32.dll
 0001:00006c78       _DecodePointer@4           10007c78 f   kernel32:KERNEL32.dll
 0001:00006c7e       _IsDebuggerPresent@0       10007c7e f   kernel32:KERNEL32.dll
 0001:00006c84       _IsProcessorFeaturePresent@4 10007c84 f   kernel32:KERNEL32.dll
 0001:00006c8a       _QueryPerformanceCounter@4 10007c8a f   kernel32:KERNEL32.dll
 0001:00006c90       _GetCurrentProcessId@0     10007c90 f   kernel32:KERNEL32.dll
 0001:00006c96       _GetCurrentThreadId@0      10007c96 f   kernel32:KERNEL32.dll
 0001:00006c9c       _GetSystemTimeAsFileTime@4 10007c9c f   kernel32:KERNEL32.dll
 0001:00006ca2       _DisableThreadLibraryCalls@4 10007ca2 f   kernel32:KERNEL32.dll
 0002:00000000       __imp__DisableThreadLibraryCalls@4 10009000     kernel32:KERNEL32.dll
 0002:00000004       __imp__GetSystemTimeAsFileTime@4 10009004     kernel32:KERNEL32.dll
 0002:00000008       __imp__GetCurrentThreadId@0 10009008     kernel32:KERNEL32.dll
 0002:0000000c       __imp__GetCurrentProcessId@0 1000900c     kernel32:KERNEL32.dll
 0002:00000010       __imp__QueryPerformanceCounter@4 10009010     kernel32:KERNEL32.dll
 0002:00000014       __imp__IsProcessorFeaturePresent@4 10009014     kernel32:KERNEL32.dll
 0002:00000018       __imp__IsDebuggerPresent@0 10009018     kernel32:KERNEL32.dll
 0002:0000001c       __imp__DecodePointer@4     1000901c     kernel32:KERNEL32.dll
 0002:00000020       __imp__EncodePointer@4     10009020     kernel32:KERNEL32.dll
 0002:00000024       \177KERNEL32_NULL_THUNK_DATA 10009024     kernel32:KERNEL32.dll
 0002:00000028       __imp_?_Syserror_map@std@@YAPBDH@Z 10009028     msvcprt:MSVCP120.dll
 0002:0000002c       __imp_?_Xout_of_range@std@@YAXPBD@Z 1000902c     msvcprt:MSVCP120.dll
 0002:00000030       __imp_?_Xlength_error@std@@YAXPBD@Z 10009030     msvcprt:MSVCP120.dll
 0002:00000034       __imp_?_Xbad_alloc@std@@YAXXZ 10009034     msvcprt:MSVCP120.dll
 0002:00000038       __imp_?_Winerror_map@std@@YAPBDH@Z 10009038     msvcprt:MSVCP120.dll
 0002:0000003c       \177MSVCP120_NULL_THUNK_DATA 1000903c     msvcprt:MSVCP120.dll
 0002:00000040       __imp___initterm_e         10009040     MSVCRT:MSVCR120.dll
 0002:00000044       __imp___initterm           10009044     MSVCRT:MSVCR120.dll
 0002:00000048       __imp___malloc_crt         10009048     MSVCRT:MSVCR120.dll
 0002:0000004c       __imp___amsg_exit          1000904c     MSVCRT:MSVCR120.dll
 0002:00000050       __imp____CppXcptFilter     10009050     MSVCRT:MSVCR120.dll
 0002:00000054       __imp_??1type_info@@UAE@XZ 10009054     MSVCRT:MSVCR120.dll
 0002:00000058       __imp___onexit             10009058     MSVCRT:MSVCR120.dll
 0002:0000005c       __imp____dllonexit         1000905c     MSVCRT:MSVCR120.dll
 0002:00000060       __imp___calloc_crt         10009060     MSVCRT:MSVCR120.dll
 0002:00000064       __imp___unlock             10009064     MSVCRT:MSVCR120.dll
 0002:00000068       __imp___lock               10009068     MSVCRT:MSVCR120.dll
 0002:0000006c       __imp__isalpha             1000906c     MSVCRT:MSVCR120.dll
 0002:00000070       __imp____iob_func          10009070     MSVCRT:MSVCR120.dll
 0002:00000074       __imp__fputs               10009074     MSVCRT:MSVCR120.dll
 0002:00000078       __imp__fgets               10009078     MSVCRT:MSVCR120.dll
 0002:0000007c       __imp__feof                1000907c     MSVCRT:MSVCR120.dll
 0002:00000080       __imp__atoi                10009080     MSVCRT:MSVCR120.dll
 0002:00000084       __imp__atof                10009084     MSVCRT:MSVCR120.dll
 0002:00000088       __imp___libm_sse2_exp_precise 10009088     MSVCRT:MSVCR120.dll
 0002:0000008c       __imp__strncmp             1000908c     MSVCRT:MSVCR120.dll
 0002:00000090       __imp__sscanf              10009090     MSVCRT:MSVCR120.dll
 0002:00000094       __imp__malloc              10009094     MSVCRT:MSVCR120.dll
 0002:00000098       __imp__free                10009098     MSVCRT:MSVCR120.dll
 0002:0000009c       __imp__calloc              1000909c     MSVCRT:MSVCR120.dll
 0002:000000a0       __imp__putc                100090a0     MSVCRT:MSVCR120.dll
 0002:000000a4       __imp__fprintf             100090a4     MSVCRT:MSVCR120.dll
 0002:000000a8       __imp__fopen               100090a8     MSVCRT:MSVCR120.dll
 0002:000000ac       __imp__fclose              100090ac     MSVCRT:MSVCR120.dll
 0002:000000b0       __imp__memcpy              100090b0     MSVCRT:MSVCR120.dll
 0002:000000b4       __imp____CxxFrameHandler3  100090b4     MSVCRT:MSVCR120.dll
 0002:000000b8       __imp___CxxThrowException@8 100090b8     MSVCRT:MSVCR120.dll
 0002:000000bc       __imp___hypot              100090bc     MSVCRT:MSVCR120.dll
 0002:000000c0       __imp__memmove             100090c0     MSVCRT:MSVCR120.dll
 0002:000000c4       __imp_??3@YAXPAX@Z         100090c4     MSVCRT:MSVCR120.dll
 0002:000000c8       __imp_??2@YAPAXI@Z         100090c8     MSVCRT:MSVCR120.dll
 0002:000000cc       __imp___purecall           100090cc     MSVCRT:MSVCR120.dll
 0002:000000d0       __imp___except_handler4_common 100090d0     MSVCRT:MSVCR120.dll
 0002:000000d4       __imp_?terminate@@YAXXZ    100090d4     MSVCRT:MSVCR120.dll
 0002:000000d8       __imp____crtTerminateProcess 100090d8     MSVCRT:MSVCR120.dll
 0002:000000dc       __imp____crtUnhandledException 100090dc     MSVCRT:MSVCR120.dll
 0002:000000e0       __imp____clean_type_info_names_internal 100090e0     MSVCRT:MSVCR120.dll
 0002:000000e4       __imp___crt_debugger_hook  100090e4     MSVCRT:MSVCR120.dll
 0002:000000e8       \177MSVCR120_NULL_THUNK_DATA 100090e8     MSVCRT:MSVCR120.dll
 0002:000000ec       __imp_??0QChar@@QAE@UQLatin1Char@@@Z 100090ec     Qt5Core:Qt5Core.dll
 0002:000000f0       __imp_?constData@QByteArray@@QBEPBDXZ 100090f0     Qt5Core:Qt5Core.dll
 0002:000000f4       __imp_?unlock@QMutexLocker@@QAEXXZ 100090f4     Qt5Core:Qt5Core.dll
 0002:000000f8       __imp_??0QString@@QAE@ABV0@@Z 100090f8     Qt5Core:Qt5Core.dll
 0002:000000fc       __imp_??1QString@@QAE@XZ   100090fc     Qt5Core:Qt5Core.dll
 0002:00000100       __imp_?arg@QString@@QBE?AV1@ABV1@HVQChar@@@Z 10009100     Qt5Core:Qt5Core.dll
 0002:00000104       __imp_?append@QString@@QAEAAV1@ABV1@@Z 10009104     Qt5Core:Qt5Core.dll
 0002:00000108       __imp_??YQString@@QAEAAV0@VQChar@@@Z 10009108     Qt5Core:Qt5Core.dll
 0002:0000010c       __imp_?fromUtf8@QString@@SA?AV1@PBDH@Z 1000910c     Qt5Core:Qt5Core.dll
 0002:00000110       __imp_??1QMutexLocker@@QAE@XZ 10009110     Qt5Core:Qt5Core.dll
 0002:00000114       __imp_?detach_grow@QListData@@QAEPAUData@1@PAHH@Z 10009114     Qt5Core:Qt5Core.dll
 0002:00000118       __imp_?dispose@QListData@@SAXPAUData@1@@Z 10009118     Qt5Core:Qt5Core.dll
 0002:0000011c       __imp_?append@QListData@@QAEPAPAXXZ 1000911c     Qt5Core:Qt5Core.dll
 0002:00000120       __imp_?reset@QIODevice@@UAE_NXZ 10009120     Qt5Core:Qt5Core.dll
 0002:00000124       __imp_??0QDir@@QAE@ABVQString@@@Z 10009124     Qt5Core:Qt5Core.dll
 0002:00000128       __imp_??1QDir@@QAE@XZ      10009128     Qt5Core:Qt5Core.dll
 0002:0000012c       __imp_?remove@QDir@@QAE_NABVQString@@@Z 1000912c     Qt5Core:Qt5Core.dll
 0002:00000130       __imp_?separator@QDir@@SA?AVQChar@@XZ 10009130     Qt5Core:Qt5Core.dll
 0002:00000134       __imp_??0QTemporaryFile@@QAE@XZ 10009134     Qt5Core:Qt5Core.dll
 0002:00000138       __imp_??1QTemporaryFile@@UAE@XZ 10009138     Qt5Core:Qt5Core.dll
 0002:0000013c       __imp_?childEvent@QObject@@MAEXPAVQChildEvent@@@Z 1000913c     Qt5Core:Qt5Core.dll
 0002:00000140       __imp_?connectNotify@QObject@@MAEXABVQMetaMethod@@@Z 10009140     Qt5Core:Qt5Core.dll
 0002:00000144       __imp_?customEvent@QObject@@MAEXPAVQEvent@@@Z 10009144     Qt5Core:Qt5Core.dll
 0002:00000148       __imp_?disconnectNotify@QObject@@MAEXABVQMetaMethod@@@Z 10009148     Qt5Core:Qt5Core.dll
 0002:0000014c       __imp_?event@QObject@@UAE_NPAVQEvent@@@Z 1000914c     Qt5Core:Qt5Core.dll
 0002:00000150       __imp_?eventFilter@QObject@@UAE_NPAV1@PAVQEvent@@@Z 10009150     Qt5Core:Qt5Core.dll
 0002:00000154       __imp_?timerEvent@QObject@@MAEXPAVQTimerEvent@@@Z 10009154     Qt5Core:Qt5Core.dll
 0002:00000158       __imp_?shared_null@QListData@@2UData@1@B 10009158     Qt5Core:Qt5Core.dll
 0002:0000015c       __imp_?tr@QMetaObject@@QBE?AVQString@@PBD0H@Z 1000915c     Qt5Core:Qt5Core.dll
 0002:00000160       __imp_?open@QTemporaryFile@@QAE_NXZ 10009160     Qt5Core:Qt5Core.dll
 0002:00000164       __imp_??0QTextStream@@QAE@PAVQIODevice@@@Z 10009164     Qt5Core:Qt5Core.dll
 0002:00000168       __imp_??1QTextStream@@UAE@XZ 10009168     Qt5Core:Qt5Core.dll
 0002:0000016c       __imp_??6QTextStream@@QAEAAV0@D@Z 1000916c     Qt5Core:Qt5Core.dll
 0002:00000170       __imp_??6QTextStream@@QAEAAV0@H@Z 10009170     Qt5Core:Qt5Core.dll
 0002:00000174       __imp_??6QTextStream@@QAEAAV0@PBD@Z 10009174     Qt5Core:Qt5Core.dll
 0002:00000178       __imp_??0QMessageLogger@@QAE@PBDH0@Z 10009178     Qt5Core:Qt5Core.dll
 0002:0000017c       __imp_?debug@QMessageLogger@@QBAXPBDZZ 1000917c     Qt5Core:Qt5Core.dll
 0002:00000180       __imp_??0QByteArray@@QAE@XZ 10009180     Qt5Core:Qt5Core.dll
 0002:00000184       __imp_??1QByteArray@@QAE@XZ 10009184     Qt5Core:Qt5Core.dll
 0002:00000188       __imp_??4QByteArray@@QAEAAV0@$$QAV0@@Z 10009188     Qt5Core:Qt5Core.dll
 0002:0000018c       __imp_?data@QByteArray@@QAEPADXZ 1000918c     Qt5Core:Qt5Core.dll
 0002:00000190       __imp_?toLatin1@QString@@QBE?AVQByteArray@@XZ 10009190     Qt5Core:Qt5Core.dll
 0002:00000194       __imp_?toLocal8Bit@QString@@QBE?AVQByteArray@@XZ 10009194     Qt5Core:Qt5Core.dll
 0002:00000198       __imp_?detach@QListData@@QAEPAUData@1@H@Z 10009198     Qt5Core:Qt5Core.dll
 0002:0000019c       __imp_??0QFile@@QAE@ABVQString@@@Z 1000919c     Qt5Core:Qt5Core.dll
 0002:000001a0       __imp_??1QFile@@UAE@XZ     100091a0     Qt5Core:Qt5Core.dll
 0002:000001a4       __imp_?open@QFile@@UAE_NV?$QFlags@W4OpenModeFlag@QIODevice@@@@@Z 100091a4     Qt5Core:Qt5Core.dll
 0002:000001a8       __imp_?atEnd@QTextStream@@QBE_NXZ 100091a8     Qt5Core:Qt5Core.dll
 0002:000001ac       __imp_?readLine@QTextStream@@QAE?AVQString@@_J@Z 100091ac     Qt5Core:Qt5Core.dll
 0002:000001b0       __imp_??5QTextStream@@QAEAAV0@AAH@Z 100091b0     Qt5Core:Qt5Core.dll
 0002:000001b4       __imp_??5QTextStream@@QAEAAV0@AAN@Z 100091b4     Qt5Core:Qt5Core.dll
 0002:000001b8       __imp_??5QTextStream@@QAEAAV0@AAVQByteArray@@@Z 100091b8     Qt5Core:Qt5Core.dll
 0002:000001bc       __imp_?append@QByteArray@@QAEAAV1@D@Z 100091bc     Qt5Core:Qt5Core.dll
 0002:000001c0       __imp_??5QTextStream@@QAEAAV0@AAM@Z 100091c0     Qt5Core:Qt5Core.dll
 0002:000001c4       __imp_?dynamicMetaObject@QObjectData@@QBEPAUQMetaObject@@XZ 100091c4     Qt5Core:Qt5Core.dll
 0002:000001c8       __imp_?qRegisterResourceData@@YA_NHPBE00@Z 100091c8     Qt5Core:Qt5Core.dll
 0002:000001cc       __imp_?qUnregisterResourceData@@YA_NHPBE00@Z 100091cc     Qt5Core:Qt5Core.dll
 0002:000001d0       __imp_??0QMutexLocker@@QAE@PAVQBasicMutex@@@Z 100091d0     Qt5Core:Qt5Core.dll
 0002:000001d4       __imp_??1QMutex@@QAE@XZ    100091d4     Qt5Core:Qt5Core.dll
 0002:000001d8       __imp_??0QMutex@@QAE@W4RecursionMode@0@@Z 100091d8     Qt5Core:Qt5Core.dll
 0002:000001dc       __imp_?fromAscii_helper@QString@@CAPAU?$QTypedArrayData@G@@PBDH@Z 100091dc     Qt5Core:Qt5Core.dll
 0002:000001e0       __imp_??0QString@@QAE@XZ   100091e0     Qt5Core:Qt5Core.dll
 0002:000001e4       \177Qt5Core_NULL_THUNK_DATA 100091e4     Qt5Core:Qt5Core.dll
 0002:000001e8       __imp_?setRgb@QColor@@QAEXHHHH@Z 100091e8     Qt5Gui:Qt5Gui.dll
 0002:000001ec       \177Qt5Gui_NULL_THUNK_DATA 100091ec     Qt5Gui:Qt5Gui.dll
 0002:000001f0       __imp_??0SecStructPredictTask@U2@@QAE@ABVQByteArray@@@Z 100091f0     U2Algorithm:U2Algorithm.dll
 0002:000001f4       __imp_??1SecStructPredictTask@U2@@UAE@XZ 100091f4     U2Algorithm:U2Algorithm.dll
 0002:000001f8       __imp_?staticMetaObject@SecStructPredictTask@U2@@2UQMetaObject@@B 100091f8     U2Algorithm:U2Algorithm.dll
 0002:000001fc       __imp_?qt_metacall@SecStructPredictTask@U2@@UAEHW4Call@QMetaObject@@HPAPAX@Z 100091fc     U2Algorithm:U2Algorithm.dll
 0002:00000200       __imp_?qt_metacast@SecStructPredictTask@U2@@UAEPAXPBD@Z 10009200     U2Algorithm:U2Algorithm.dll
 0002:00000204       __imp_??_7SecStructPredictTaskFactory@U2@@6B@ 10009204     U2Algorithm:U2Algorithm.dll
 0002:00000208       __imp_?registerAlgorithm@SecStructPredictAlgRegistry@U2@@QAE_NPAVSecStructPredictTaskFactory@2@ABVQString@@@Z 10009208     U2Algorithm:U2Algorithm.dll
 0002:0000020c       __imp_?prepare@SecStructPredictTask@U2@@UAEXXZ 1000920c     U2Algorithm:U2Algorithm.dll
 0002:00000210       __imp_?tr@SecStructPredictTask@U2@@SA?AVQString@@PBD0H@Z 10009210     U2Algorithm:U2Algorithm.dll
 0002:00000214       \177U2Algorithm_NULL_THUNK_DATA 10009214     U2Algorithm:U2Algorithm.dll
 0002:00000218       __imp_??1GCounter@U2@@UAE@XZ 10009218     U2Core:U2Core.dll
 0002:0000021c       __imp_??0GReportableCounter@U2@@QAE@ABVQString@@0N@Z 1000921c     U2Core:U2Core.dll
 0002:00000220       __imp_?staticMetaObject@Plugin@U2@@2UQMetaObject@@B 10009220     U2Core:U2Core.dll
 0002:00000224       __imp_?qt_metacall@Plugin@U2@@UAEHW4Call@QMetaObject@@HPAPAX@Z 10009224     U2Core:U2Core.dll
 0002:00000228       __imp_?qt_metacast@Plugin@U2@@UAEPAXPBD@Z 10009228     U2Core:U2Core.dll
 0002:0000022c       __imp_?SecStructTypeQualifierName@BioStruct3D@U2@@2VQString@@A 1000922c     U2Core:U2Core.dll
 0002:00000230       __imp_?changeSettings@AnnotationSettingsRegistry@U2@@QAEXABV?$QList@PAVAnnotationSettings@U2@@@@_N@Z 10009230     U2Core:U2Core.dll
 0002:00000234       __imp_??0AnnotationSettings@U2@@QAE@ABVQString@@_NABVQColor@@1@Z 10009234     U2Core:U2Core.dll
 0002:00000238       __imp_?getSecStructPredictAlgRegistry@AppContext@U2@@SAPAVSecStructPredictAlgRegistry@2@XZ 10009238     U2Core:U2Core.dll
 0002:0000023c       __imp_?getAnnotationsSettingsRegistry@AppContext@U2@@SAPAVAnnotationSettingsRegistry@2@XZ 1000923c     U2Core:U2Core.dll
 0002:00000240       __imp_??1Plugin@U2@@UAE@XZ 10009240     U2Core:U2Core.dll
 0002:00000244       __imp_??0Plugin@U2@@QAE@ABVQString@@0_NW4PluginState@1@@Z 10009244     U2Core:U2Core.dll
 0002:00000248       __imp_?setReportingSupported@Task@U2@@UAEX_N@Z 10009248     U2Core:U2Core.dll
 0002:0000024c       __imp_?setReportingEnabled@Task@U2@@UAEX_N@Z 1000924c     U2Core:U2Core.dll
 0002:00000250       __imp_?setNotificationReport@Task@U2@@UAEX_N@Z 10009250     U2Core:U2Core.dll
 0002:00000254       __imp_?setNoAutoDelete@Task@U2@@UAEX_N@Z 10009254     U2Core:U2Core.dll
 0002:00000258       __imp_?setCollectChildrensWarningsFlag@Task@U2@@UAEX_N@Z 10009258     U2Core:U2Core.dll
 0002:0000025c       __imp_?report@Task@U2@@UAE?AW4ReportResult@12@XZ 1000925c     U2Core:U2Core.dll
 0002:00000260       __imp_?propagateSubtaskError@Task@U2@@UAE_NXZ 10009260     U2Core:U2Core.dll
 0002:00000264       __imp_?onSubTaskFinished@Task@U2@@MAE?AV?$QList@PAVTask@U2@@@@PAV12@@Z 10009264     U2Core:U2Core.dll
 0002:00000268       __imp_?isTopLevelTask@Task@U2@@UBE_NXZ 10009268     U2Core:U2Core.dll
 0002:0000026c       __imp_?isReportingSupported@Task@U2@@UBE_NXZ 1000926c     U2Core:U2Core.dll
 0002:00000270       __imp_?isReportingEnabled@Task@U2@@UBE_NXZ 10009270     U2Core:U2Core.dll
 0002:00000274       __imp_?isNotificationReport@Task@U2@@UBE_NXZ 10009274     U2Core:U2Core.dll
 0002:00000278       __imp_?hasWarning@Task@U2@@UBE_NXZ 10009278     U2Core:U2Core.dll
 0002:0000027c       __imp_?hasSubtasksWithErrors@Task@U2@@UBE_NXZ 1000927c     U2Core:U2Core.dll
 0002:00000280       __imp_?getWarnings@Task@U2@@UBE?AVQStringList@@XZ 10009280     U2Core:U2Core.dll
 0002:00000284       __imp_?getTopLevelParentTask@Task@U2@@UAEPAV12@XZ 10009284     U2Core:U2Core.dll
 0002:00000288       __imp_?getTaskId@Task@U2@@UBE_JXZ 10009288     U2Core:U2Core.dll
 0002:0000028c       __imp_?getSubtaskWithErrors@Task@U2@@UBEPAV12@XZ 1000928c     U2Core:U2Core.dll
 0002:00000290       __imp_?getParentTask@Task@U2@@UBEPAV12@XZ 10009290     U2Core:U2Core.dll
 0002:00000294       __imp_?getNumParallelSubtasks@Task@U2@@UBEHXZ 10009294     U2Core:U2Core.dll
 0002:00000298       __imp_?generateReport@Task@U2@@UBE?AVQString@@XZ 10009298     U2Core:U2Core.dll
 0002:0000029c       __imp_?cleanup@Task@U2@@UAEXXZ 1000929c     U2Core:U2Core.dll
 0002:000002a0       __imp_??1Logger@U2@@UAE@XZ 100092a0     U2Core:U2Core.dll
 0002:000002a4       __imp_??0Logger@U2@@QAE@ABVQString@@@Z 100092a4     U2Core:U2Core.dll
 0002:000002a8       __imp_?getUserTemporaryDirPath@UserAppsSettings@U2@@QBE?AVQString@@XZ 100092a8     U2Core:U2Core.dll
 0002:000002ac       __imp_?getAppSettings@AppContext@U2@@SAPAVAppSettings@2@XZ 100092ac     U2Core:U2Core.dll
 0002:000002b0       __imp_??1AnnotationData@U2@@QAE@XZ 100092b0     U2Core:U2Core.dll
 0002:000002b4       \177U2Core_NULL_THUNK_DATA 100092b4     U2Core:U2Core.dll
 0002:000002b8       __imp_?saveAlgorithmResultsAsAnnotations@SecStructPredictUtils@U2@@SA?AV?$QList@V?$QSharedDataPointer@VAnnotationData@U2@@@@@@ABVQByteArray@@ABVQString@@@Z 100092b8     U2View:U2View.dll
 0002:000002bc       \177U2View_NULL_THUNK_DATA 100092bc     U2View:U2View.dll
 0002:000002c0       ___xc_a                    100092c0     MSVCRT:cinitexe.obj
 0002:000003e8       ___xc_z                    100093e8     MSVCRT:cinitexe.obj
 0002:000003ec       ___xi_a                    100093ec     MSVCRT:cinitexe.obj
 0002:000003f8       ___xi_z                    100093f8     MSVCRT:cinitexe.obj
 0002:00000438       ??_C@_00CNPNBAHC@?$AA@     10009438     PsipredAlgTask.obj
 0002:00000440       ??_7error_category@std@@6B@ 10009440     PsipredAlgTask.obj
 0002:0000045c       ??_7_Generic_error_category@std@@6B@ 1000945c     PsipredAlgTask.obj
 0002:00000474       ??_C@_07DCLBNMLN@generic?$AA@ 10009474     PsipredAlgTask.obj
 0002:0000047c       ??_C@_0O@BFJCFAAK@unknown?5error?$AA@ 1000947c     PsipredAlgTask.obj
 0002:00000490       ??_7_Iostream_error_category@std@@6B@ 10009490     PsipredAlgTask.obj
 0002:000004a8       ??_C@_08LLGCOLLL@iostream?$AA@ 100094a8     PsipredAlgTask.obj
 0002:000004b4       ??_C@_0BG@PADBLCHM@iostream?5stream?5error?$AA@ 100094b4     PsipredAlgTask.obj
 0002:000004d0       ??_7_System_error_category@std@@6B@ 100094d0     PsipredAlgTask.obj
 0002:000004e8       ??_C@_06FHFOAHML@system?$AA@ 100094e8     PsipredAlgTask.obj
 0002:000004f4       ??_7?$AbstractId@H@U2@@6B@ 100094f4     PsipredAlgTask.obj
 0002:00000500       ??_7AbstractInt32Id@U2@@6B@ 10009500     PsipredAlgTask.obj
 0002:0000050c       ??_7ServiceType@U2@@6B@    1000950c     PsipredAlgTask.obj
 0002:00000514       ??_C@_0L@JLHNEGIN@Algorithms?$AA@ 10009514     PsipredAlgTask.obj
 0002:00000520       ??_C@_07PGLPGHFC@Console?$AA@ 10009520     PsipredAlgTask.obj
 0002:00000528       ??_C@_0O@BOFHOPCF@Core?5Services?$AA@ 10009528     PsipredAlgTask.obj
 0002:00000538       ??_C@_0N@PPADAKBM@Input?1Output?$AA@ 10009538     PsipredAlgTask.obj
 0002:00000548       ??_C@_0M@KPPBKPKK@Performance?$AA@ 10009548     PsipredAlgTask.obj
 0002:00000554       ??_C@_07BFDHHBBI@Scripts?$AA@ 10009554     PsipredAlgTask.obj
 0002:0000055c       ??_C@_05EEGKELMG@Tasks?$AA@ 1000955c     PsipredAlgTask.obj
 0002:00000564       ??_C@_0P@NIIOBHGA@User?5Interface?$AA@ 10009564     PsipredAlgTask.obj
 0002:00000574       ??_C@_0N@JINCGGMN@User?5Actions?$AA@ 10009574     PsipredAlgTask.obj
 0002:00000588       ??_7PsipredAlgTask@U2@@6B@ 10009588     PsipredAlgTask.obj
 0002:00000614       ??_C@_0P@CPPPGNFA@PsipredAlgTask?$AA@ 10009614     PsipredAlgTask.obj
 0002:00000624       ??_C@_0DF@PCDHGCFJ@psipred?3?5sequence?5is?5too?5long?0?5m@ 10009624     PsipredAlgTask.obj
 0002:0000065c       ??_C@_0DC@BHELKIDI@psipred?3?5sequence?5is?5too?5short?0?5@ 1000965c     PsipredAlgTask.obj
 0002:00000690       ??_C@_0BC@LOFDAABB@psipred?5error?3?5?$CF1?$AA@ 10009690     PsipredAlgTask.obj
 0002:000006a4       ??_C@_0CB@ILKMJCEA@?3psipred?1datafiles?1weights_s?4dat@ 100096a4     PsipredAlgTask.obj
 0002:000006c8       ??_C@_0CC@JLCHLJHD@?3psipred?1datafiles?1weights_s?4dat@ 100096c8     PsipredAlgTask.obj
 0002:000006ec       ??_C@_0CC@ICDMIIDC@?3psipred?1datafiles?1weights_s?4dat@ 100096ec     PsipredAlgTask.obj
 0002:00000710       ??_C@_05LBJMNBOG@empty?$AA@ 10009710     PsipredAlgTask.obj
 0002:00000718       ??_C@_0CC@EHIIFIMM@?3psipred?1datafiles?1weights_p2?4da@ 10009718     PsipredAlgTask.obj
 0002:0000073c       ??_C@_01HIHLOKLC@1?$AA@    1000973c     PsipredAlgTask.obj
 0002:00000740       ??_C@_03HLLJOCDO@1?40?$AA@ 10009740     PsipredAlgTask.obj
 0002:00000744       ??_C@_0BA@HCAMPDEK@psipred_results?$AA@ 10009744     PsipredAlgTask.obj
 0002:00000754       ??_C@_09HCKPPOD@output?4ss?$AA@ 10009754     PsipredAlgTask.obj
 0002:00000760       ??_C@_0L@NEHEMNEM@output?4ss2?$AA@ 10009760     PsipredAlgTask.obj
 0002:0000076c       ??_C@_0BA@JFNIOLAK@string?5too?5long?$AA@ 1000976c     PsipredAlgTask.obj
 0002:0000077c       ??_C@_0BI@CFPLBAOH@invalid?5string?5position?$AA@ 1000977c     PsipredAlgTask.obj
 0002:00000798       __real@3ff0000000000000    10009798     PsipredAlgTask.obj
 0002:000007a4       ??_7PsipredPlugin@U2@@6B@  100097a4     PsipredPlugin.obj
 0002:000007d4       ??_7Factory@PsipredAlgTask@U2@@6B@ 100097d4     PsipredPlugin.obj
 0002:000007dc       ??_C@_0CP@OELKJOBL@PsiPred?5protein?5secondary?5struct@ 100097dc     PsipredPlugin.obj
 0002:0000080c       ??_C@_07ILCIEHMA@PsiPred?$AA@ 1000980c     PsipredPlugin.obj
 0002:00000814       ??_C@_0BI@PONJDEKM@ARNDCQEGHILKMFPSTWYVBZX?$AA@ 10009814     seq2mtx.obj
 0002:00000c54       ??_C@_0BL@INDPGPOC@XAXCDEFGHIKLMNPQRSTVWXYXXX?$AA@ 10009c54     seq2mtx.obj
 0002:00000c70       ??_C@_0BH@KNIJPLNL@Sequence?5length?5error?$CB?$AA@ 10009c70     seq2mtx.obj
 0002:00000c88       ??_C@_01NOFIACDB@w?$AA@    10009c88     seq2mtx.obj
 0002:00000c8c       ??_C@_0BN@LDOOAJGD@open?5file?5for?5writing?5failed?$AA@ 10009c8c     seq2mtx.obj
 0002:00000cac       ??_C@_03PMGGPEJJ@?$CFd?6?$AA@ 10009cac     seq2mtx.obj
 0002:00000cb0       ??_C@_0BK@GMEHHPHO@?60?60?60?60?60?60?60?60?60?60?60?60?6?$AA@ 10009cb0     seq2mtx.obj
 0002:00000ccc       ??_C@_04CJHBKKIA@?$CFd?5?5?$AA@ 10009ccc     seq2mtx.obj
 0002:00000cd4       ??_C@_08PBLOKGHP@?932768?5?5?$AA@ 10009cd4     seq2mtx.obj
 0002:00000ce0       ??_C@_02KNHHEEKP@?5?5?$AA@ 10009ce0     seq2mtx.obj
 0002:00000ce4       ??_C@_07FBCKBNBJ@?932768?5?$AA@ 10009ce4     seq2mtx.obj
 0002:00000cec       ??_C@_0BF@OHJIHCMG@init?3?5Out?5of?5Memory?$CB?$AA@ 10009cec     sspred_avpred.obj
 0002:00000d04       ??_C@_0CA@OODDDHD@failed?5opening?5file?5for?5writing?$AA@ 10009d04     sspred_avpred.obj
 0002:00000d24       ??_C@_0BO@BGDDCGOF@?$CF4d?5?$CFc?5?$CFc?5?5?$CF6?43f?5?$CF6?43f?5?$CF6?43f?6?$AA@ 10009d24     sspred_avpred.obj
 0002:00000d44       ??_C@_02DKCKIIND@?$CFs?$AA@ 10009d44     sspred_avpred.obj
 0002:00000d48       ??_C@_0CD@CEEGCNJ@Bad?5mtx?5file?5?9?5no?5sequence?5lengt@ 10009d48     sspred_avpred.obj
 0002:00000d6c       ??_C@_0BJ@PBBGNDFL@Input?5sequence?5too?5long?$CB?$AA@ 10009d6c     sspred_avpred.obj
 0002:00000d88       ??_C@_0BM@DFCFNHJF@Bad?5mtx?5file?5?9?5no?5sequence?$CB?$AA@ 10009d88     sspred_avpred.obj
 0002:00000da4       ??_C@_0DC@EEDNOHIB@?$CF?$CKd?$CFd?$CF?$CKd?$CFd?$CFd?$CFd?$CFd?$CFd?$CFd?$CFd?$CFd?$CFd?$CFd?$CFd?$CFd@ 10009da4     sspred_avpred.obj
 0002:00000dd8       ??_C@_0BA@OIPGHGKI@Bad?5mtx?5format?$CB?$AA@ 10009dd8     sspred_avpred.obj
 0002:00000de8       __real@3f800000            10009de8     sspred_avpred.obj
 0002:00000dec       __real@40000000            10009dec     sspred_avpred.obj
 0002:00000df0       __real@408f400000000000    10009df0     sspred_avpred.obj
 0002:00000e00       __xmm@80000000800000008000000080000000 10009e00     sspred_avpred.obj
 0002:00000e10       ??_C@_03GNPBBFFL@ALA?$AA@  10009e10     sspred_hmulti.obj
 0002:00000e14       ??_C@_03CNBDDMKH@ARG?$AA@  10009e14     sspred_hmulti.obj
 0002:00000e18       ??_C@_03PNBDONNJ@ASN?$AA@  10009e18     sspred_hmulti.obj
 0002:00000e1c       ??_C@_03CJFCNCAG@ASP?$AA@  10009e1c     sspred_hmulti.obj
 0002:00000e20       ??_C@_03KFOBMMJI@CYS?$AA@  10009e20     sspred_hmulti.obj
 0002:00000e24       ??_C@_03MPACFGEI@GLN?$AA@  10009e24     sspred_hmulti.obj
 0002:00000e28       ??_C@_03GGDEJNNC@GLU?$AA@  10009e28     sspred_hmulti.obj
 0002:00000e2c       ??_C@_03MKIBNCNO@GLY?$AA@  10009e2c     sspred_hmulti.obj
 0002:00000e30       ??_C@_03GOMGOIOJ@HIS?$AA@  10009e30     sspred_hmulti.obj
 0002:00000e34       ??_C@_03MMCJPILA@ILE?$AA@  10009e34     sspred_hmulti.obj
 0002:00000e38       ??_C@_03LOOECBFM@LEU?$AA@  10009e38     sspred_hmulti.obj
 0002:00000e3c       ??_C@_03PNICNMMO@LYS?$AA@  10009e3c     sspred_hmulti.obj
 0002:00000e40       ??_C@_03BPEDHHHI@MET?$AA@  10009e40     sspred_hmulti.obj
 0002:00000e44       ??_C@_03OGDBEIHJ@PHE?$AA@  10009e44     sspred_hmulti.obj
 0002:00000e48       ??_C@_03NGPIGFF@PRO?$AA@   10009e48     sspred_hmulti.obj
 0002:00000e4c       ??_C@_03PJNPPAFC@SER?$AA@  10009e4c     sspred_hmulti.obj
 0002:00000e50       ??_C@_03GMNAFLLI@THR?$AA@  10009e50     sspred_hmulti.obj
 0002:00000e54       ??_C@_03EPFHBPJM@TRP?$AA@  10009e54     sspred_hmulti.obj
 0002:00000e58       ??_C@_03HBDEJCPP@TYR?$AA@  10009e58     sspred_hmulti.obj
 0002:00000e5c       ??_C@_03BNEJJHGD@VAL?$AA@  10009e5c     sspred_hmulti.obj
 0002:00000e60       ??_C@_03BBKEAIF@?$DP?$DP?$DP?$AA@ 10009e60     sspred_hmulti.obj
 0002:00000e64       ??_C@_0BJ@LNCKNOJM@cannot?5open?5weights?5file?$AA@ 10009e64     sspred_hmulti.obj
 0002:00000e80       ??_C@_0BJ@PHPBHCEG@Cannot?5open?5output?5file?$CB?$AA@ 10009e80     sspred_hmulti.obj
 0002:00000e9c       ??_C@_0DC@NBKENGBC@?$CD?5PSIPRED?5VFORMAT?5?$CIPSIPRED?5V2?46?5@ 10009e9c     sspred_hmulti.obj
 0002:00000ed0       ??_C@_06DLPGJKHM@?$CFf?$CFf?$CFf?$AA@ 10009ed0     sspred_hmulti.obj
 0002:00000ed8       ??_C@_0M@IDBKLAKB@Bad?5format?$CB?$AA@ 10009ed8     sspred_hmulti.obj
 0002:00000ee8       ??_C@_0EI@EIOPGEPA@usage?5?3?5psipass2?5weight?9file?5ite@ 10009ee8     sspred_hmulti.obj
 0002:00000f30       ??_C@_01KDCPPGHE@r?$AA@    10009f30     sspred_hmulti.obj
 0002:00000f34       ??_C@_0CA@GIMJIKLI@failed?5opening?5file?5for?5reading?$AA@ 10009f34     sspred_hmulti.obj
 0002:00000f58       __real@3fe0000000000000    10009f58     sspred_hmulti.obj
 0002:00000f60       __real@4059000000000000    10009f60     sspred_hmulti.obj
 0002:00000f70       __xmm@80000000000000008000000000000000 10009f70     sspred_hmulti.obj
 0002:00000f80       ??_C@_03OFAPEBGM@?$CFs?6?$AA@ 10009f80     sspred_utils.obj
 0002:000d92d2       ?value@?$integral_constant@_N$0A@@std@@2_NB 100e22d2     MSVCRT:ti_inst.obj
 0002:000d92d3       ?value@?$integral_constant@_N$00@std@@2_NB 100e22d3     MSVCRT:ti_inst.obj
 0002:000d92d8       ??_7type_info@@6B@         100e22d8     MSVCRT:ti_inst.obj
 0002:000d92dc       __pDefaultRawDllMain       100e22dc     MSVCRT:crtdll.obj
 0002:000d92dc       __pRawDllMain              100e22dc     MSVCRT:crtdll.obj
 0002:000d92e8       ?ProcessDetach@NativeDll@<CrtImplementationDetails>@@0IB 100e22e8     MSVCRT:initsect.obj
 0002:000d92ec       ?ProcessAttach@NativeDll@<CrtImplementationDetails>@@0IB 100e22ec     MSVCRT:initsect.obj
 0002:000d92f0       ?ThreadAttach@NativeDll@<CrtImplementationDetails>@@0IB 100e22f0     MSVCRT:initsect.obj
 0002:000d92f4       ?ThreadDetach@NativeDll@<CrtImplementationDetails>@@0IB 100e22f4     MSVCRT:initsect.obj
 0002:000d92f8       ?ProcessVerifier@NativeDll@<CrtImplementationDetails>@@0IB 100e22f8     MSVCRT:initsect.obj
 0002:000d9300       __load_config_used         100e2300     MSVCRT:loadcfg.obj
 0002:000d93b8       ??_R4error_category@std@@6B@ 100e23b8     PsipredAlgTask.obj
 0002:000d93cc       ??_R3error_category@std@@8 100e23cc     PsipredAlgTask.obj
 0002:000d93dc       ??_R2error_category@std@@8 100e23dc     PsipredAlgTask.obj
 0002:000d93e4       ??_R1A@?0A@EA@error_category@std@@8 100e23e4     PsipredAlgTask.obj
 0002:000d9400       ??_R4_Generic_error_category@std@@6B@ 100e2400     PsipredAlgTask.obj
 0002:000d9414       ??_R3_Generic_error_category@std@@8 100e2414     PsipredAlgTask.obj
 0002:000d9424       ??_R2_Generic_error_category@std@@8 100e2424     PsipredAlgTask.obj
 0002:000d9430       ??_R1A@?0A@EA@_Generic_error_category@std@@8 100e2430     PsipredAlgTask.obj
 0002:000d944c       ??_R4_Iostream_error_category@std@@6B@ 100e244c     PsipredAlgTask.obj
 0002:000d9460       ??_R3_Iostream_error_category@std@@8 100e2460     PsipredAlgTask.obj
 0002:000d9470       ??_R2_Iostream_error_category@std@@8 100e2470     PsipredAlgTask.obj
 0002:000d9480       ??_R1A@?0A@EA@_Iostream_error_category@std@@8 100e2480     PsipredAlgTask.obj
 0002:000d949c       ??_R4_System_error_category@std@@6B@ 100e249c     PsipredAlgTask.obj
 0002:000d94b0       ??_R3_System_error_category@std@@8 100e24b0     PsipredAlgTask.obj
 0002:000d94c0       ??_R2_System_error_category@std@@8 100e24c0     PsipredAlgTask.obj
 0002:000d94d0       ??_R1A@?0A@EA@_System_error_category@std@@8 100e24d0     PsipredAlgTask.obj
 0002:000d94ec       ??_R4AbstractInt32Id@U2@@6B@ 100e24ec     PsipredAlgTask.obj
 0002:000d9500       ??_R3AbstractInt32Id@U2@@8 100e2500     PsipredAlgTask.obj
 0002:000d9510       ??_R2AbstractInt32Id@U2@@8 100e2510     PsipredAlgTask.obj
 0002:000d951c       ??_R1A@?0A@EA@AbstractInt32Id@U2@@8 100e251c     PsipredAlgTask.obj
 0002:000d9538       ??_R1A@?0A@EA@?$AbstractId@H@U2@@8 100e2538     PsipredAlgTask.obj
 0002:000d9554       ??_R3?$AbstractId@H@U2@@8  100e2554     PsipredAlgTask.obj
 0002:000d9564       ??_R2?$AbstractId@H@U2@@8  100e2564     PsipredAlgTask.obj
 0002:000d956c       ??_R4?$AbstractId@H@U2@@6B@ 100e256c     PsipredAlgTask.obj
 0002:000d9580       ??_R4ServiceType@U2@@6B@   100e2580     PsipredAlgTask.obj
 0002:000d9594       ??_R3ServiceType@U2@@8     100e2594     PsipredAlgTask.obj
 0002:000d95a4       ??_R2ServiceType@U2@@8     100e25a4     PsipredAlgTask.obj
 0002:000d95b4       ??_R1A@?0A@EA@ServiceType@U2@@8 100e25b4     PsipredAlgTask.obj
 0002:000d95d0       ??_R4PsipredAlgTask@U2@@6B@ 100e25d0     PsipredAlgTask.obj
 0002:000d95e4       ??_R3PsipredAlgTask@U2@@8  100e25e4     PsipredAlgTask.obj
 0002:000d95f4       ??_R2PsipredAlgTask@U2@@8  100e25f4     PsipredAlgTask.obj
 0002:000d9608       ??_R1A@?0A@EA@PsipredAlgTask@U2@@8 100e2608     PsipredAlgTask.obj
 0002:000d9624       ??_R1A@?0A@EA@SecStructPredictTask@U2@@8 100e2624     PsipredAlgTask.obj
 0002:000d9640       ??_R3SecStructPredictTask@U2@@8 100e2640     PsipredAlgTask.obj
 0002:000d9650       ??_R2SecStructPredictTask@U2@@8 100e2650     PsipredAlgTask.obj
 0002:000d9660       ??_R1A@?0A@EA@Task@U2@@8   100e2660     PsipredAlgTask.obj
 0002:000d967c       ??_R3Task@U2@@8            100e267c     PsipredAlgTask.obj
 0002:000d968c       ??_R2Task@U2@@8            100e268c     PsipredAlgTask.obj
 0002:000d9698       ??_R1A@?0A@EA@QObject@@8   100e2698     PsipredAlgTask.obj
 0002:000d96b4       ??_R3QObject@@8            100e26b4     PsipredAlgTask.obj
 0002:000d96c4       ??_R2QObject@@8            100e26c4     PsipredAlgTask.obj
 0002:000d96cc       ??_R4PsipredPlugin@U2@@6B@ 100e26cc     PsipredPlugin.obj
 0002:000d96e0       ??_R3PsipredPlugin@U2@@8   100e26e0     PsipredPlugin.obj
 0002:000d96f0       ??_R2PsipredPlugin@U2@@8   100e26f0     PsipredPlugin.obj
 0002:000d9700       ??_R1A@?0A@EA@PsipredPlugin@U2@@8 100e2700     PsipredPlugin.obj
 0002:000d971c       ??_R1A@?0A@EA@Plugin@U2@@8 100e271c     PsipredPlugin.obj
 0002:000d9738       ??_R3Plugin@U2@@8          100e2738     PsipredPlugin.obj
 0002:000d9748       ??_R2Plugin@U2@@8          100e2748     PsipredPlugin.obj
 0002:000d9754       ??_R4Factory@PsipredAlgTask@U2@@6B@ 100e2754     PsipredPlugin.obj
 0002:000d9768       ??_R3Factory@PsipredAlgTask@U2@@8 100e2768     PsipredPlugin.obj
 0002:000d9778       ??_R2Factory@PsipredAlgTask@U2@@8 100e2778     PsipredPlugin.obj
 0002:000d9784       ??_R1A@?0A@EA@Factory@PsipredAlgTask@U2@@8 100e2784     PsipredPlugin.obj
 0002:000d97a0       ??_R1A@?0A@EA@SecStructPredictTaskFactory@U2@@8 100e27a0     PsipredPlugin.obj
 0002:000d97bc       ??_R3SecStructPredictTaskFactory@U2@@8 100e27bc     PsipredPlugin.obj
 0002:000d97cc       ??_R2SecStructPredictTaskFactory@U2@@8 100e27cc     PsipredPlugin.obj
 0002:000d97d4       ??_R4type_info@@6B@        100e27d4     MSVCRT:ti_inst.obj
 0002:000d97e8       ??_R3type_info@@8          100e27e8     MSVCRT:ti_inst.obj
 0002:000d97f8       ??_R2type_info@@8          100e27f8     MSVCRT:ti_inst.obj
 0002:000d9800       ??_R1A@?0A@EA@type_info@@8 100e2800     MSVCRT:ti_inst.obj
 0002:000d9820       ___safe_se_handler_table   100e2820     <linker-defined>
 0002:000d98ec       ___rtc_iaa                 100e28ec     MSVCRT:initsect.obj
 0002:000d98f0       ___rtc_izz                 100e28f0     MSVCRT:initsect.obj
 0002:000d98f4       ___rtc_taa                 100e28f4     MSVCRT:initsect.obj
 0002:000d98f8       ___rtc_tzz                 100e28f8     MSVCRT:initsect.obj
 0002:000da5a4       __TI2CPAD                  100e35a4     sspred_utils.obj
 0002:000da5b4       __CTA2PAD                  100e35b4     sspred_utils.obj
 0002:000da5c0       __CT??_R0PAD@84            100e35c0     sspred_utils.obj
 0002:000da5dc       __CT??_R0PAX@84            100e35dc     sspred_utils.obj
 0002:000da880       __IMPORT_DESCRIPTOR_U2Core 100e3880     U2Core:U2Core.dll
 0002:000da894       __IMPORT_DESCRIPTOR_U2Algorithm 100e3894     U2Algorithm:U2Algorithm.dll
 0002:000da8a8       __IMPORT_DESCRIPTOR_U2View 100e38a8     U2View:U2View.dll
 0002:000da8bc       __IMPORT_DESCRIPTOR_Qt5Gui 100e38bc     Qt5Gui:Qt5Gui.dll
 0002:000da8d0       __IMPORT_DESCRIPTOR_Qt5Core 100e38d0     Qt5Core:Qt5Core.dll
 0002:000da8e4       __IMPORT_DESCRIPTOR_MSVCP120 100e38e4     msvcprt:MSVCP120.dll
 0002:000da8f8       __IMPORT_DESCRIPTOR_MSVCR120 100e38f8     MSVCRT:MSVCR120.dll
 0002:000da90c       __IMPORT_DESCRIPTOR_KERNEL32 100e390c     kernel32:KERNEL32.dll
 0002:000da920       __NULL_IMPORT_DESCRIPTOR   100e3920     U2Core:U2Core.dll
 0003:00000000       ?_Generic_object@?$_Error_objects@H@std@@2V_Generic_error_category@2@A 100e6000     PsipredAlgTask.obj
 0003:00000004       ?_Iostream_object@?$_Error_objects@H@std@@2V_Iostream_error_category@2@A 100e6004     PsipredAlgTask.obj
 0003:00000008       ?_System_object@?$_Error_objects@H@std@@2V_System_error_category@2@A 100e6008     PsipredAlgTask.obj
 0003:000000dc       ?rescodes@@3PBDB           100e60dc     seq2mtx.obj
 0003:000000e0       ?rnames@@3PAPBDA           100e60e0     sspred_hmulti.obj
 0003:00000134       ?staticMetaObject@PsipredAlgTask@U2@@2UQMetaObject@@B 100e6134     moc_PsipredAlgTask.obj
 0003:000001b4       ?staticMetaObject@PsipredPlugin@U2@@2UQMetaObject@@B 100e61b4     moc_PsipredPlugin.obj
 0003:000001d0       ___security_cookie         100e61d0     MSVCRT:gs_cookie.obj
 0003:000001d4       ___security_cookie_complement 100e61d4     MSVCRT:gs_cookie.obj
 0003:000001e0       ___native_dllmain_reason   100e61e0     MSVCRT:natstart.obj
 0003:000001e4       ??_R0PAD@8                 100e61e4     PsipredAlgTask.obj
 0003:000001f4       ??_R0?AVerror_category@std@@@8 100e61f4     PsipredAlgTask.obj
 0003:00000218       ??_R0?AV_Generic_error_category@std@@@8 100e6218     PsipredAlgTask.obj
 0003:00000244       ??_R0?AV_Iostream_error_category@std@@@8 100e6244     PsipredAlgTask.obj
 0003:00000270       ??_R0?AV_System_error_category@std@@@8 100e6270     PsipredAlgTask.obj
 0003:0000029c       ??_R0?AVAbstractInt32Id@U2@@@8 100e629c     PsipredAlgTask.obj
 0003:000002c0       ??_R0?AV?$AbstractId@H@U2@@@8 100e62c0     PsipredAlgTask.obj
 0003:000002e0       ??_R0?AVServiceType@U2@@@8 100e62e0     PsipredAlgTask.obj
 0003:00000300       ??_R0?AVPsipredAlgTask@U2@@@8 100e6300     PsipredAlgTask.obj
 0003:00000320       ??_R0?AVSecStructPredictTask@U2@@@8 100e6320     PsipredAlgTask.obj
 0003:00000348       ??_R0?AVTask@U2@@@8        100e6348     PsipredAlgTask.obj
 0003:00000360       ??_R0?AVQObject@@@8        100e6360     PsipredAlgTask.obj
 0003:00000378       ??_R0?AVPsipredPlugin@U2@@@8 100e6378     PsipredPlugin.obj
 0003:00000398       ??_R0?AVPlugin@U2@@@8      100e6398     PsipredPlugin.obj
 0003:000003b0       ??_R0?AVFactory@PsipredAlgTask@U2@@@8 100e63b0     PsipredPlugin.obj
 0003:000003d8       ??_R0?AVSecStructPredictTaskFactory@U2@@@8 100e63d8     PsipredPlugin.obj
 0003:00000408       ??_R0PAX@8                 100e6408     sspred_utils.obj
 0003:00000418       ??_R0?AVtype_info@@@8      100e6418     MSVCRT:ti_inst.obj
 0003:00000474       ?runLock@PsipredAlgTask@U2@@0VQMutex@@A 100e6474     PsipredAlgTask.obj
 0003:00000480       ?id@?$num_put@DV?$back_insert_iterator@V?$basic_string@DU?$char_traits@D@std@@V?$allocator@D@2@@std@@@std@@@std@@2V0locale@2@A 100e6480     PsipredAlgTask.obj
 0003:00000484       ?id@?$num_put@_WV?$back_insert_iterator@V?$basic_string@_WU?$char_traits@_W@std@@V?$allocator@_W@2@@std@@@std@@@std@@2V0locale@2@A 100e6484     PsipredAlgTask.obj
 0003:0000055c       ?dummy@?A0x86132f99@@3Uinitializer@1@A 100e655c     qrc_psipred.obj
 0003:00000888       ?__type_info_root_node@@3U__type_info_node@@A 100e6888     MSVCRT:tncleanup.obj
 0003:00000890       ___native_startup_lock     100e6890     <common>
 0003:00000894       ___native_startup_state    100e6894     <common>
 0003:00000898       ___dyn_tls_init_callback   100e6898     <common>
 0003:0000089c       ___onexitend               100e689c     <common>
 0003:000008a0       ___onexitbegin             100e68a0     <common>

 entry point at        0001:000063e0

 Static symbols

 0000:fff16000       .debug$S                   10000000     MSVCRT:MSVCR120.dll
 0000:fff16000       .debug$S                   10000000     MSVCRT:MSVCR120.dll
 0000:fff16000       .debug$S                   10000000     MSVCRT:MSVCR120.dll
 0000:fff16000       .debug$S                   10000000     MSVCRT:MSVCR120.dll
 0000:fff16000       .debug$S                   10000000     MSVCRT:MSVCR120.dll
 0000:fff16000       .debug$S                   10000000     MSVCRT:MSVCR120.dll
 0000:fff16000       .debug$S                   10000000     MSVCRT:MSVCR120.dll
 0000:fff16000       .debug$S                   10000000     U2Core:U2Core.dll
 0000:fff16000       .debug$S                   10000000     U2Core:U2Core.dll
 0000:fff16000       .debug$S                   10000000     U2Core:U2Core.dll
 0000:fff16000       .debug$S                   10000000     U2Core:U2Core.dll
 0000:fff16000       .debug$S                   10000000     U2Core:U2Core.dll
 0000:fff16000       .debug$S                   10000000     U2Core:U2Core.dll
 0000:fff16000       .debug$S                   10000000     U2Core:U2Core.dll
 0000:fff16000       .debug$S                   10000000     U2Core:U2Core.dll
 0000:fff16000       .debug$S                   10000000     U2Core:U2Core.dll
 0000:fff16000       .debug$S                   10000000     U2Core:U2Core.dll
 0000:fff16000       .debug$S                   10000000     U2Core:U2Core.dll
 0000:fff16000       .debug$S                   10000000     U2Core:U2Core.dll
 0000:fff16000       .debug$S                   10000000     U2Core:U2Core.dll
 0000:fff16000       .debug$S                   10000000     U2Core:U2Core.dll
 0000:fff16000       .debug$S                   10000000     U2Core:U2Core.dll
 0000:fff16000       .debug$S                   10000000     U2Core:U2Core.dll
 0000:fff16000       .debug$S                   10000000     U2Core:U2Core.dll
 0000:fff16000       .debug$S                   10000000     U2Core:U2Core.dll
 0000:fff16000       .debug$S                   10000000     U2Core:U2Core.dll
 0000:fff16000       .debug$S                   10000000     U2Core:U2Core.dll
 0000:fff16000       .debug$S                   10000000     U2Core:U2Core.dll
 0000:fff16000       .debug$S                   10000000     U2Core:U2Core.dll
 0000:fff16000       .debug$S                   10000000     U2Core:U2Core.dll
 0000:fff16000       .debug$S                   10000000     U2Core:U2Core.dll
 0000:fff16000       .debug$S                   10000000     U2Core:U2Core.dll
 0000:fff16000       .debug$S                   10000000     U2Core:U2Core.dll
 0000:fff16000       .debug$S                   10000000     U2Core:U2Core.dll
 0000:fff16000       .debug$S                   10000000     U2Core:U2Core.dll
 0000:fff16000       .debug$S                   10000000     U2Core:U2Core.dll
 0000:fff16000       .debug$S                   10000000     U2Core:U2Core.dll
 0000:fff16000       .debug$S                   10000000     U2Core:U2Core.dll
 0000:fff16000       .debug$S                   10000000     U2Core:U2Core.dll
 0000:fff16000       .debug$S                   10000000     U2Core:U2Core.dll
 0000:fff16000       .debug$S                   10000000     U2Core:U2Core.dll
 0000:fff16000       .debug$S                   10000000     U2Core:U2Core.dll
 0000:fff16000       .debug$S                   10000000     U2Core:U2Core.dll
 0000:fff16000       .debug$S                   10000000     U2Core:U2Core.dll
 0000:fff16000       .debug$S                   10000000     U2Core:U2Core.dll
 0000:fff16000       .debug$S                   10000000     U2Algorithm:U2Algorithm.dll
 0000:fff16000       .debug$S                   10000000     U2Algorithm:U2Algorithm.dll
 0000:fff16000       .debug$S                   10000000     U2Algorithm:U2Algorithm.dll
 0001:fffff000       __ehhandler$?_Copy@?$basic_string@DU?$char_traits@D@std@@V?$allocator@D@2@@std@@QAEXII@Z 10000000 f   moc_PsipredPlugin.obj
 0000:fff16000       .debug$S                   10000000     U2Algorithm:U2Algorithm.dll
 0000:fff16000       .debug$S                   10000000     U2Algorithm:U2Algorithm.dll
 0000:fff16000       .debug$S                   10000000     U2Algorithm:U2Algorithm.dll
 0000:fff16000       .debug$S                   10000000     U2Algorithm:U2Algorithm.dll
 0000:fff16000       .debug$S                   10000000     U2Algorithm:U2Algorithm.dll
 0000:fff16000       .debug$S                   10000000     U2Algorithm:U2Algorithm.dll
 0002:ffff7000       __catchsym$?_Copy@?$basic_string@DU?$char_traits@D@std@@V?$allocator@D@2@@std@@QAEXII@Z$5 10000000     moc_PsipredPlugin.obj
 0000:fff16000       .debug$S                   10000000     MSVCRT:MSVCR120.dll
 0000:fff16000       .debug$S                   10000000     MSVCRT:MSVCR120.dll
 0000:fff16000       .debug$S                   10000000     MSVCRT:MSVCR120.dll
 0000:fff16000       .debug$S                   10000000     MSVCRT:MSVCR120.dll
 0000:fff16000       .debug$S                   10000000     MSVCRT:MSVCR120.dll
 0000:fff16000       .debug$S                   10000000     MSVCRT:MSVCR120.dll
 0000:fff16000       .debug$S                   10000000     MSVCRT:MSVCR120.dll
 0000:fff16000       .debug$S                   10000000     MSVCRT:MSVCR120.dll
 0000:fff16000       .debug$S                   10000000     MSVCRT:MSVCR120.dll
 0000:fff16000       .debug$S                   10000000     MSVCRT:MSVCR120.dll
 0000:fff16000       .debug$S                   10000000     MSVCRT:MSVCR120.dll
 0000:fff16000       .debug$S                   10000000     MSVCRT:MSVCR120.dll
 0000:fff16000       .debug$S                   10000000     MSVCRT:MSVCR120.dll
 0000:fff16000       .debug$S                   10000000     MSVCRT:MSVCR120.dll
 0000:fff16000       .debug$S                   10000000     MSVCRT:MSVCR120.dll
 0000:fff16000       .debug$S                   10000000     MSVCRT:MSVCR120.dll
 0000:fff16000       .debug$S                   10000000     MSVCRT:MSVCR120.dll
 0000:fff16000       .debug$S                   10000000     U2View:U2View.dll
 0000:fff16000       .debug$S                   10000000     Qt5Gui:Qt5Gui.dll
 0000:fff16000       .debug$S                   10000000     Qt5Core:Qt5Core.dll
 0000:fff16000       .debug$S                   10000000     Qt5Core:Qt5Core.dll
 0000:fff16000       .debug$S                   10000000     Qt5Core:Qt5Core.dll
 0000:fff16000       .debug$S                   10000000     Qt5Core:Qt5Core.dll
 0000:fff16000       .debug$S                   10000000     Qt5Core:Qt5Core.dll
 0002:ffff7000       ?_System_object$initializer$@?$_Error_objects@H@std@@2P6AXXZA 10000000     PsipredPlugin.obj
 0002:ffff7000       ?_Iostream_object$initializer$@?$_Error_objects@H@std@@2P6AXXZA 10000000     PsipredPlugin.obj
 0002:ffff7000       ?_Generic_object$initializer$@?$_Error_objects@H@std@@2P6AXXZA 10000000     PsipredPlugin.obj
 0000:fff16000       .debug$S                   10000000     Qt5Core:Qt5Core.dll
 0000:fff16000       .debug$S                   10000000     Qt5Core:Qt5Core.dll
 0000:fff16000       .debug$S                   10000000     Qt5Core:Qt5Core.dll
 0000:fff16000       .debug$S                   10000000     Qt5Core:Qt5Core.dll
 0002:ffff7000       ?_Generic_object$initializer$@?$_Error_objects@H@std@@2P6AXXZA 10000000     moc_PsipredPlugin.obj
 0002:ffff7000       ?_Iostream_object$initializer$@?$_Error_objects@H@std@@2P6AXXZA 10000000     moc_PsipredPlugin.obj
 0002:ffff7000       ?_System_object$initializer$@?$_Error_objects@H@std@@2P6AXXZA 10000000     moc_PsipredPlugin.obj
 0000:fff16000       .debug$S                   10000000     Qt5Core:Qt5Core.dll
 0000:fff16000       .debug$S                   10000000     Qt5Core:Qt5Core.dll
 0000:fff16000       .debug$S                   10000000     Qt5Core:Qt5Core.dll
 0000:fff16000       .debug$S                   10000000     Qt5Core:Qt5Core.dll
 0000:fff16000       .debug$S                   10000000     Qt5Core:Qt5Core.dll
 0000:fff16000       .debug$S                   10000000     Qt5Core:Qt5Core.dll
 0000:fff16000       .debug$S                   10000000     Qt5Core:Qt5Core.dll
 0000:fff16000       .debug$S                   10000000     Qt5Core:Qt5Core.dll
 0000:fff16000       .debug$S                   10000000     Qt5Core:Qt5Core.dll
 0000:fff16000       .debug$S                   10000000     Qt5Core:Qt5Core.dll
 0000:fff16000       .debug$S                   10000000     Qt5Core:Qt5Core.dll
 0000:fff16000       .debug$S                   10000000     Qt5Core:Qt5Core.dll
 0000:fff16000       .debug$S                   10000000     Qt5Core:Qt5Core.dll
 0000:fff16000       .debug$S                   10000000     Qt5Core:Qt5Core.dll
 0000:fff16000       .debug$S                   10000000     Qt5Core:Qt5Core.dll
 0000:fff16000       .debug$S                   10000000     Qt5Core:Qt5Core.dll
 0000:fff16000       .debug$S                   10000000     Qt5Core:Qt5Core.dll
 0000:fff16000       .debug$S                   10000000     Qt5Core:Qt5Core.dll
 0000:fff16000       .debug$S                   10000000     Qt5Core:Qt5Core.dll
 0000:fff16000       .debug$S                   10000000     Qt5Core:Qt5Core.dll
 0000:fff16000       .debug$S                   10000000     Qt5Core:Qt5Core.dll
 0000:fff16000       .debug$S                   10000000     Qt5Core:Qt5Core.dll
 0000:fff16000       .debug$S                   10000000     Qt5Core:Qt5Core.dll
 0000:fff16000       .debug$S                   10000000     Qt5Core:Qt5Core.dll
 0000:fff16000       .debug$S                   10000000     Qt5Core:Qt5Core.dll
 0000:fff16000       .debug$S                   10000000     Qt5Core:Qt5Core.dll
 0000:fff16000       .debug$S                   10000000     Qt5Core:Qt5Core.dll
 0001:fffff000       __ehhandler$?_Copy@?$basic_string@DU?$char_traits@D@std@@V?$allocator@D@2@@std@@QAEXII@Z 10000000 f   moc_PsipredAlgTask.obj
 0000:fff16000       .debug$S                   10000000     Qt5Core:Qt5Core.dll
 0002:ffff7000       __catchsym$?node_copy@?$QList@VQString@@@@AAEXPAUNode@1@00@Z$6 10000000     PsipredPlugin.obj
 0002:ffff7000       __unwindtable$?node_construct@?$QList@VQString@@@@AAEXPAUNode@1@ABVQString@@@Z 10000000     PsipredPlugin.obj
 0002:ffff7000       __catchsym$?detach_helper_grow@?$QList@VQString@@@@AAEPAUNode@1@HH@Z$5 10000000     PsipredPlugin.obj
 0002:ffff7000       __catchsym$?append@?$QList@VQString@@@@QAEXABVQString@@@Z$13 10000000     PsipredPlugin.obj
 0002:ffff7000       __catchsym$?_Copy@?$basic_string@DU?$char_traits@D@std@@V?$allocator@D@2@@std@@QAEXII@Z$5 10000000     PsipredPlugin.obj
 0001:fffff000       __unwindfunclet$?node_copy@?$QList@VQString@@@@AAEXPAUNode@1@00@Z$5 10000000 f   PsipredPlugin.obj
 0001:fffff000       __unwindfunclet$?node_construct@?$QList@VQString@@@@AAEXPAUNode@1@ABVQString@@@Z$1 10000000 f   PsipredPlugin.obj
 0000:fff16000       .debug$S                   10000000     U2Core:U2Core.dll
 0001:fffff000       __ehhandler$?detach_helper_grow@?$QList@VQString@@@@AAEPAUNode@1@HH@Z 10000000 f   PsipredPlugin.obj
 0001:fffff000       __unwindfunclet$?append@?$QList@VQString@@@@QAEXABVQString@@@Z$7 10000000 f   PsipredPlugin.obj
 0001:fffff000       __ehhandler$?_Copy@?$basic_string@DU?$char_traits@D@std@@V?$allocator@D@2@@std@@QAEXII@Z 10000000 f   PsipredPlugin.obj
 0002:ffff7000       ?_System_object$initializer$@?$_Error_objects@H@std@@2P6AXXZA 10000000     seq2mtx.obj
 0002:ffff7000       ?_Iostream_object$initializer$@?$_Error_objects@H@std@@2P6AXXZA 10000000     seq2mtx.obj
 0002:ffff7000       ?_Generic_object$initializer$@?$_Error_objects@H@std@@2P6AXXZA 10000000     seq2mtx.obj
 0000:fff16000       .debug$S                   10000000     Qt5Core:Qt5Core.dll
 0000:fff16000       .debug$S                   10000000     Qt5Core:Qt5Core.dll
 0000:fff16000       .debug$S                   10000000     Qt5Core:Qt5Core.dll
 0000:fff16000       .debug$S                   10000000     Qt5Core:Qt5Core.dll
 0000:fff16000       .debug$S                   10000000     Qt5Core:Qt5Core.dll
 0000:fff16000       .debug$S                   10000000     Qt5Core:Qt5Core.dll
 0002:ffff7000       __catchsym$?_Copy@?$basic_string@DU?$char_traits@D@std@@V?$allocator@D@2@@std@@QAEXII@Z$5 10000000     seq2mtx.obj
 0001:fffff000       __ehhandler$?_Copy@?$basic_string@DU?$char_traits@D@std@@V?$allocator@D@2@@std@@QAEXII@Z 10000000 f   seq2mtx.obj
 0002:ffff7000       ?_System_object$initializer$@?$_Error_objects@H@std@@2P6AXXZA 10000000     sspred_avpred.obj
 0002:ffff7000       __catchsym$?_Copy@?$basic_string@DU?$char_traits@D@std@@V?$allocator@D@2@@std@@QAEXII@Z$5 10000000     moc_PsipredAlgTask.obj
 0000:fff16000       .debug$S                   10000000     MSVCRT:MSVCR120.dll
 0000:fff16000       .debug$S                   10000000     MSVCRT:MSVCR120.dll
 0000:fff16000       .debug$S                   10000000     MSVCRT:MSVCR120.dll
 0000:fff16000       .debug$S                   10000000     MSVCRT:MSVCR120.dll
 0000:fff16000       .debug$S                   10000000     MSVCRT:MSVCR120.dll
 0000:fff16000       .debug$S                   10000000     MSVCRT:MSVCR120.dll
 0000:fff16000       .debug$S                   10000000     MSVCRT:MSVCR120.dll
 0000:fff16000       .debug$S                   10000000     MSVCRT:MSVCR120.dll
 0000:fff16000       .debug$S                   10000000     MSVCRT:MSVCR120.dll
 0000:fff16000       .debug$S                   10000000     MSVCRT:MSVCR120.dll
 0000:fff16000       .debug$S                   10000000     MSVCRT:MSVCR120.dll
 0000:fff16000       .debug$S                   10000000     MSVCRT:MSVCR120.dll
 0000:fff16000       .debug$S                   10000000     MSVCRT:MSVCR120.dll
 0000:fff16000       .debug$S                   10000000     MSVCRT:MSVCR120.dll
 0000:fff16000       .debug$S                   10000000     MSVCRT:MSVCR120.dll
 0000:fff16000       .debug$S                   10000000     MSVCRT:MSVCR120.dll
 0000:fff16000       .debug$S                   10000000     MSVCRT:MSVCR120.dll
 0000:fff16000       .debug$S                   10000000     MSVCRT:MSVCR120.dll
 0002:ffff7000       ?_Iostream_object$initializer$@?$_Error_objects@H@std@@2P6AXXZA 10000000     sspred_avpred.obj
 0002:ffff7000       ?_Generic_object$initializer$@?$_Error_objects@H@std@@2P6AXXZA 10000000     sspred_avpred.obj
 0000:fff16000       .debug$S                   10000000     Qt5Core:Qt5Core.dll
 0000:fff16000       .debug$S                   10000000     Qt5Core:Qt5Core.dll
 0000:fff16000       .debug$S                   10000000     Qt5Core:Qt5Core.dll
 0000:fff16000       .debug$S                   10000000     Qt5Core:Qt5Core.dll
 0000:fff16000       .debug$S                   10000000     Qt5Core:Qt5Core.dll
 0000:fff16000       .debug$S                   10000000     Qt5Core:Qt5Core.dll
 0000:fff16000       .debug$S                   10000000     msvcprt:MSVCP120.dll
 0000:fff16000       .debug$S                   10000000     msvcprt:MSVCP120.dll
 0000:fff16000       .debug$S                   10000000     msvcprt:MSVCP120.dll
 0000:fff16000       .debug$S                   10000000     msvcprt:MSVCP120.dll
 0000:fff16000       .debug$S                   10000000     msvcprt:MSVCP120.dll
 0000:fff16000       .debug$S                   10000000     Qt5Core:Qt5Core.dll
 0000:fff16000       .debug$S                   10000000     Qt5Core:Qt5Core.dll
 0000:fff16000       .debug$S                   10000000     Qt5Core:Qt5Core.dll
 0000:fff16000       .debug$S                   10000000     Qt5Core:Qt5Core.dll
 0000:fff16000       .debug$S                   10000000     Qt5Core:Qt5Core.dll
 0000:fff16000       .debug$S                   10000000     Qt5Core:Qt5Core.dll
 0000:fff16000       .debug$S                   10000000     Qt5Core:Qt5Core.dll
 0000:fff16000       .debug$S                   10000000     Qt5Core:Qt5Core.dll
 0002:ffff7000       __catchsym$?node_copy@?$QList@VQString@@@@AAEXPAUNode@1@00@Z$6 10000000     sspred_avpred.obj
 0000:fff16000       .debug$S                   10000000     Qt5Core:Qt5Core.dll
 0002:ffff7000       ?_Generic_object$initializer$@?$_Error_objects@H@std@@2P6AXXZA 10000000     moc_PsipredAlgTask.obj
 0002:ffff7000       ?_Iostream_object$initializer$@?$_Error_objects@H@std@@2P6AXXZA 10000000     moc_PsipredAlgTask.obj
 0002:ffff7000       ?_System_object$initializer$@?$_Error_objects@H@std@@2P6AXXZA 10000000     moc_PsipredAlgTask.obj
 0000:fff16000       .debug$S                   10000000     Qt5Core:Qt5Core.dll
 0000:fff16000       .debug$S                   10000000     Qt5Core:Qt5Core.dll
 0000:fff16000       .debug$S                   10000000     Qt5Core:Qt5Core.dll
 0002:ffff7000       __unwindtable$??H@YA?BVQString@@ABV0@PBD@Z 10000000     sspred_avpred.obj
 0002:ffff7000       __unwindtable$??H@YA?BVQString@@ABV0@VQChar@@@Z 10000000     sspred_avpred.obj
 0002:ffff7000       __catchsym$?_Copy@?$basic_string@DU?$char_traits@D@std@@V?$allocator@D@2@@std@@QAEXII@Z$5 10000000     sspred_avpred.obj
 0001:fffff000       __unwindfunclet$?node_copy@?$QList@VQString@@@@AAEXPAUNode@1@00@Z$5 10000000 f   sspred_avpred.obj
 0001:fffff000       __ehhandler$?_Copy@?$basic_string@DU?$char_traits@D@std@@V?$allocator@D@2@@std@@QAEXII@Z 10000000 f   sspred_hmulti.obj
 0001:fffff000       __unwindfunclet$??H@YA?BVQString@@ABV0@PBD@Z$0 10000000 f   sspred_avpred.obj
 0001:fffff000       __unwindfunclet$??H@YA?BVQString@@ABV0@VQChar@@@Z$0 10000000 f   sspred_avpred.obj
 0001:fffff000       __ehhandler$?_Copy@?$basic_string@DU?$char_traits@D@std@@V?$allocator@D@2@@std@@QAEXII@Z 10000000 f   sspred_avpred.obj
 0001:fffff000       __unwindfunclet$??H@YA?BVQString@@ABV0@VQChar@@@Z$0 10000000 f   sspred_hmulti.obj
 0002:ffff7000       ?_System_object$initializer$@?$_Error_objects@H@std@@2P6AXXZA 10000000     sspred_hmulti.obj
 0001:fffff000       __unwindfunclet$??H@YA?BVQString@@ABV0@PBD@Z$0 10000000 f   sspred_hmulti.obj
 0002:ffff7000       ?_Iostream_object$initializer$@?$_Error_objects@H@std@@2P6AXXZA 10000000     sspred_hmulti.obj
 0002:ffff7000       ?_Generic_object$initializer$@?$_Error_objects@H@std@@2P6AXXZA 10000000     sspred_hmulti.obj
 0000:fff16000       .debug$S                   10000000     Qt5Core:Qt5Core.dll
 0000:fff16000       .debug$S                   10000000     kernel32:KERNEL32.dll
 0000:fff16000       .debug$S                   10000000     kernel32:KERNEL32.dll
 0000:fff16000       .debug$S                   10000000     kernel32:KERNEL32.dll
 0000:fff16000       .debug$S                   10000000     kernel32:KERNEL32.dll
 0000:fff16000       .debug$S                   10000000     kernel32:KERNEL32.dll
 0000:fff16000       .debug$S                   10000000     kernel32:KERNEL32.dll
 0000:fff16000       .debug$S                   10000000     kernel32:KERNEL32.dll
 0000:fff16000       .debug$S                   10000000     kernel32:KERNEL32.dll
 0000:fff16000       .debug$S                   10000000     kernel32:KERNEL32.dll
 0002:ffff7000       __unwindtable$??H@YA?BVQString@@ABV0@PBD@Z 10000000     sspred_hmulti.obj
 0002:ffff7000       __unwindtable$??H@YA?BVQString@@ABV0@VQChar@@@Z 10000000     sspred_hmulti.obj
 0002:ffff7000       __catchsym$?_Copy@?$basic_string@DU?$char_traits@D@std@@V?$allocator@D@2@@std@@QAEXII@Z$5 10000000     sspred_hmulti.obj
 0002:ffff7008       __ehfuncinfo$??H@YA?BVQString@@ABV0@VQChar@@@Z 10000008     sspred_hmulti.obj
 0002:ffff7008       __ehfuncinfo$??H@YA?BVQString@@ABV0@VQChar@@@Z 10000008     sspred_avpred.obj
 0002:ffff7010       __ehfuncinfo$?node_construct@?$QList@VQString@@@@AAEXPAUNode@1@ABVQString@@@Z 10000010     PsipredPlugin.obj
 0002:ffff7010       __tryblocktable$?node_copy@?$QList@VQString@@@@AAEXPAUNode@1@00@Z 10000010     sspred_avpred.obj
 0002:ffff7010       __catchsym$?_Copy@?$basic_string@DU?$char_traits@D@std@@V?$allocator@D@2@@std@@QAEXII@Z$4 10000010     sspred_hmulti.obj
 0002:ffff7010       __catchsym$?_Copy@?$basic_string@DU?$char_traits@D@std@@V?$allocator@D@2@@std@@QAEXII@Z$4 10000010     moc_PsipredPlugin.obj
 0002:ffff7010       __tryblocktable$?node_copy@?$QList@VQString@@@@AAEXPAUNode@1@00@Z 10000010     PsipredPlugin.obj
 0002:ffff7010       __catchsym$?_Copy@?$basic_string@DU?$char_traits@D@std@@V?$allocator@D@2@@std@@QAEXII@Z$4 10000010     PsipredPlugin.obj
 0002:ffff7010       __catchsym$?append@?$QList@VQString@@@@QAEXABVQString@@@Z$12 10000010     PsipredPlugin.obj
 0002:ffff7010       __ehfuncinfo$??H@YA?BVQString@@ABV0@PBD@Z 10000010     sspred_hmulti.obj
 0002:ffff7010       __ehfuncinfo$??H@YA?BVQString@@ABV0@PBD@Z 10000010     sspred_avpred.obj
 0002:ffff7010       __catchsym$?_Copy@?$basic_string@DU?$char_traits@D@std@@V?$allocator@D@2@@std@@QAEXII@Z$4 10000010     seq2mtx.obj
 0002:ffff7010       __catchsym$?_Copy@?$basic_string@DU?$char_traits@D@std@@V?$allocator@D@2@@std@@QAEXII@Z$4 10000010     moc_PsipredAlgTask.obj
 0002:ffff7010       __catchsym$?_Copy@?$basic_string@DU?$char_traits@D@std@@V?$allocator@D@2@@std@@QAEXII@Z$4 10000010     sspred_avpred.obj
 0002:ffff7010       __catchsym$?detach_helper_grow@?$QList@VQString@@@@AAEPAUNode@1@HH@Z$4 10000010     PsipredPlugin.obj
 0001:fffff011       __ehhandler$?node_construct@?$QList@VQString@@@@AAEXPAUNode@1@ABVQString@@@Z 10000011 f   PsipredPlugin.obj
 0001:fffff011       __ehhandler$?node_copy@?$QList@VQString@@@@AAEXPAUNode@1@00@Z 10000011 f   sspred_avpred.obj
 0001:fffff011       __ehhandler$?node_copy@?$QList@VQString@@@@AAEXPAUNode@1@00@Z 10000011 f   PsipredPlugin.obj
 0001:fffff011       __unwindfunclet$?append@?$QList@VQString@@@@QAEXABVQString@@@Z$11 10000011 f   PsipredPlugin.obj
 0001:fffff01a       __ehhandler$??H@YA?BVQString@@ABV0@VQChar@@@Z 1000001a f   sspred_hmulti.obj
 0001:fffff01a       __unwindfunclet$??H@YA?BVQString@@ABV0@PBD@Z$1 1000001a f   sspred_avpred.obj
 0001:fffff01a       __ehhandler$??H@YA?BVQString@@ABV0@VQChar@@@Z 1000001a f   sspred_avpred.obj
 0001:fffff01a       __unwindfunclet$??H@YA?BVQString@@ABV0@PBD@Z$1 1000001a f   sspred_hmulti.obj
 0002:ffff7020       __ehfuncinfo$?append@?$QList@VQString@@@@QAEXABVQString@@@Z 10000020     PsipredPlugin.obj
 0002:ffff7020       __unwindtable$?_Copy@?$basic_string@DU?$char_traits@D@std@@V?$allocator@D@2@@std@@QAEXII@Z 10000020     PsipredPlugin.obj
 0002:ffff7020       __unwindtable$?_Copy@?$basic_string@DU?$char_traits@D@std@@V?$allocator@D@2@@std@@QAEXII@Z 10000020     seq2mtx.obj
 0002:ffff7020       __unwindtable$?_Copy@?$basic_string@DU?$char_traits@D@std@@V?$allocator@D@2@@std@@QAEXII@Z 10000020     sspred_avpred.obj
 0002:ffff7020       __unwindtable$?detach_helper_grow@?$QList@VQString@@@@AAEPAUNode@1@HH@Z 10000020     PsipredPlugin.obj
 0002:ffff7020       __unwindtable$?_Copy@?$basic_string@DU?$char_traits@D@std@@V?$allocator@D@2@@std@@QAEXII@Z 10000020     sspred_hmulti.obj
 0002:ffff7020       __unwindtable$?_Copy@?$basic_string@DU?$char_traits@D@std@@V?$allocator@D@2@@std@@QAEXII@Z 10000020     moc_PsipredPlugin.obj
 0002:ffff7020       __unwindtable$?_Copy@?$basic_string@DU?$char_traits@D@std@@V?$allocator@D@2@@std@@QAEXII@Z 10000020     moc_PsipredAlgTask.obj
 0001:fffff022       __ehhandler$?append@?$QList@VQString@@@@QAEXABVQString@@@Z 10000022 f   PsipredPlugin.obj
 0001:fffff023       __ehhandler$??H@YA?BVQString@@ABV0@PBD@Z 10000023 f   sspred_avpred.obj
 0001:fffff023       __ehhandler$??H@YA?BVQString@@ABV0@PBD@Z 10000023 f   sspred_hmulti.obj
 0002:ffff7024       __ehfuncinfo$?node_copy@?$QList@VQString@@@@AAEXPAUNode@1@00@Z 10000024     sspred_avpred.obj
 0002:ffff7024       __ehfuncinfo$?node_copy@?$QList@VQString@@@@AAEXPAUNode@1@00@Z 10000024     PsipredPlugin.obj
 0002:ffff7040       __ehfuncinfo$?_Copy@?$basic_string@DU?$char_traits@D@std@@V?$allocator@D@2@@std@@QAEXII@Z 10000040     seq2mtx.obj
 0002:ffff7040       __ehfuncinfo$?_Copy@?$basic_string@DU?$char_traits@D@std@@V?$allocator@D@2@@std@@QAEXII@Z 10000040     sspred_avpred.obj
 0002:ffff7040       __ehfuncinfo$?_Copy@?$basic_string@DU?$char_traits@D@std@@V?$allocator@D@2@@std@@QAEXII@Z 10000040     moc_PsipredPlugin.obj
 0002:ffff7040       __ehfuncinfo$?_Copy@?$basic_string@DU?$char_traits@D@std@@V?$allocator@D@2@@std@@QAEXII@Z 10000040     sspred_hmulti.obj
 0002:ffff7040       __ehfuncinfo$?_Copy@?$basic_string@DU?$char_traits@D@std@@V?$allocator@D@2@@std@@QAEXII@Z 10000040     PsipredPlugin.obj
 0002:ffff7040       __ehfuncinfo$?detach_helper_grow@?$QList@VQString@@@@AAEPAUNode@1@HH@Z 10000040     PsipredPlugin.obj
 0002:ffff7040       __ehfuncinfo$?_Copy@?$basic_string@DU?$char_traits@D@std@@V?$allocator@D@2@@std@@QAEXII@Z 10000040     moc_PsipredAlgTask.obj
 0002:ffff7044       __tryblocktable$?append@?$QList@VQString@@@@QAEXABVQString@@@Z 10000044     PsipredPlugin.obj
 0002:ffff7048       __unwindtable$?node_copy@?$QList@VQString@@@@AAEXPAUNode@1@00@Z 10000048     PsipredPlugin.obj
 0002:ffff7048       __unwindtable$?node_copy@?$QList@VQString@@@@AAEXPAUNode@1@00@Z 10000048     sspred_avpred.obj
 0001:fffff062       __catch$?node_copy@?$QList@VQString@@@@AAEXPAUNode@1@00@Z$2 10000062 f   sspred_avpred.obj
 0001:fffff062       __catch$?node_copy@?$QList@VQString@@@@AAEXPAUNode@1@00@Z$2 10000062 f   PsipredPlugin.obj
 0002:ffff7064       __tryblocktable$?_Copy@?$basic_string@DU?$char_traits@D@std@@V?$allocator@D@2@@std@@QAEXII@Z 10000064     PsipredPlugin.obj
 0002:ffff7064       __tryblocktable$?detach_helper_grow@?$QList@VQString@@@@AAEPAUNode@1@HH@Z 10000064     PsipredPlugin.obj
 0002:ffff7064       __tryblocktable$?_Copy@?$basic_string@DU?$char_traits@D@std@@V?$allocator@D@2@@std@@QAEXII@Z 10000064     sspred_hmulti.obj
 0002:ffff7064       __tryblocktable$?_Copy@?$basic_string@DU?$char_traits@D@std@@V?$allocator@D@2@@std@@QAEXII@Z 10000064     moc_PsipredAlgTask.obj
 0002:ffff7064       __tryblocktable$?_Copy@?$basic_string@DU?$char_traits@D@std@@V?$allocator@D@2@@std@@QAEXII@Z 10000064     sspred_avpred.obj
 0002:ffff7064       __tryblocktable$?_Copy@?$basic_string@DU?$char_traits@D@std@@V?$allocator@D@2@@std@@QAEXII@Z 10000064     moc_PsipredPlugin.obj
 0002:ffff7064       __tryblocktable$?_Copy@?$basic_string@DU?$char_traits@D@std@@V?$allocator@D@2@@std@@QAEXII@Z 10000064     seq2mtx.obj
 0002:ffff706c       __unwindtable$?append@?$QList@VQString@@@@QAEXABVQString@@@Z 1000006c     PsipredPlugin.obj
 0001:fffff07d       __catch$?append@?$QList@VQString@@@@QAEXABVQString@@@Z$0 1000007d f   PsipredPlugin.obj
 0001:fffff096       __catch$?_Copy@?$basic_string@DU?$char_traits@D@std@@V?$allocator@D@2@@std@@QAEXII@Z$0 10000096 f   seq2mtx.obj
 0001:fffff096       __catch$?_Copy@?$basic_string@DU?$char_traits@D@std@@V?$allocator@D@2@@std@@QAEXII@Z$0 10000096 f   sspred_avpred.obj
 0001:fffff096       __catch$?_Copy@?$basic_string@DU?$char_traits@D@std@@V?$allocator@D@2@@std@@QAEXII@Z$0 10000096 f   sspred_hmulti.obj
 0001:fffff096       __catch$?_Copy@?$basic_string@DU?$char_traits@D@std@@V?$allocator@D@2@@std@@QAEXII@Z$0 10000096 f   PsipredPlugin.obj
 0001:fffff096       __catch$?_Copy@?$basic_string@DU?$char_traits@D@std@@V?$allocator@D@2@@std@@QAEXII@Z$0 10000096 f   moc_PsipredPlugin.obj
 0001:fffff096       __catch$?_Copy@?$basic_string@DU?$char_traits@D@std@@V?$allocator@D@2@@std@@QAEXII@Z$0 10000096 f   moc_PsipredAlgTask.obj
 0001:fffff0ce       __catch$?append@?$QList@VQString@@@@QAEXABVQString@@@Z$4 100000ce f   PsipredPlugin.obj
 0001:fffff0d3       __catch$?_Copy@?$basic_string@DU?$char_traits@D@std@@V?$allocator@D@2@@std@@QAEXII@Z$1 100000d3 f   sspred_avpred.obj
 0001:fffff0d3       __catch$?_Copy@?$basic_string@DU?$char_traits@D@std@@V?$allocator@D@2@@std@@QAEXII@Z$1 100000d3 f   seq2mtx.obj
 0001:fffff0d3       __catch$?_Copy@?$basic_string@DU?$char_traits@D@std@@V?$allocator@D@2@@std@@QAEXII@Z$1 100000d3 f   moc_PsipredPlugin.obj
 0001:fffff0d3       __catch$?_Copy@?$basic_string@DU?$char_traits@D@std@@V?$allocator@D@2@@std@@QAEXII@Z$1 100000d3 f   PsipredPlugin.obj
 0001:fffff0d3       __catch$?_Copy@?$basic_string@DU?$char_traits@D@std@@V?$allocator@D@2@@std@@QAEXII@Z$1 100000d3 f   sspred_hmulti.obj
 0001:fffff0d3       __catch$?_Copy@?$basic_string@DU?$char_traits@D@std@@V?$allocator@D@2@@std@@QAEXII@Z$1 100000d3 f   moc_PsipredAlgTask.obj
 0001:fffff11e       __catch$?detach_helper_grow@?$QList@VQString@@@@AAEPAUNode@1@HH@Z$2 1000011e f   PsipredPlugin.obj
 0001:fffff159       __catch$?detach_helper_grow@?$QList@VQString@@@@AAEPAUNode@1@HH@Z$0 10000159 f   PsipredPlugin.obj
 0001:00000000       ??__E?_Generic_object@?$_Error_objects@H@std@@2V_Generic_error_category@2@A@@YAXXZ 10001000 f   PsipredAlgTask.obj
 0001:00000010       ??__E?_Iostream_object@?$_Error_objects@H@std@@2V_Iostream_error_category@2@A@@YAXXZ 10001010 f   PsipredAlgTask.obj
 0001:00000020       ??__E?_System_object@?$_Error_objects@H@std@@2V_System_error_category@2@A@@YAXXZ 10001020 f   PsipredAlgTask.obj
 0001:00000030       ??__E?runLock@PsipredAlgTask@U2@@0VQMutex@@A@@YAXXZ 10001030 f   PsipredAlgTask.obj
 0001:00000050       ??__EService_DNAExport@U2@@YAXXZ 10001050 f   PsipredAlgTask.obj
 0001:00000060       ??__EService_DNAGraphPack@U2@@YAXXZ 10001060 f   PsipredAlgTask.obj
 0001:00000070       ??__EService_ExternalToolSupport@U2@@YAXXZ 10001070 f   PsipredAlgTask.obj
 0001:00000080       ??__EService_GUITesting@U2@@YAXXZ 10001080 f   PsipredAlgTask.obj
 0001:00000090       ??__EService_MaxCoreServiceId@U2@@YAXXZ 10001090 f   PsipredAlgTask.obj
 0001:000000a0       ??__EService_MinCoreServiceId@U2@@YAXXZ 100010a0 f   PsipredAlgTask.obj
 0001:000000b0       ??__EService_PluginViewer@U2@@YAXXZ 100010b0 f   PsipredAlgTask.obj
 0001:000000c0       ??__EService_Project@U2@@YAXXZ 100010c0 f   PsipredAlgTask.obj
 0001:000000d0       ??__EService_ProjectView@U2@@YAXXZ 100010d0 f   PsipredAlgTask.obj
 0001:000000e0       ??__EService_QueryDesigner@U2@@YAXXZ 100010e0 f   PsipredAlgTask.obj
 0001:000000f0       ??__EService_ScriptRegistry@U2@@YAXXZ 100010f0 f   PsipredAlgTask.obj
 0001:00000100       ??__EService_TestRunner@U2@@YAXXZ 10001100 f   PsipredAlgTask.obj
 0001:00000110       ??__EService_WorkflowDesigner@U2@@YAXXZ 10001110 f   PsipredAlgTask.obj
 0001:00000120       ??__EalgoLog@U2@@YAXXZ     10001120 f   PsipredAlgTask.obj
 0001:000001a0       ??__EcmdLog@U2@@YAXXZ      100011a0 f   PsipredAlgTask.obj
 0001:00000220       ??__EcoreLog@U2@@YAXXZ     10001220 f   PsipredAlgTask.obj
 0001:000002a0       ??__EioLog@U2@@YAXXZ       100012a0 f   PsipredAlgTask.obj
 0001:00000320       ??__EperfLog@U2@@YAXXZ     10001320 f   PsipredAlgTask.obj
 0001:000003a0       ??__EscriptLog@U2@@YAXXZ   100013a0 f   PsipredAlgTask.obj
 0001:00000420       ??__EtaskLog@U2@@YAXXZ     10001420 f   PsipredAlgTask.obj
 0001:000004a0       ??__EuiLog@U2@@YAXXZ       100014a0 f   PsipredAlgTask.obj
 0001:00000520       ??__EuserActLog@U2@@YAXXZ  10001520 f   PsipredAlgTask.obj
 0001:000005a0       ??__E?_Generic_object@?$_Error_objects@H@std@@2V_Generic_error_category@2@A@@YAXXZ 100015a0 f   PsipredPlugin.obj
 0001:000005b0       ??__E?_Iostream_object@?$_Error_objects@H@std@@2V_Iostream_error_category@2@A@@YAXXZ 100015b0 f   PsipredPlugin.obj
 0001:000005c0       ??__E?_System_object@?$_Error_objects@H@std@@2V_System_error_category@2@A@@YAXXZ 100015c0 f   PsipredPlugin.obj
 0001:000005d0       ??__EService_DNAExport@U2@@YAXXZ 100015d0 f   PsipredPlugin.obj
 0001:000005e0       ??__EService_DNAGraphPack@U2@@YAXXZ 100015e0 f   PsipredPlugin.obj
 0001:000005f0       ??__EService_ExternalToolSupport@U2@@YAXXZ 100015f0 f   PsipredPlugin.obj
 0001:00000600       ??__EService_GUITesting@U2@@YAXXZ 10001600 f   PsipredPlugin.obj
 0001:00000610       ??__EService_MaxCoreServiceId@U2@@YAXXZ 10001610 f   PsipredPlugin.obj
 0001:00000620       ??__EService_MinCoreServiceId@U2@@YAXXZ 10001620 f   PsipredPlugin.obj
 0001:00000630       ??__EService_PluginViewer@U2@@YAXXZ 10001630 f   PsipredPlugin.obj
 0001:00000640       ??__EService_Project@U2@@YAXXZ 10001640 f   PsipredPlugin.obj
 0001:00000650       ??__EService_ProjectView@U2@@YAXXZ 10001650 f   PsipredPlugin.obj
 0001:00000660       ??__EService_QueryDesigner@U2@@YAXXZ 10001660 f   PsipredPlugin.obj
 0001:00000670       ??__EService_ScriptRegistry@U2@@YAXXZ 10001670 f   PsipredPlugin.obj
 0001:00000680       ??__EService_TestRunner@U2@@YAXXZ 10001680 f   PsipredPlugin.obj
 0001:00000690       ??__EService_WorkflowDesigner@U2@@YAXXZ 10001690 f   PsipredPlugin.obj
 0001:000006a0       ??__EalgoLog@U2@@YAXXZ     100016a0 f   PsipredPlugin.obj
 0001:00000720       ??__EcmdLog@U2@@YAXXZ      10001720 f   PsipredPlugin.obj
 0001:000007a0       ??__EcoreLog@U2@@YAXXZ     100017a0 f   PsipredPlugin.obj
 0001:00000820       ??__EioLog@U2@@YAXXZ       10001820 f   PsipredPlugin.obj
 0001:000008a0       ??__EperfLog@U2@@YAXXZ     100018a0 f   PsipredPlugin.obj
 0001:00000920       ??__EscriptLog@U2@@YAXXZ   10001920 f   PsipredPlugin.obj
 0001:000009a0       ??__EtaskLog@U2@@YAXXZ     100019a0 f   PsipredPlugin.obj
 0001:00000a20       ??__EuiLog@U2@@YAXXZ       10001a20 f   PsipredPlugin.obj
 0001:00000aa0       ??__EuserActLog@U2@@YAXXZ  10001aa0 f   PsipredPlugin.obj
 0001:00000b20       ??__E?_Generic_object@?$_Error_objects@H@std@@2V_Generic_error_category@2@A@@YAXXZ 10001b20 f   seq2mtx.obj
 0001:00000b30       ??__E?_Iostream_object@?$_Error_objects@H@std@@2V_Iostream_error_category@2@A@@YAXXZ 10001b30 f   seq2mtx.obj
 0001:00000b40       ??__E?_System_object@?$_Error_objects@H@std@@2V_System_error_category@2@A@@YAXXZ 10001b40 f   seq2mtx.obj
 0001:00000b50       ??__E?_Generic_object@?$_Error_objects@H@std@@2V_Generic_error_category@2@A@@YAXXZ 10001b50 f   sspred_avpred.obj
 0001:00000b60       ??__E?_Iostream_object@?$_Error_objects@H@std@@2V_Iostream_error_category@2@A@@YAXXZ 10001b60 f   sspred_avpred.obj
 0001:00000b70       ??__E?_System_object@?$_Error_objects@H@std@@2V_System_error_category@2@A@@YAXXZ 10001b70 f   sspred_avpred.obj
 0001:00000b80       ??__E?_Generic_object@?$_Error_objects@H@std@@2V_Generic_error_category@2@A@@YAXXZ 10001b80 f   sspred_hmulti.obj
 0001:00000b90       ??__E?_Iostream_object@?$_Error_objects@H@std@@2V_Iostream_error_category@2@A@@YAXXZ 10001b90 f   sspred_hmulti.obj
 0001:00000ba0       ??__E?_System_object@?$_Error_objects@H@std@@2V_System_error_category@2@A@@YAXXZ 10001ba0 f   sspred_hmulti.obj
 0001:00000bb0       ??__E?_Generic_object@?$_Error_objects@H@std@@2V_Generic_error_category@2@A@@YAXXZ 10001bb0 f   moc_PsipredAlgTask.obj
 0001:00000bc0       ??__E?_Iostream_object@?$_Error_objects@H@std@@2V_Iostream_error_category@2@A@@YAXXZ 10001bc0 f   moc_PsipredAlgTask.obj
 0001:00000bd0       ??__E?_System_object@?$_Error_objects@H@std@@2V_System_error_category@2@A@@YAXXZ 10001bd0 f   moc_PsipredAlgTask.obj
 0001:00000be0       ??__E?staticMetaObject@PsipredAlgTask@U2@@2UQMetaObject@@B@@YAXXZ 10001be0 f   moc_PsipredAlgTask.obj
 0001:00000bf0       ??__EalgoLog@U2@@YAXXZ     10001bf0 f   moc_PsipredAlgTask.obj
 0001:00000c70       ??__EcmdLog@U2@@YAXXZ      10001c70 f   moc_PsipredAlgTask.obj
 0001:00000cf0       ??__EcoreLog@U2@@YAXXZ     10001cf0 f   moc_PsipredAlgTask.obj
 0001:00000d70       ??__EioLog@U2@@YAXXZ       10001d70 f   moc_PsipredAlgTask.obj
 0001:00000df0       ??__EperfLog@U2@@YAXXZ     10001df0 f   moc_PsipredAlgTask.obj
 0001:00000e70       ??__EscriptLog@U2@@YAXXZ   10001e70 f   moc_PsipredAlgTask.obj
 0001:00000ef0       ??__EtaskLog@U2@@YAXXZ     10001ef0 f   moc_PsipredAlgTask.obj
 0001:00000f70       ??__EuiLog@U2@@YAXXZ       10001f70 f   moc_PsipredAlgTask.obj
 0001:00000ff0       ??__EuserActLog@U2@@YAXXZ  10001ff0 f   moc_PsipredAlgTask.obj
 0001:00001070       ??__E?_Generic_object@?$_Error_objects@H@std@@2V_Generic_error_category@2@A@@YAXXZ 10002070 f   moc_PsipredPlugin.obj
 0001:00001080       ??__E?_Iostream_object@?$_Error_objects@H@std@@2V_Iostream_error_category@2@A@@YAXXZ 10002080 f   moc_PsipredPlugin.obj
 0001:00001090       ??__E?_System_object@?$_Error_objects@H@std@@2V_System_error_category@2@A@@YAXXZ 10002090 f   moc_PsipredPlugin.obj
 0001:000010a0       ??__E?staticMetaObject@PsipredPlugin@U2@@2UQMetaObject@@B@@YAXXZ 100020a0 f   moc_PsipredPlugin.obj
 0001:000010b0       ??__EService_DNAExport@U2@@YAXXZ 100020b0 f   moc_PsipredPlugin.obj
 0001:000010c0       ??__EService_DNAGraphPack@U2@@YAXXZ 100020c0 f   moc_PsipredPlugin.obj
 0001:000010d0       ??__EService_ExternalToolSupport@U2@@YAXXZ 100020d0 f   moc_PsipredPlugin.obj
 0001:000010e0       ??__EService_GUITesting@U2@@YAXXZ 100020e0 f   moc_PsipredPlugin.obj
 0001:000010f0       ??__EService_MaxCoreServiceId@U2@@YAXXZ 100020f0 f   moc_PsipredPlugin.obj
 0001:00001100       ??__EService_MinCoreServiceId@U2@@YAXXZ 10002100 f   moc_PsipredPlugin.obj
 0001:00001110       ??__EService_PluginViewer@U2@@YAXXZ 10002110 f   moc_PsipredPlugin.obj
 0001:00001120       ??__EService_Project@U2@@YAXXZ 10002120 f   moc_PsipredPlugin.obj
 0001:00001130       ??__EService_ProjectView@U2@@YAXXZ 10002130 f   moc_PsipredPlugin.obj
 0001:00001140       ??__EService_QueryDesigner@U2@@YAXXZ 10002140 f   moc_PsipredPlugin.obj
 0001:00001150       ??__EService_ScriptRegistry@U2@@YAXXZ 10002150 f   moc_PsipredPlugin.obj
 0001:00001160       ??__EService_TestRunner@U2@@YAXXZ 10002160 f   moc_PsipredPlugin.obj
 0001:00001170       ??__EService_WorkflowDesigner@U2@@YAXXZ 10002170 f   moc_PsipredPlugin.obj
 0001:00001180       ??__Edummy@?A0x86132f99@@YAXXZ 10002180 f   qrc_psipred.obj
 0001:00001bd6       __catch$?_Copy@?$basic_string@DU?$char_traits@D@std@@V?$allocator@D@2@@std@@QAEXII@Z$0 10002bd6 f i PsipredAlgTask.obj
 0001:00001c13       __catch$?_Copy@?$basic_string@DU?$char_traits@D@std@@V?$allocator@D@2@@std@@QAEXII@Z$1 10002c13 f i PsipredAlgTask.obj
 0001:00001f2d       __catch$?append@?$QList@VQString@@@@QAEXABVQString@@@Z$0 10002f2d f i PsipredAlgTask.obj
 0001:00001f7e       __catch$?append@?$QList@VQString@@@@QAEXABVQString@@@Z$4 10002f7e f i PsipredAlgTask.obj
 0001:000024ae       __catch$?detach_helper_grow@?$QList@VQString@@@@AAEPAUNode@1@HH@Z$2 100034ae f i PsipredAlgTask.obj
 0001:000024e9       __catch$?detach_helper_grow@?$QList@VQString@@@@AAEPAUNode@1@HH@Z$0 100034e9 f i PsipredAlgTask.obj
 0001:00002952       __catch$?node_copy@?$QList@VQString@@@@AAEXPAUNode@1@00@Z$2 10003952 f i PsipredAlgTask.obj
 0001:00002e53       __catch$?run@PsipredAlgTask@U2@@UAEXXZ$4 10003e53 f   PsipredAlgTask.obj
 0001:00002f2f       __catch$?run@PsipredAlgTask@U2@@UAEXXZ$2 10003f2f f   PsipredAlgTask.obj
 0001:0000301c       __catch$?run@PsipredAlgTask@U2@@UAEXXZ$0 1000401c f   PsipredAlgTask.obj
 0001:000034f5       __catch$?append@?$QList@PAVAnnotationSettings@U2@@@@QAEXABQAVAnnotationSettings@U2@@@Z$4 100044f5 f i PsipredPlugin.obj
 0001:00003681       __catch$?detach_helper_grow@?$QList@PAVAnnotationSettings@U2@@@@AAEPAUNode@1@HH@Z$2 10004681 f i PsipredPlugin.obj
 0001:00003681       __catch$?detach_helper_grow@?$QList@PAVAnnotationSettings@U2@@@@AAEPAUNode@1@HH@Z$0 10004681 f i PsipredPlugin.obj
 0001:00003ade       __catch$??0?$QList@VQString@@@@QAE@ABV0@@Z$0 10004ade f i sspred_avpred.obj
 0001:000060a0       $$000000                   100070a0     MSVCRT:chkstk.obj
 0001:00006196       _pre_c_init                10007196 f   MSVCRT:crtdll.obj
 0001:00006403       ___DllMainCRTStartup       10007403 f   MSVCRT:crtdll.obj
 0001:00006550       $$000000                   10007550     MSVCRT:sehprolg4.obj
 0001:00006965       ?ArrayUnwindFilter@@YAHPAU_EXCEPTION_POINTERS@@@Z 10007965 f   MSVCRT:ehvecdtr.obj
 0001:00006cb0       __unwindfunclet$??0PsipredAlgTask@U2@@QAE@ABVQByteArray@@@Z$0 10007cb0 f   PsipredAlgTask.obj
 0001:00006cb9       __unwindfunclet$??0PsipredAlgTask@U2@@QAE@ABVQByteArray@@@Z$1 10007cb9 f   PsipredAlgTask.obj
 0001:00006cc7       __unwindfunclet$??0PsipredAlgTask@U2@@QAE@ABVQByteArray@@@Z$2 10007cc7 f   PsipredAlgTask.obj
 0001:00006cd0       __unwindfunclet$??0PsipredAlgTask@U2@@QAE@ABVQByteArray@@@Z$3 10007cd0 f   PsipredAlgTask.obj
 0001:00006cd9       __ehhandler$??0PsipredAlgTask@U2@@QAE@ABVQByteArray@@@Z 10007cd9 f   PsipredAlgTask.obj
 0001:00006d00       __unwindfunclet$??H@YA?BVQString@@ABV0@PBD@Z$0 10007d00 f   PsipredAlgTask.obj
 0001:00006d1a       __unwindfunclet$??H@YA?BVQString@@ABV0@PBD@Z$1 10007d1a f   PsipredAlgTask.obj
 0001:00006d23       __ehhandler$??H@YA?BVQString@@ABV0@PBD@Z 10007d23 f   PsipredAlgTask.obj
 0001:00006d40       __unwindfunclet$??H@YA?BVQString@@ABV0@VQChar@@@Z$0 10007d40 f   PsipredAlgTask.obj
 0001:00006d5a       __ehhandler$??H@YA?BVQString@@ABV0@VQChar@@@Z 10007d5a f   PsipredAlgTask.obj
 0001:00006d80       __unwindfunclet$??__EalgoLog@U2@@YAXXZ$0 10007d80 f   PsipredAlgTask.obj
 0001:00006d89       __ehhandler$??__EalgoLog@U2@@YAXXZ 10007d89 f   PsipredAlgTask.obj
 0001:00006db0       __unwindfunclet$??__EcmdLog@U2@@YAXXZ$0 10007db0 f   PsipredAlgTask.obj
 0001:00006db9       __ehhandler$??__EcmdLog@U2@@YAXXZ 10007db9 f   PsipredAlgTask.obj
 0001:00006de0       __unwindfunclet$??__EcoreLog@U2@@YAXXZ$0 10007de0 f   PsipredAlgTask.obj
 0001:00006de9       __ehhandler$??__EcoreLog@U2@@YAXXZ 10007de9 f   PsipredAlgTask.obj
 0001:00006e10       __unwindfunclet$??__EioLog@U2@@YAXXZ$0 10007e10 f   PsipredAlgTask.obj
 0001:00006e19       __ehhandler$??__EioLog@U2@@YAXXZ 10007e19 f   PsipredAlgTask.obj
 0001:00006e40       __unwindfunclet$??__EperfLog@U2@@YAXXZ$0 10007e40 f   PsipredAlgTask.obj
 0001:00006e49       __ehhandler$??__EperfLog@U2@@YAXXZ 10007e49 f   PsipredAlgTask.obj
 0001:00006e70       __unwindfunclet$??__EscriptLog@U2@@YAXXZ$0 10007e70 f   PsipredAlgTask.obj
 0001:00006e79       __ehhandler$??__EscriptLog@U2@@YAXXZ 10007e79 f   PsipredAlgTask.obj
 0001:00006ea0       __unwindfunclet$??__EtaskLog@U2@@YAXXZ$0 10007ea0 f   PsipredAlgTask.obj
 0001:00006ea9       __ehhandler$??__EtaskLog@U2@@YAXXZ 10007ea9 f   PsipredAlgTask.obj
 0001:00006ed0       __unwindfunclet$??__EuiLog@U2@@YAXXZ$0 10007ed0 f   PsipredAlgTask.obj
 0001:00006ed9       __ehhandler$??__EuiLog@U2@@YAXXZ 10007ed9 f   PsipredAlgTask.obj
 0001:00006f00       __unwindfunclet$??__EuserActLog@U2@@YAXXZ$0 10007f00 f   PsipredAlgTask.obj
 0001:00006f09       __ehhandler$??__EuserActLog@U2@@YAXXZ 10007f09 f   PsipredAlgTask.obj
 0001:00006f30       __ehhandler$?_Copy@?$basic_string@DU?$char_traits@D@std@@V?$allocator@D@2@@std@@QAEXII@Z 10007f30 f   PsipredAlgTask.obj
 0001:00006f50       __unwindfunclet$?append@?$QList@VQString@@@@QAEXABVQString@@@Z$7 10007f50 f   PsipredAlgTask.obj
 0001:00006f61       __unwindfunclet$?append@?$QList@VQString@@@@QAEXABVQString@@@Z$11 10007f61 f   PsipredAlgTask.obj
 0001:00006f72       __ehhandler$?append@?$QList@VQString@@@@QAEXABVQString@@@Z 10007f72 f   PsipredAlgTask.obj
 0001:00006f90       __ehhandler$?detach_helper_grow@?$QList@VQString@@@@AAEPAUNode@1@HH@Z 10007f90 f   PsipredAlgTask.obj
 0001:00006fb0       __unwindfunclet$?node_construct@?$QList@VQString@@@@AAEXPAUNode@1@ABVQString@@@Z$1 10007fb0 f   PsipredAlgTask.obj
 0001:00006fc1       __ehhandler$?node_construct@?$QList@VQString@@@@AAEXPAUNode@1@ABVQString@@@Z 10007fc1 f   PsipredAlgTask.obj
 0001:00006fe0       __unwindfunclet$?node_copy@?$QList@VQString@@@@AAEXPAUNode@1@00@Z$5 10007fe0 f   PsipredAlgTask.obj
 0001:00006ff1       __ehhandler$?node_copy@?$QList@VQString@@@@AAEXPAUNode@1@00@Z 10007ff1 f   PsipredAlgTask.obj
 0001:00007010       __unwindfunclet$?run@PsipredAlgTask@U2@@UAEXXZ$6 10008010 f   PsipredAlgTask.obj
 0001:0000701c       __unwindfunclet$?run@PsipredAlgTask@U2@@UAEXXZ$7 1000801c f   PsipredAlgTask.obj
 0001:00007028       __unwindfunclet$?run@PsipredAlgTask@U2@@UAEXXZ$8 10008028 f   PsipredAlgTask.obj
 0001:00007034       __unwindfunclet$?run@PsipredAlgTask@U2@@UAEXXZ$9 10008034 f   PsipredAlgTask.obj
 0001:00007040       __unwindfunclet$?run@PsipredAlgTask@U2@@UAEXXZ$13 10008040 f   PsipredAlgTask.obj
 0001:0000704b       __unwindfunclet$?run@PsipredAlgTask@U2@@UAEXXZ$14 1000804b f   PsipredAlgTask.obj
 0001:00007057       __unwindfunclet$?run@PsipredAlgTask@U2@@UAEXXZ$15 10008057 f   PsipredAlgTask.obj
 0001:00007063       __unwindfunclet$?run@PsipredAlgTask@U2@@UAEXXZ$16 10008063 f   PsipredAlgTask.obj
 0001:0000706f       __unwindfunclet$?run@PsipredAlgTask@U2@@UAEXXZ$17 1000806f f   PsipredAlgTask.obj
 0001:0000707a       __unwindfunclet$?run@PsipredAlgTask@U2@@UAEXXZ$21 1000807a f   PsipredAlgTask.obj
 0001:00007085       __unwindfunclet$?run@PsipredAlgTask@U2@@UAEXXZ$25 10008085 f   PsipredAlgTask.obj
 0001:00007091       __unwindfunclet$?run@PsipredAlgTask@U2@@UAEXXZ$27 10008091 f   PsipredAlgTask.obj
 0001:0000709d       __unwindfunclet$?run@PsipredAlgTask@U2@@UAEXXZ$28 1000809d f   PsipredAlgTask.obj
 0001:000070a9       __unwindfunclet$?run@PsipredAlgTask@U2@@UAEXXZ$29 100080a9 f   PsipredAlgTask.obj
 0001:000070b5       __unwindfunclet$?run@PsipredAlgTask@U2@@UAEXXZ$30 100080b5 f   PsipredAlgTask.obj
 0001:000070c1       __unwindfunclet$?run@PsipredAlgTask@U2@@UAEXXZ$31 100080c1 f   PsipredAlgTask.obj
 0001:000070cd       __unwindfunclet$?run@PsipredAlgTask@U2@@UAEXXZ$32 100080cd f   PsipredAlgTask.obj
 0001:000070d9       __unwindfunclet$?run@PsipredAlgTask@U2@@UAEXXZ$33 100080d9 f   PsipredAlgTask.obj
 0001:000070e5       __unwindfunclet$?run@PsipredAlgTask@U2@@UAEXXZ$34 100080e5 f   PsipredAlgTask.obj
 0001:000070f1       __unwindfunclet$?run@PsipredAlgTask@U2@@UAEXXZ$22 100080f1 f   PsipredAlgTask.obj
 0001:000070fd       __unwindfunclet$?run@PsipredAlgTask@U2@@UAEXXZ$23 100080fd f   PsipredAlgTask.obj
 0001:00007109       __unwindfunclet$?run@PsipredAlgTask@U2@@UAEXXZ$24 10008109 f   PsipredAlgTask.obj
 0001:00007115       __unwindfunclet$?run@PsipredAlgTask@U2@@UAEXXZ$18 10008115 f   PsipredAlgTask.obj
 0001:00007121       __unwindfunclet$?run@PsipredAlgTask@U2@@UAEXXZ$19 10008121 f   PsipredAlgTask.obj
 0001:0000712d       __unwindfunclet$?run@PsipredAlgTask@U2@@UAEXXZ$20 1000812d f   PsipredAlgTask.obj
 0001:00007139       __unwindfunclet$?run@PsipredAlgTask@U2@@UAEXXZ$10 10008139 f   PsipredAlgTask.obj
 0001:00007145       __unwindfunclet$?run@PsipredAlgTask@U2@@UAEXXZ$11 10008145 f   PsipredAlgTask.obj
 0001:00007151       __unwindfunclet$?run@PsipredAlgTask@U2@@UAEXXZ$12 10008151 f   PsipredAlgTask.obj
 0001:0000715d       __ehhandler$?run@PsipredAlgTask@U2@@UAEXXZ 1000815d f   PsipredAlgTask.obj
 0001:00007190       __unwindfunclet$??0PsipredPlugin@U2@@QAE@XZ$0 10008190 f   PsipredPlugin.obj
 0001:00007199       __unwindfunclet$??0PsipredPlugin@U2@@QAE@XZ$1 10008199 f   PsipredPlugin.obj
 0001:000071a2       __unwindfunclet$??0PsipredPlugin@U2@@QAE@XZ$2 100081a2 f   PsipredPlugin.obj
 0001:000071ab       __unwindfunclet$??0PsipredPlugin@U2@@QAE@XZ$4 100081ab f   PsipredPlugin.obj
 0001:000071b4       __unwindfunclet$??0PsipredPlugin@U2@@QAE@XZ$5 100081b4 f   PsipredPlugin.obj
 0001:000071bf       __unwindfunclet$??0PsipredPlugin@U2@@QAE@XZ$6 100081bf f   PsipredPlugin.obj
 0001:000071d9       __unwindfunclet$??0PsipredPlugin@U2@@QAE@XZ$7 100081d9 f   PsipredPlugin.obj
 0001:000071e1       __ehhandler$??0PsipredPlugin@U2@@QAE@XZ 100081e1 f   PsipredPlugin.obj
 0001:00007210       __unwindfunclet$??__EalgoLog@U2@@YAXXZ$0 10008210 f   PsipredPlugin.obj
 0001:00007219       __ehhandler$??__EalgoLog@U2@@YAXXZ 10008219 f   PsipredPlugin.obj
 0001:00007240       __unwindfunclet$??__EcmdLog@U2@@YAXXZ$0 10008240 f   PsipredPlugin.obj
 0001:00007249       __ehhandler$??__EcmdLog@U2@@YAXXZ 10008249 f   PsipredPlugin.obj
 0001:00007270       __unwindfunclet$??__EcoreLog@U2@@YAXXZ$0 10008270 f   PsipredPlugin.obj
 0001:00007279       __ehhandler$??__EcoreLog@U2@@YAXXZ 10008279 f   PsipredPlugin.obj
 0001:000072a0       __unwindfunclet$??__EioLog@U2@@YAXXZ$0 100082a0 f   PsipredPlugin.obj
 0001:000072a9       __ehhandler$??__EioLog@U2@@YAXXZ 100082a9 f   PsipredPlugin.obj
 0001:000072d0       __unwindfunclet$??__EperfLog@U2@@YAXXZ$0 100082d0 f   PsipredPlugin.obj
 0001:000072d9       __ehhandler$??__EperfLog@U2@@YAXXZ 100082d9 f   PsipredPlugin.obj
 0001:00007300       __unwindfunclet$??__EscriptLog@U2@@YAXXZ$0 10008300 f   PsipredPlugin.obj
 0001:00007309       __ehhandler$??__EscriptLog@U2@@YAXXZ 10008309 f   PsipredPlugin.obj
 0001:00007330       __unwindfunclet$??__EtaskLog@U2@@YAXXZ$0 10008330 f   PsipredPlugin.obj
 0001:00007339       __ehhandler$??__EtaskLog@U2@@YAXXZ 10008339 f   PsipredPlugin.obj
 0001:00007360       __unwindfunclet$??__EuiLog@U2@@YAXXZ$0 10008360 f   PsipredPlugin.obj
 0001:00007369       __ehhandler$??__EuiLog@U2@@YAXXZ 10008369 f   PsipredPlugin.obj
 0001:00007390       __unwindfunclet$??__EuserActLog@U2@@YAXXZ$0 10008390 f   PsipredPlugin.obj
 0001:00007399       __ehhandler$??__EuserActLog@U2@@YAXXZ 10008399 f   PsipredPlugin.obj
 0001:000073c0       __ehhandler$?append@?$QList@PAVAnnotationSettings@U2@@@@QAEXABQAVAnnotationSettings@U2@@@Z 100083c0 f   PsipredPlugin.obj
 0001:000073e0       __unwindfunclet$?createTaskInstance@Factory@PsipredAlgTask@U2@@UAEPAVSecStructPredictTask@3@ABVQByteArray@@@Z$0 100083e0 f   PsipredPlugin.obj
 0001:000073eb       __ehhandler$?createTaskInstance@Factory@PsipredAlgTask@U2@@UAEPAVSecStructPredictTask@3@ABVQByteArray@@@Z 100083eb f   PsipredPlugin.obj
 0001:00007410       __ehhandler$?detach_helper_grow@?$QList@PAVAnnotationSettings@U2@@@@AAEPAUNode@1@HH@Z 10008410 f   PsipredPlugin.obj
 0001:00007430       __unwindfunclet$?seq2mtx@@YAHPBDHPAVQTemporaryFile@@@Z$0 10008430 f   seq2mtx.obj
 0001:00007439       __ehhandler$?seq2mtx@@YAHPBDHPAVQTemporaryFile@@@Z 10008439 f   seq2mtx.obj
 0001:00007460       __ehhandler$??0?$QList@VQString@@@@QAE@ABV0@@Z 10008460 f   sspred_avpred.obj
 0001:00007480       __unwindfunclet$??0PsiPassOne@@QAE@PAVQTemporaryFile@@ABVQStringList@@@Z$0 10008480 f   sspred_avpred.obj
 0001:0000748c       __ehhandler$??0PsiPassOne@@QAE@PAVQTemporaryFile@@ABVQStringList@@@Z 1000848c f   sspred_avpred.obj
 0001:000074b0       __unwindfunclet$??1PsiPassOne@@QAE@XZ$0 100084b0 f   sspred_avpred.obj
 0001:000074bc       __ehhandler$??1PsiPassOne@@QAE@XZ 100084bc f   sspred_avpred.obj
 0001:000074e0       __unwindfunclet$?getmtx@PsiPassOne@@QAEHXZ$0 100084e0 f   sspred_avpred.obj
 0001:000074e9       __unwindfunclet$?getmtx@PsiPassOne@@QAEHXZ$1 100084e9 f   sspred_avpred.obj
 0001:000074f2       __unwindfunclet$?getmtx@PsiPassOne@@QAEHXZ$2 100084f2 f   sspred_avpred.obj
 0001:000074fb       __unwindfunclet$?getmtx@PsiPassOne@@QAEHXZ$3 100084fb f   sspred_avpred.obj
 0001:00007504       __unwindfunclet$?getmtx@PsiPassOne@@QAEHXZ$4 10008504 f   sspred_avpred.obj
 0001:0000750d       __unwindfunclet$?getmtx@PsiPassOne@@QAEHXZ$5 1000850d f   sspred_avpred.obj
 0001:00007516       __unwindfunclet$?getmtx@PsiPassOne@@QAEHXZ$6 10008516 f   sspred_avpred.obj
 0001:0000751f       __unwindfunclet$?getmtx@PsiPassOne@@QAEHXZ$7 1000851f f   sspred_avpred.obj
 0001:00007528       __ehhandler$?getmtx@PsiPassOne@@QAEHXZ 10008528 f   sspred_avpred.obj
 0001:00007550       __unwindfunclet$?load_wts@PsiPassOne@@QAEXPBD@Z$0 10008550 f   sspred_avpred.obj
 0001:00007559       __unwindfunclet$?load_wts@PsiPassOne@@QAEXPBD@Z$1 10008559 f   sspred_avpred.obj
 0001:00007562       __unwindfunclet$?load_wts@PsiPassOne@@QAEXPBD@Z$2 10008562 f   sspred_avpred.obj
 0001:0000756b       __ehhandler$?load_wts@PsiPassOne@@QAEXPBD@Z 1000856b f   sspred_avpred.obj
 0001:00007590       __unwindfunclet$?predict@PsiPassOne@@QAEXXZ$0 10008590 f   sspred_avpred.obj
 0001:00007598       __unwindfunclet$?predict@PsiPassOne@@QAEXXZ$1 10008598 f   sspred_avpred.obj
 0001:000075a1       __unwindfunclet$?predict@PsiPassOne@@QAEXXZ$2 100085a1 f   sspred_avpred.obj
 0001:000075aa       __unwindfunclet$?predict@PsiPassOne@@QAEXXZ$3 100085aa f   sspred_avpred.obj
 0001:000075b3       __unwindfunclet$?predict@PsiPassOne@@QAEXXZ$4 100085b3 f   sspred_avpred.obj
 0001:000075bc       __unwindfunclet$?predict@PsiPassOne@@QAEXXZ$5 100085bc f   sspred_avpred.obj
 0001:000075c5       __unwindfunclet$?predict@PsiPassOne@@QAEXXZ$6 100085c5 f   sspred_avpred.obj
 0001:000075ce       __ehhandler$?predict@PsiPassOne@@QAEXXZ 100085ce f   sspred_avpred.obj
 0001:000075f0       __unwindfunclet$?load_wts@PsiPassTwo@@QAEXPBD@Z$0 100085f0 f   sspred_hmulti.obj
 0001:000075f9       __unwindfunclet$?load_wts@PsiPassTwo@@QAEXPBD@Z$1 100085f9 f   sspred_hmulti.obj
 0001:00007602       __unwindfunclet$?load_wts@PsiPassTwo@@QAEXPBD@Z$2 10008602 f   sspred_hmulti.obj
 0001:0000760b       __ehhandler$?load_wts@PsiPassTwo@@QAEXPBD@Z 1000860b f   sspred_hmulti.obj
 0001:00007630       __unwindfunclet$?predict@PsiPassTwo@@QAE?AVQByteArray@@HMMPBD@Z$0 10008630 f   sspred_hmulti.obj
 0001:0000764a       __ehhandler$?predict@PsiPassTwo@@QAE?AVQByteArray@@HMMPBD@Z 1000864a f   sspred_hmulti.obj
 0001:00007670       __unwindfunclet$?runPsiPass@PsiPassTwo@@QAEHHQAPBDAAVQByteArray@@@Z$0 10008670 f   sspred_hmulti.obj
 0001:00007679       __unwindfunclet$?runPsiPass@PsiPassTwo@@QAEHHQAPBDAAVQByteArray@@@Z$1 10008679 f   sspred_hmulti.obj
 0001:00007682       __unwindfunclet$?runPsiPass@PsiPassTwo@@QAEHHQAPBDAAVQByteArray@@@Z$2 10008682 f   sspred_hmulti.obj
 0001:0000768b       __unwindfunclet$?runPsiPass@PsiPassTwo@@QAEHHQAPBDAAVQByteArray@@@Z$3 1000868b f   sspred_hmulti.obj
 0001:00007694       __unwindfunclet$?runPsiPass@PsiPassTwo@@QAEHHQAPBDAAVQByteArray@@@Z$4 10008694 f   sspred_hmulti.obj
 0001:0000769d       __unwindfunclet$?runPsiPass@PsiPassTwo@@QAEHHQAPBDAAVQByteArray@@@Z$5 1000869d f   sspred_hmulti.obj
 0001:000076a6       __unwindfunclet$?runPsiPass@PsiPassTwo@@QAEHHQAPBDAAVQByteArray@@@Z$6 100086a6 f   sspred_hmulti.obj
 0001:000076af       __unwindfunclet$?runPsiPass@PsiPassTwo@@QAEHHQAPBDAAVQByteArray@@@Z$7 100086af f   sspred_hmulti.obj
 0001:000076b8       __unwindfunclet$?runPsiPass@PsiPassTwo@@QAEHHQAPBDAAVQByteArray@@@Z$8 100086b8 f   sspred_hmulti.obj
 0001:000076c1       __ehhandler$?runPsiPass@PsiPassTwo@@QAEHHQAPBDAAVQByteArray@@@Z 100086c1 f   sspred_hmulti.obj
 0001:000076e0       __unwindfunclet$??__EalgoLog@U2@@YAXXZ$0 100086e0 f   moc_PsipredAlgTask.obj
 0001:000076e9       __ehhandler$??__EalgoLog@U2@@YAXXZ 100086e9 f   moc_PsipredAlgTask.obj
 0001:00007710       __unwindfunclet$??__EcmdLog@U2@@YAXXZ$0 10008710 f   moc_PsipredAlgTask.obj
 0001:00007719       __ehhandler$??__EcmdLog@U2@@YAXXZ 10008719 f   moc_PsipredAlgTask.obj
 0001:00007740       __unwindfunclet$??__EcoreLog@U2@@YAXXZ$0 10008740 f   moc_PsipredAlgTask.obj
 0001:00007749       __ehhandler$??__EcoreLog@U2@@YAXXZ 10008749 f   moc_PsipredAlgTask.obj
 0001:00007770       __unwindfunclet$??__EioLog@U2@@YAXXZ$0 10008770 f   moc_PsipredAlgTask.obj
 0001:00007779       __ehhandler$??__EioLog@U2@@YAXXZ 10008779 f   moc_PsipredAlgTask.obj
 0001:000077a0       __unwindfunclet$??__EperfLog@U2@@YAXXZ$0 100087a0 f   moc_PsipredAlgTask.obj
 0001:000077a9       __ehhandler$??__EperfLog@U2@@YAXXZ 100087a9 f   moc_PsipredAlgTask.obj
 0001:000077d0       __unwindfunclet$??__EscriptLog@U2@@YAXXZ$0 100087d0 f   moc_PsipredAlgTask.obj
 0001:000077d9       __ehhandler$??__EscriptLog@U2@@YAXXZ 100087d9 f   moc_PsipredAlgTask.obj
 0001:00007800       __unwindfunclet$??__EtaskLog@U2@@YAXXZ$0 10008800 f   moc_PsipredAlgTask.obj
 0001:00007809       __ehhandler$??__EtaskLog@U2@@YAXXZ 10008809 f   moc_PsipredAlgTask.obj
 0001:00007830       __unwindfunclet$??__EuiLog@U2@@YAXXZ$0 10008830 f   moc_PsipredAlgTask.obj
 0001:00007839       __ehhandler$??__EuiLog@U2@@YAXXZ 10008839 f   moc_PsipredAlgTask.obj
 0001:00007860       __unwindfunclet$??__EuserActLog@U2@@YAXXZ$0 10008860 f   moc_PsipredAlgTask.obj
 0001:00007869       __ehhandler$??__EuserActLog@U2@@YAXXZ 10008869 f   moc_PsipredAlgTask.obj
 0001:00007890       ??__F?_Generic_object@?$_Error_objects@H@std@@2V_Generic_error_category@2@A@@YAXXZ 10008890 f   PsipredAlgTask.obj
 0001:000078a0       ??__F?_Iostream_object@?$_Error_objects@H@std@@2V_Iostream_error_category@2@A@@YAXXZ 100088a0 f   PsipredAlgTask.obj
 0001:000078b0       ??__F?_System_object@?$_Error_objects@H@std@@2V_System_error_category@2@A@@YAXXZ 100088b0 f   PsipredAlgTask.obj
 0001:000078c0       ??__F?runLock@PsipredAlgTask@U2@@0VQMutex@@A@@YAXXZ 100088c0 f   PsipredAlgTask.obj
 0001:000078d0       ??__FService_DNAExport@U2@@YAXXZ 100088d0 f   PsipredAlgTask.obj
 0001:000078e0       ??__FService_DNAGraphPack@U2@@YAXXZ 100088e0 f   PsipredAlgTask.obj
 0001:000078f0       ??__FService_ExternalToolSupport@U2@@YAXXZ 100088f0 f   PsipredAlgTask.obj
 0001:00007900       ??__FService_GUITesting@U2@@YAXXZ 10008900 f   PsipredAlgTask.obj
 0001:00007910       ??__FService_MaxCoreServiceId@U2@@YAXXZ 10008910 f   PsipredAlgTask.obj
 0001:00007920       ??__FService_MinCoreServiceId@U2@@YAXXZ 10008920 f   PsipredAlgTask.obj
 0001:00007930       ??__FService_PluginViewer@U2@@YAXXZ 10008930 f   PsipredAlgTask.obj
 0001:00007940       ??__FService_Project@U2@@YAXXZ 10008940 f   PsipredAlgTask.obj
 0001:00007950       ??__FService_ProjectView@U2@@YAXXZ 10008950 f   PsipredAlgTask.obj
 0001:00007960       ??__FService_QueryDesigner@U2@@YAXXZ 10008960 f   PsipredAlgTask.obj
 0001:00007970       ??__FService_ScriptRegistry@U2@@YAXXZ 10008970 f   PsipredAlgTask.obj
 0001:00007980       ??__FService_TestRunner@U2@@YAXXZ 10008980 f   PsipredAlgTask.obj
 0001:00007990       ??__FService_WorkflowDesigner@U2@@YAXXZ 10008990 f   PsipredAlgTask.obj
 0001:000079a0       ??__FalgoLog@U2@@YAXXZ     100089a0 f   PsipredAlgTask.obj
 0001:000079b0       ??__FcmdLog@U2@@YAXXZ      100089b0 f   PsipredAlgTask.obj
 0001:000079c0       ??__FcoreLog@U2@@YAXXZ     100089c0 f   PsipredAlgTask.obj
 0001:000079d0       ??__Fcvar@?1???0PsipredAlgTask@U2@@QAE@ABVQByteArray@@@Z@YAXXZ 100089d0 f   PsipredAlgTask.obj
 0001:000079e0       ??__FioLog@U2@@YAXXZ       100089e0 f   PsipredAlgTask.obj
 0001:000079f0       ??__FperfLog@U2@@YAXXZ     100089f0 f   PsipredAlgTask.obj
 0001:00007a00       ??__FscriptLog@U2@@YAXXZ   10008a00 f   PsipredAlgTask.obj
 0001:00007a10       ??__FtaskLog@U2@@YAXXZ     10008a10 f   PsipredAlgTask.obj
 0001:00007a20       ??__FuiLog@U2@@YAXXZ       10008a20 f   PsipredAlgTask.obj
 0001:00007a30       ??__FuserActLog@U2@@YAXXZ  10008a30 f   PsipredAlgTask.obj
 0001:00007a40       ??__F?_Generic_object@?$_Error_objects@H@std@@2V_Generic_error_category@2@A@@YAXXZ 10008a40 f   PsipredPlugin.obj
 0001:00007a50       ??__F?_Iostream_object@?$_Error_objects@H@std@@2V_Iostream_error_category@2@A@@YAXXZ 10008a50 f   PsipredPlugin.obj
 0001:00007a60       ??__F?_System_object@?$_Error_objects@H@std@@2V_System_error_category@2@A@@YAXXZ 10008a60 f   PsipredPlugin.obj
 0001:00007a70       ??__FService_DNAExport@U2@@YAXXZ 10008a70 f   PsipredPlugin.obj
 0001:00007a80       ??__FService_DNAGraphPack@U2@@YAXXZ 10008a80 f   PsipredPlugin.obj
 0001:00007a90       ??__FService_ExternalToolSupport@U2@@YAXXZ 10008a90 f   PsipredPlugin.obj
 0001:00007aa0       ??__FService_GUITesting@U2@@YAXXZ 10008aa0 f   PsipredPlugin.obj
 0001:00007ab0       ??__FService_MaxCoreServiceId@U2@@YAXXZ 10008ab0 f   PsipredPlugin.obj
 0001:00007ac0       ??__FService_MinCoreServiceId@U2@@YAXXZ 10008ac0 f   PsipredPlugin.obj
 0001:00007ad0       ??__FService_PluginViewer@U2@@YAXXZ 10008ad0 f   PsipredPlugin.obj
 0001:00007ae0       ??__FService_Project@U2@@YAXXZ 10008ae0 f   PsipredPlugin.obj
 0001:00007af0       ??__FService_ProjectView@U2@@YAXXZ 10008af0 f   PsipredPlugin.obj
 0001:00007b00       ??__FService_QueryDesigner@U2@@YAXXZ 10008b00 f   PsipredPlugin.obj
 0001:00007b10       ??__FService_ScriptRegistry@U2@@YAXXZ 10008b10 f   PsipredPlugin.obj
 0001:00007b20       ??__FService_TestRunner@U2@@YAXXZ 10008b20 f   PsipredPlugin.obj
 0001:00007b30       ??__FService_WorkflowDesigner@U2@@YAXXZ 10008b30 f   PsipredPlugin.obj
 0001:00007b40       ??__FalgoLog@U2@@YAXXZ     10008b40 f   PsipredPlugin.obj
 0001:00007b50       ??__FcmdLog@U2@@YAXXZ      10008b50 f   PsipredPlugin.obj
 0001:00007b60       ??__FcoreLog@U2@@YAXXZ     10008b60 f   PsipredPlugin.obj
 0001:00007b70       ??__FioLog@U2@@YAXXZ       10008b70 f   PsipredPlugin.obj
 0001:00007b80       ??__FperfLog@U2@@YAXXZ     10008b80 f   PsipredPlugin.obj
 0001:00007b90       ??__FscriptLog@U2@@YAXXZ   10008b90 f   PsipredPlugin.obj
 0001:00007ba0       ??__FtaskLog@U2@@YAXXZ     10008ba0 f   PsipredPlugin.obj
 0001:00007bb0       ??__FuiLog@U2@@YAXXZ       10008bb0 f   PsipredPlugin.obj
 0001:00007bc0       ??__FuserActLog@U2@@YAXXZ  10008bc0 f   PsipredPlugin.obj
 0001:00007bd0       ??__F?_Generic_object@?$_Error_objects@H@std@@2V_Generic_error_category@2@A@@YAXXZ 10008bd0 f   seq2mtx.obj
 0001:00007be0       ??__F?_Iostream_object@?$_Error_objects@H@std@@2V_Iostream_error_category@2@A@@YAXXZ 10008be0 f   seq2mtx.obj
 0001:00007bf0       ??__F?_System_object@?$_Error_objects@H@std@@2V_System_error_category@2@A@@YAXXZ 10008bf0 f   seq2mtx.obj
 0001:00007c00       ??__F?_Generic_object@?$_Error_objects@H@std@@2V_Generic_error_category@2@A@@YAXXZ 10008c00 f   sspred_avpred.obj
 0001:00007c10       ??__F?_Iostream_object@?$_Error_objects@H@std@@2V_Iostream_error_category@2@A@@YAXXZ 10008c10 f   sspred_avpred.obj
 0001:00007c20       ??__F?_System_object@?$_Error_objects@H@std@@2V_System_error_category@2@A@@YAXXZ 10008c20 f   sspred_avpred.obj
 0001:00007c30       ??__F?_Generic_object@?$_Error_objects@H@std@@2V_Generic_error_category@2@A@@YAXXZ 10008c30 f   sspred_hmulti.obj
 0001:00007c40       ??__F?_Iostream_object@?$_Error_objects@H@std@@2V_Iostream_error_category@2@A@@YAXXZ 10008c40 f   sspred_hmulti.obj
 0001:00007c50       ??__F?_System_object@?$_Error_objects@H@std@@2V_System_error_category@2@A@@YAXXZ 10008c50 f   sspred_hmulti.obj
 0001:00007c60       ??__F?_Generic_object@?$_Error_objects@H@std@@2V_Generic_error_category@2@A@@YAXXZ 10008c60 f   moc_PsipredAlgTask.obj
 0001:00007c70       ??__F?_Iostream_object@?$_Error_objects@H@std@@2V_Iostream_error_category@2@A@@YAXXZ 10008c70 f   moc_PsipredAlgTask.obj
 0001:00007c80       ??__F?_System_object@?$_Error_objects@H@std@@2V_System_error_category@2@A@@YAXXZ 10008c80 f   moc_PsipredAlgTask.obj
 0001:00007c90       ??__FalgoLog@U2@@YAXXZ     10008c90 f   moc_PsipredAlgTask.obj
 0001:00007ca0       ??__FcmdLog@U2@@YAXXZ      10008ca0 f   moc_PsipredAlgTask.obj
 0001:00007cb0       ??__FcoreLog@U2@@YAXXZ     10008cb0 f   moc_PsipredAlgTask.obj
 0001:00007cc0       ??__FioLog@U2@@YAXXZ       10008cc0 f   moc_PsipredAlgTask.obj
 0001:00007cd0       ??__FperfLog@U2@@YAXXZ     10008cd0 f   moc_PsipredAlgTask.obj
 0001:00007ce0       ??__FscriptLog@U2@@YAXXZ   10008ce0 f   moc_PsipredAlgTask.obj
 0001:00007cf0       ??__FtaskLog@U2@@YAXXZ     10008cf0 f   moc_PsipredAlgTask.obj
 0001:00007d00       ??__FuiLog@U2@@YAXXZ       10008d00 f   moc_PsipredAlgTask.obj
 0001:00007d10       ??__FuserActLog@U2@@YAXXZ  10008d10 f   moc_PsipredAlgTask.obj
 0001:00007d20       ??__F?_Generic_object@?$_Error_objects@H@std@@2V_Generic_error_category@2@A@@YAXXZ 10008d20 f   moc_PsipredPlugin.obj
 0001:00007d30       ??__F?_Iostream_object@?$_Error_objects@H@std@@2V_Iostream_error_category@2@A@@YAXXZ 10008d30 f   moc_PsipredPlugin.obj
 0001:00007d40       ??__F?_System_object@?$_Error_objects@H@std@@2V_System_error_category@2@A@@YAXXZ 10008d40 f   moc_PsipredPlugin.obj
 0001:00007d50       ??__FService_DNAExport@U2@@YAXXZ 10008d50 f   moc_PsipredPlugin.obj
 0001:00007d60       ??__FService_DNAGraphPack@U2@@YAXXZ 10008d60 f   moc_PsipredPlugin.obj
 0001:00007d70       ??__FService_ExternalToolSupport@U2@@YAXXZ 10008d70 f   moc_PsipredPlugin.obj
 0001:00007d80       ??__FService_GUITesting@U2@@YAXXZ 10008d80 f   moc_PsipredPlugin.obj
 0001:00007d90       ??__FService_MaxCoreServiceId@U2@@YAXXZ 10008d90 f   moc_PsipredPlugin.obj
 0001:00007da0       ??__FService_MinCoreServiceId@U2@@YAXXZ 10008da0 f   moc_PsipredPlugin.obj
 0001:00007db0       ??__FService_PluginViewer@U2@@YAXXZ 10008db0 f   moc_PsipredPlugin.obj
 0001:00007dc0       ??__FService_Project@U2@@YAXXZ 10008dc0 f   moc_PsipredPlugin.obj
 0001:00007dd0       ??__FService_ProjectView@U2@@YAXXZ 10008dd0 f   moc_PsipredPlugin.obj
 0001:00007de0       ??__FService_QueryDesigner@U2@@YAXXZ 10008de0 f   moc_PsipredPlugin.obj
 0001:00007df0       ??__FService_ScriptRegistry@U2@@YAXXZ 10008df0 f   moc_PsipredPlugin.obj
 0001:00007e00       ??__FService_TestRunner@U2@@YAXXZ 10008e00 f   moc_PsipredPlugin.obj
 0001:00007e10       ??__FService_WorkflowDesigner@U2@@YAXXZ 10008e10 f   moc_PsipredPlugin.obj
 0001:00007e20       ??__Fdummy@?A0x86132f99@@YAXXZ 10008e20 f   qrc_psipred.obj
 0002:000002c4       _Service_PluginViewer$initializer$ 100092c4     PsipredAlgTask.obj
 0002:000002c8       _Service_Project$initializer$ 100092c8     PsipredAlgTask.obj
 0002:000002cc       _Service_ProjectView$initializer$ 100092cc     PsipredAlgTask.obj
 0002:000002d0       _Service_DNAGraphPack$initializer$ 100092d0     PsipredAlgTask.obj
 0002:000002d4       _Service_DNAExport$initializer$ 100092d4     PsipredAlgTask.obj
 0002:000002d8       _Service_TestRunner$initializer$ 100092d8     PsipredAlgTask.obj
 0002:000002dc       _Service_ScriptRegistry$initializer$ 100092dc     PsipredAlgTask.obj
 0002:000002e0       _Service_ExternalToolSupport$initializer$ 100092e0     PsipredAlgTask.obj
 0002:000002e4       _Service_GUITesting$initializer$ 100092e4     PsipredAlgTask.obj
 0002:000002e8       _Service_WorkflowDesigner$initializer$ 100092e8     PsipredAlgTask.obj
 0002:000002ec       _Service_QueryDesigner$initializer$ 100092ec     PsipredAlgTask.obj
 0002:000002f0       _Service_MinCoreServiceId$initializer$ 100092f0     PsipredAlgTask.obj
 0002:000002f4       _Service_MaxCoreServiceId$initializer$ 100092f4     PsipredAlgTask.obj
 0002:000002f8       _algoLog$initializer$      100092f8     PsipredAlgTask.obj
 0002:000002fc       _cmdLog$initializer$       100092fc     PsipredAlgTask.obj
 0002:00000300       _coreLog$initializer$      10009300     PsipredAlgTask.obj
 0002:00000304       _ioLog$initializer$        10009304     PsipredAlgTask.obj
 0002:00000308       _perfLog$initializer$      10009308     PsipredAlgTask.obj
 0002:0000030c       _scriptLog$initializer$    1000930c     PsipredAlgTask.obj
 0002:00000310       _taskLog$initializer$      10009310     PsipredAlgTask.obj
 0002:00000314       _uiLog$initializer$        10009314     PsipredAlgTask.obj
 0002:00000318       _userActLog$initializer$   10009318     PsipredAlgTask.obj
 0002:0000031c       ?runLock$initializer$@PsipredAlgTask@U2@@0P6AXXZA 1000931c     PsipredAlgTask.obj
 0002:00000320       ?_Generic_object$initializer$@?$_Error_objects@H@std@@2P6AXXZA 10009320     PsipredAlgTask.obj
 0002:00000324       ?_Iostream_object$initializer$@?$_Error_objects@H@std@@2P6AXXZA 10009324     PsipredAlgTask.obj
 0002:00000328       ?_System_object$initializer$@?$_Error_objects@H@std@@2P6AXXZA 10009328     PsipredAlgTask.obj
 0002:0000032c       _algoLog$initializer$      1000932c     PsipredPlugin.obj
 0002:00000330       _cmdLog$initializer$       10009330     PsipredPlugin.obj
 0002:00000334       _coreLog$initializer$      10009334     PsipredPlugin.obj
 0002:00000338       _ioLog$initializer$        10009338     PsipredPlugin.obj
 0002:0000033c       _perfLog$initializer$      1000933c     PsipredPlugin.obj
 0002:00000340       _scriptLog$initializer$    10009340     PsipredPlugin.obj
 0002:00000344       _taskLog$initializer$      10009344     PsipredPlugin.obj
 0002:00000348       _uiLog$initializer$        10009348     PsipredPlugin.obj
 0002:0000034c       _userActLog$initializer$   1000934c     PsipredPlugin.obj
 0002:00000350       _Service_PluginViewer$initializer$ 10009350     PsipredPlugin.obj
 0002:00000354       _Service_Project$initializer$ 10009354     PsipredPlugin.obj
 0002:00000358       _Service_ProjectView$initializer$ 10009358     PsipredPlugin.obj
 0002:0000035c       _Service_DNAGraphPack$initializer$ 1000935c     PsipredPlugin.obj
 0002:00000360       _Service_DNAExport$initializer$ 10009360     PsipredPlugin.obj
 0002:00000364       _Service_TestRunner$initializer$ 10009364     PsipredPlugin.obj
 0002:00000368       _Service_ScriptRegistry$initializer$ 10009368     PsipredPlugin.obj
 0002:0000036c       _Service_ExternalToolSupport$initializer$ 1000936c     PsipredPlugin.obj
 0002:00000370       _Service_GUITesting$initializer$ 10009370     PsipredPlugin.obj
 0002:00000374       _Service_WorkflowDesigner$initializer$ 10009374     PsipredPlugin.obj
 0002:00000378       _Service_QueryDesigner$initializer$ 10009378     PsipredPlugin.obj
 0002:0000037c       _Service_MinCoreServiceId$initializer$ 1000937c     PsipredPlugin.obj
 0002:00000380       _Service_MaxCoreServiceId$initializer$ 10009380     PsipredPlugin.obj
 0002:00000384       _algoLog$initializer$      10009384     moc_PsipredAlgTask.obj
 0002:00000388       _cmdLog$initializer$       10009388     moc_PsipredAlgTask.obj
 0002:0000038c       _coreLog$initializer$      1000938c     moc_PsipredAlgTask.obj
 0002:00000390       _ioLog$initializer$        10009390     moc_PsipredAlgTask.obj
 0002:00000394       _perfLog$initializer$      10009394     moc_PsipredAlgTask.obj
 0002:00000398       _scriptLog$initializer$    10009398     moc_PsipredAlgTask.obj
 0002:0000039c       _taskLog$initializer$      1000939c     moc_PsipredAlgTask.obj
 0002:000003a0       _uiLog$initializer$        100093a0     moc_PsipredAlgTask.obj
 0002:000003a4       _userActLog$initializer$   100093a4     moc_PsipredAlgTask.obj
 0002:000003a8       ?staticMetaObject$initializer$@PsipredAlgTask@U2@@2P6AXXZA 100093a8     moc_PsipredAlgTask.obj
 0002:000003ac       _Service_PluginViewer$initializer$ 100093ac     moc_PsipredPlugin.obj
 0002:000003b0       _Service_Project$initializer$ 100093b0     moc_PsipredPlugin.obj
 0002:000003b4       _Service_ProjectView$initializer$ 100093b4     moc_PsipredPlugin.obj
 0002:000003b8       _Service_DNAGraphPack$initializer$ 100093b8     moc_PsipredPlugin.obj
 0002:000003bc       _Service_DNAExport$initializer$ 100093bc     moc_PsipredPlugin.obj
 0002:000003c0       _Service_TestRunner$initializer$ 100093c0     moc_PsipredPlugin.obj
 0002:000003c4       _Service_ScriptRegistry$initializer$ 100093c4     moc_PsipredPlugin.obj
 0002:000003c8       _Service_ExternalToolSupport$initializer$ 100093c8     moc_PsipredPlugin.obj
 0002:000003cc       _Service_GUITesting$initializer$ 100093cc     moc_PsipredPlugin.obj
 0002:000003d0       _Service_WorkflowDesigner$initializer$ 100093d0     moc_PsipredPlugin.obj
 0002:000003d4       _Service_QueryDesigner$initializer$ 100093d4     moc_PsipredPlugin.obj
 0002:000003d8       _Service_MinCoreServiceId$initializer$ 100093d8     moc_PsipredPlugin.obj
 0002:000003dc       _Service_MaxCoreServiceId$initializer$ 100093dc     moc_PsipredPlugin.obj
 0002:000003e0       ?staticMetaObject$initializer$@PsipredPlugin@U2@@2P6AXXZA 100093e0     moc_PsipredPlugin.obj
 0002:000003e4       _dummy$initializer$        100093e4     qrc_psipred.obj
 0002:000003f0       _pcinit                    100093f0     MSVCRT:crtdll.obj
 0002:000003f4       _pinit                     100093f4     MSVCRT:atonexit.obj
 0002:00000830       _aamat                     10009830     seq2mtx.obj
 0002:00000f88       ?aacvs@?1??aanum@@YAHH@Z@4QBHB 10009f88     sspred_utils.obj
 0002:00000ff4       _qt_meta_stringdata_U2__PsipredAlgTask 10009ff4     moc_PsipredAlgTask.obj
 0002:00001018       _qt_meta_data_U2__PsipredAlgTask 1000a018     moc_PsipredAlgTask.obj
 0002:00001054       _qt_meta_stringdata_U2__PsipredPlugin 1000a054     moc_PsipredPlugin.obj
 0002:00001078       _qt_meta_data_U2__PsipredPlugin 1000a078     moc_PsipredPlugin.obj
 0002:000010b8       _qt_resource_data          1000a0b8     qrc_psipred.obj
 0002:000d91b8       _qt_resource_name          100e21b8     qrc_psipred.obj
 0002:000d9270       _qt_resource_struct        100e2270     qrc_psipred.obj
 0002:000d92e0       _GS_ExceptionPointers      100e22e0     MSVCRT:gs_report.obj
 0002:000d9900       __catchsym$?_Copy@?$basic_string@DU?$char_traits@D@std@@V?$allocator@D@2@@std@@QAEXII@Z$5 100e2900     PsipredAlgTask.obj
 0002:000d9910       __catchsym$?_Copy@?$basic_string@DU?$char_traits@D@std@@V?$allocator@D@2@@std@@QAEXII@Z$4 100e2910     PsipredAlgTask.obj
 0002:000d9920       __unwindtable$?_Copy@?$basic_string@DU?$char_traits@D@std@@V?$allocator@D@2@@std@@QAEXII@Z 100e2920     PsipredAlgTask.obj
 0002:000d9940       __ehfuncinfo$?_Copy@?$basic_string@DU?$char_traits@D@std@@V?$allocator@D@2@@std@@QAEXII@Z 100e2940     PsipredAlgTask.obj
 0002:000d9964       __tryblocktable$?_Copy@?$basic_string@DU?$char_traits@D@std@@V?$allocator@D@2@@std@@QAEXII@Z 100e2964     PsipredAlgTask.obj
 0002:000d998c       __unwindtable$??H@YA?BVQString@@ABV0@VQChar@@@Z 100e298c     PsipredAlgTask.obj
 0002:000d9994       __ehfuncinfo$??H@YA?BVQString@@ABV0@VQChar@@@Z 100e2994     PsipredAlgTask.obj
 0002:000d99b8       __unwindtable$??H@YA?BVQString@@ABV0@PBD@Z 100e29b8     PsipredAlgTask.obj
 0002:000d99c8       __ehfuncinfo$??H@YA?BVQString@@ABV0@PBD@Z 100e29c8     PsipredAlgTask.obj
 0002:000d99ec       __catchsym$?append@?$QList@VQString@@@@QAEXABVQString@@@Z$13 100e29ec     PsipredAlgTask.obj
 0002:000d99fc       __catchsym$?append@?$QList@VQString@@@@QAEXABVQString@@@Z$12 100e29fc     PsipredAlgTask.obj
 0002:000d9a0c       __ehfuncinfo$?append@?$QList@VQString@@@@QAEXABVQString@@@Z 100e2a0c     PsipredAlgTask.obj
 0002:000d9a30       __tryblocktable$?append@?$QList@VQString@@@@QAEXABVQString@@@Z 100e2a30     PsipredAlgTask.obj
 0002:000d9a58       __unwindtable$?append@?$QList@VQString@@@@QAEXABVQString@@@Z 100e2a58     PsipredAlgTask.obj
 0002:000d9ab8       __catchsym$?detach_helper_grow@?$QList@VQString@@@@AAEPAUNode@1@HH@Z$5 100e2ab8     PsipredAlgTask.obj
 0002:000d9ac8       __catchsym$?detach_helper_grow@?$QList@VQString@@@@AAEPAUNode@1@HH@Z$4 100e2ac8     PsipredAlgTask.obj
 0002:000d9ad8       __unwindtable$?detach_helper_grow@?$QList@VQString@@@@AAEPAUNode@1@HH@Z 100e2ad8     PsipredAlgTask.obj
 0002:000d9af8       __ehfuncinfo$?detach_helper_grow@?$QList@VQString@@@@AAEPAUNode@1@HH@Z 100e2af8     PsipredAlgTask.obj
 0002:000d9b1c       __tryblocktable$?detach_helper_grow@?$QList@VQString@@@@AAEPAUNode@1@HH@Z 100e2b1c     PsipredAlgTask.obj
 0002:000d9b44       __unwindtable$?node_construct@?$QList@VQString@@@@AAEXPAUNode@1@ABVQString@@@Z 100e2b44     PsipredAlgTask.obj
 0002:000d9b54       __ehfuncinfo$?node_construct@?$QList@VQString@@@@AAEXPAUNode@1@ABVQString@@@Z 100e2b54     PsipredAlgTask.obj
 0002:000d9b78       __catchsym$?node_copy@?$QList@VQString@@@@AAEXPAUNode@1@00@Z$6 100e2b78     PsipredAlgTask.obj
 0002:000d9b88       __tryblocktable$?node_copy@?$QList@VQString@@@@AAEXPAUNode@1@00@Z 100e2b88     PsipredAlgTask.obj
 0002:000d9b9c       __ehfuncinfo$?node_copy@?$QList@VQString@@@@AAEXPAUNode@1@00@Z 100e2b9c     PsipredAlgTask.obj
 0002:000d9bc0       __unwindtable$?node_copy@?$QList@VQString@@@@AAEXPAUNode@1@00@Z 100e2bc0     PsipredAlgTask.obj
 0002:000d9bf0       __unwindtable$??__EalgoLog@U2@@YAXXZ 100e2bf0     PsipredAlgTask.obj
 0002:000d9bf8       __ehfuncinfo$??__EalgoLog@U2@@YAXXZ 100e2bf8     PsipredAlgTask.obj
 0002:000d9c1c       __unwindtable$??__EcmdLog@U2@@YAXXZ 100e2c1c     PsipredAlgTask.obj
 0002:000d9c24       __ehfuncinfo$??__EcmdLog@U2@@YAXXZ 100e2c24     PsipredAlgTask.obj
 0002:000d9c48       __unwindtable$??__EcoreLog@U2@@YAXXZ 100e2c48     PsipredAlgTask.obj
 0002:000d9c50       __ehfuncinfo$??__EcoreLog@U2@@YAXXZ 100e2c50     PsipredAlgTask.obj
 0002:000d9c74       __unwindtable$??__EioLog@U2@@YAXXZ 100e2c74     PsipredAlgTask.obj
 0002:000d9c7c       __ehfuncinfo$??__EioLog@U2@@YAXXZ 100e2c7c     PsipredAlgTask.obj
 0002:000d9ca0       __unwindtable$??__EperfLog@U2@@YAXXZ 100e2ca0     PsipredAlgTask.obj
 0002:000d9ca8       __ehfuncinfo$??__EperfLog@U2@@YAXXZ 100e2ca8     PsipredAlgTask.obj
 0002:000d9ccc       __unwindtable$??__EscriptLog@U2@@YAXXZ 100e2ccc     PsipredAlgTask.obj
 0002:000d9cd4       __ehfuncinfo$??__EscriptLog@U2@@YAXXZ 100e2cd4     PsipredAlgTask.obj
 0002:000d9cf8       __unwindtable$??__EtaskLog@U2@@YAXXZ 100e2cf8     PsipredAlgTask.obj
 0002:000d9d00       __ehfuncinfo$??__EtaskLog@U2@@YAXXZ 100e2d00     PsipredAlgTask.obj
 0002:000d9d24       __unwindtable$??__EuiLog@U2@@YAXXZ 100e2d24     PsipredAlgTask.obj
 0002:000d9d2c       __ehfuncinfo$??__EuiLog@U2@@YAXXZ 100e2d2c     PsipredAlgTask.obj
 0002:000d9d50       __unwindtable$??__EuserActLog@U2@@YAXXZ 100e2d50     PsipredAlgTask.obj
 0002:000d9d58       __ehfuncinfo$??__EuserActLog@U2@@YAXXZ 100e2d58     PsipredAlgTask.obj
 0002:000d9d7c       __unwindtable$??0PsipredAlgTask@U2@@QAE@ABVQByteArray@@@Z 100e2d7c     PsipredAlgTask.obj
 0002:000d9d9c       __ehfuncinfo$??0PsipredAlgTask@U2@@QAE@ABVQByteArray@@@Z 100e2d9c     PsipredAlgTask.obj
 0002:000d9dc0       __catchsym$?run@PsipredAlgTask@U2@@UAEXXZ$39 100e2dc0     PsipredAlgTask.obj
 0002:000d9dd0       __catchsym$?run@PsipredAlgTask@U2@@UAEXXZ$38 100e2dd0     PsipredAlgTask.obj
 0002:000d9de0       __catchsym$?run@PsipredAlgTask@U2@@UAEXXZ$37 100e2de0     PsipredAlgTask.obj
 0002:000d9df0       __ehfuncinfo$?run@PsipredAlgTask@U2@@UAEXXZ 100e2df0     PsipredAlgTask.obj
 0002:000d9e14       __tryblocktable$?run@PsipredAlgTask@U2@@UAEXXZ 100e2e14     PsipredAlgTask.obj
 0002:000d9e50       __unwindtable$?run@PsipredAlgTask@U2@@UAEXXZ 100e2e50     PsipredAlgTask.obj
 0002:000d9f88       __unwindtable$??__EalgoLog@U2@@YAXXZ 100e2f88     PsipredPlugin.obj
 0002:000d9f90       __ehfuncinfo$??__EalgoLog@U2@@YAXXZ 100e2f90     PsipredPlugin.obj
 0002:000d9fb4       __unwindtable$??__EcmdLog@U2@@YAXXZ 100e2fb4     PsipredPlugin.obj
 0002:000d9fbc       __ehfuncinfo$??__EcmdLog@U2@@YAXXZ 100e2fbc     PsipredPlugin.obj
 0002:000d9fe0       __unwindtable$??__EcoreLog@U2@@YAXXZ 100e2fe0     PsipredPlugin.obj
 0002:000d9fe8       __ehfuncinfo$??__EcoreLog@U2@@YAXXZ 100e2fe8     PsipredPlugin.obj
 0002:000da00c       __unwindtable$??__EioLog@U2@@YAXXZ 100e300c     PsipredPlugin.obj
 0002:000da014       __ehfuncinfo$??__EioLog@U2@@YAXXZ 100e3014     PsipredPlugin.obj
 0002:000da038       __unwindtable$??__EperfLog@U2@@YAXXZ 100e3038     PsipredPlugin.obj
 0002:000da040       __ehfuncinfo$??__EperfLog@U2@@YAXXZ 100e3040     PsipredPlugin.obj
 0002:000da064       __unwindtable$??__EscriptLog@U2@@YAXXZ 100e3064     PsipredPlugin.obj
 0002:000da06c       __ehfuncinfo$??__EscriptLog@U2@@YAXXZ 100e306c     PsipredPlugin.obj
 0002:000da090       __unwindtable$??__EtaskLog@U2@@YAXXZ 100e3090     PsipredPlugin.obj
 0002:000da098       __ehfuncinfo$??__EtaskLog@U2@@YAXXZ 100e3098     PsipredPlugin.obj
 0002:000da0bc       __unwindtable$??__EuiLog@U2@@YAXXZ 100e30bc     PsipredPlugin.obj
 0002:000da0c4       __ehfuncinfo$??__EuiLog@U2@@YAXXZ 100e30c4     PsipredPlugin.obj
 0002:000da0e8       __unwindtable$??__EuserActLog@U2@@YAXXZ 100e30e8     PsipredPlugin.obj
 0002:000da0f0       __ehfuncinfo$??__EuserActLog@U2@@YAXXZ 100e30f0     PsipredPlugin.obj
 0002:000da114       __ehfuncinfo$??0PsipredPlugin@U2@@QAE@XZ 100e3114     PsipredPlugin.obj
 0002:000da138       __unwindtable$??0PsipredPlugin@U2@@QAE@XZ 100e3138     PsipredPlugin.obj
 0002:000da188       __unwindtable$?createTaskInstance@Factory@PsipredAlgTask@U2@@UAEPAVSecStructPredictTask@3@ABVQByteArray@@@Z 100e3188     PsipredPlugin.obj
 0002:000da190       __ehfuncinfo$?createTaskInstance@Factory@PsipredAlgTask@U2@@UAEPAVSecStructPredictTask@3@ABVQByteArray@@@Z 100e3190     PsipredPlugin.obj
 0002:000da1b4       __catchsym$?append@?$QList@PAVAnnotationSettings@U2@@@@QAEXABQAVAnnotationSettings@U2@@@Z$6 100e31b4     PsipredPlugin.obj
 0002:000da1c4       __tryblocktable$?append@?$QList@PAVAnnotationSettings@U2@@@@QAEXABQAVAnnotationSettings@U2@@@Z 100e31c4     PsipredPlugin.obj
 0002:000da1d8       __ehfuncinfo$?append@?$QList@PAVAnnotationSettings@U2@@@@QAEXABQAVAnnotationSettings@U2@@@Z 100e31d8     PsipredPlugin.obj
 0002:000da1fc       __unwindtable$?append@?$QList@PAVAnnotationSettings@U2@@@@QAEXABQAVAnnotationSettings@U2@@@Z 100e31fc     PsipredPlugin.obj
 0002:000da22c       __catchsym$?detach_helper_grow@?$QList@PAVAnnotationSettings@U2@@@@AAEPAUNode@1@HH@Z$5 100e322c     PsipredPlugin.obj
 0002:000da23c       __catchsym$?detach_helper_grow@?$QList@PAVAnnotationSettings@U2@@@@AAEPAUNode@1@HH@Z$4 100e323c     PsipredPlugin.obj
 0002:000da24c       __unwindtable$?detach_helper_grow@?$QList@PAVAnnotationSettings@U2@@@@AAEPAUNode@1@HH@Z 100e324c     PsipredPlugin.obj
 0002:000da26c       __ehfuncinfo$?detach_helper_grow@?$QList@PAVAnnotationSettings@U2@@@@AAEPAUNode@1@HH@Z 100e326c     PsipredPlugin.obj
 0002:000da290       __tryblocktable$?detach_helper_grow@?$QList@PAVAnnotationSettings@U2@@@@AAEPAUNode@1@HH@Z 100e3290     PsipredPlugin.obj
 0002:000da2b8       __unwindtable$?seq2mtx@@YAHPBDHPAVQTemporaryFile@@@Z 100e32b8     seq2mtx.obj
 0002:000da2c0       __ehfuncinfo$?seq2mtx@@YAHPBDHPAVQTemporaryFile@@@Z 100e32c0     seq2mtx.obj
 0002:000da2e4       __catchsym$??0?$QList@VQString@@@@QAE@ABV0@@Z$2 100e32e4     sspred_avpred.obj
 0002:000da2f4       __unwindtable$??0?$QList@VQString@@@@QAE@ABV0@@Z 100e32f4     sspred_avpred.obj
 0002:000da304       __tryblocktable$??0?$QList@VQString@@@@QAE@ABV0@@Z 100e3304     sspred_avpred.obj
 0002:000da318       __ehfuncinfo$??0?$QList@VQString@@@@QAE@ABV0@@Z 100e3318     sspred_avpred.obj
 0002:000da33c       __unwindtable$??0PsiPassOne@@QAE@PAVQTemporaryFile@@ABVQStringList@@@Z 100e333c     sspred_avpred.obj
 0002:000da344       __ehfuncinfo$??0PsiPassOne@@QAE@PAVQTemporaryFile@@ABVQStringList@@@Z 100e3344     sspred_avpred.obj
 0002:000da368       __unwindtable$??1PsiPassOne@@QAE@XZ 100e3368     sspred_avpred.obj
 0002:000da370       __ehfuncinfo$??1PsiPassOne@@QAE@XZ 100e3370     sspred_avpred.obj
 0002:000da394       __unwindtable$?load_wts@PsiPassOne@@QAEXPBD@Z 100e3394     sspred_avpred.obj
 0002:000da3b4       __ehfuncinfo$?load_wts@PsiPassOne@@QAEXPBD@Z 100e33b4     sspred_avpred.obj
 0002:000da3d8       __ehfuncinfo$?getmtx@PsiPassOne@@QAEHXZ 100e33d8     sspred_avpred.obj
 0002:000da3fc       __unwindtable$?getmtx@PsiPassOne@@QAEHXZ 100e33fc     sspred_avpred.obj
 0002:000da43c       __ehfuncinfo$?predict@PsiPassOne@@QAEXXZ 100e343c     sspred_avpred.obj
 0002:000da460       __unwindtable$?predict@PsiPassOne@@QAEXXZ 100e3460     sspred_avpred.obj
 0002:000da4a8       __unwindtable$?load_wts@PsiPassTwo@@QAEXPBD@Z 100e34a8     sspred_hmulti.obj
 0002:000da4c8       __ehfuncinfo$?load_wts@PsiPassTwo@@QAEXPBD@Z 100e34c8     sspred_hmulti.obj
 0002:000da4ec       __unwindtable$?predict@PsiPassTwo@@QAE?AVQByteArray@@HMMPBD@Z 100e34ec     sspred_hmulti.obj
 0002:000da4f4       __ehfuncinfo$?predict@PsiPassTwo@@QAE?AVQByteArray@@HMMPBD@Z 100e34f4     sspred_hmulti.obj
 0002:000da518       __ehfuncinfo$?runPsiPass@PsiPassTwo@@QAEHHQAPBDAAVQByteArray@@@Z 100e3518     sspred_hmulti.obj
 0002:000da53c       __unwindtable$?runPsiPass@PsiPassTwo@@QAEHHQAPBDAAVQByteArray@@@Z 100e353c     sspred_hmulti.obj
 0002:000da5f8       __unwindtable$??__EalgoLog@U2@@YAXXZ 100e35f8     moc_PsipredAlgTask.obj
 0002:000da600       __ehfuncinfo$??__EalgoLog@U2@@YAXXZ 100e3600     moc_PsipredAlgTask.obj
 0002:000da624       __unwindtable$??__EcmdLog@U2@@YAXXZ 100e3624     moc_PsipredAlgTask.obj
 0002:000da62c       __ehfuncinfo$??__EcmdLog@U2@@YAXXZ 100e362c     moc_PsipredAlgTask.obj
 0002:000da650       __unwindtable$??__EcoreLog@U2@@YAXXZ 100e3650     moc_PsipredAlgTask.obj
 0002:000da658       __ehfuncinfo$??__EcoreLog@U2@@YAXXZ 100e3658     moc_PsipredAlgTask.obj
 0002:000da67c       __unwindtable$??__EioLog@U2@@YAXXZ 100e367c     moc_PsipredAlgTask.obj
 0002:000da684       __ehfuncinfo$??__EioLog@U2@@YAXXZ 100e3684     moc_PsipredAlgTask.obj
 0002:000da6a8       __unwindtable$??__EperfLog@U2@@YAXXZ 100e36a8     moc_PsipredAlgTask.obj
 0002:000da6b0       __ehfuncinfo$??__EperfLog@U2@@YAXXZ 100e36b0     moc_PsipredAlgTask.obj
 0002:000da6d4       __unwindtable$??__EscriptLog@U2@@YAXXZ 100e36d4     moc_PsipredAlgTask.obj
 0002:000da6dc       __ehfuncinfo$??__EscriptLog@U2@@YAXXZ 100e36dc     moc_PsipredAlgTask.obj
 0002:000da700       __unwindtable$??__EtaskLog@U2@@YAXXZ 100e3700     moc_PsipredAlgTask.obj
 0002:000da708       __ehfuncinfo$??__EtaskLog@U2@@YAXXZ 100e3708     moc_PsipredAlgTask.obj
 0002:000da72c       __unwindtable$??__EuiLog@U2@@YAXXZ 100e372c     moc_PsipredAlgTask.obj
 0002:000da734       __ehfuncinfo$??__EuiLog@U2@@YAXXZ 100e3734     moc_PsipredAlgTask.obj
 0002:000da758       __unwindtable$??__EuserActLog@U2@@YAXXZ 100e3758     moc_PsipredAlgTask.obj
 0002:000da760       __ehfuncinfo$??__EuserActLog@U2@@YAXXZ 100e3760     moc_PsipredAlgTask.obj
 0002:000da788       __sehtable$__onexit        100e3788     MSVCRT:atonexit.obj
 0002:000da7a8       __sehtable$___DllMainCRTStartup 100e37a8     MSVCRT:crtdll.obj
 0002:000da7d0       __sehtable$??_M@YGXPAXIHP6EX0@Z@Z 100e37d0     MSVCRT:ehvecdtr.obj
 0002:000da7f0       __sehtable$?__ArrayUnwind@@YGXPAXIHP6EX0@Z@Z 100e37f0     MSVCRT:ehvecdtr.obj
 0002:000da810       __sehtable$__IsNonwritableInCurrentImage 100e3810     MSVCRT:pesect.obj
 0002:000da830       .edata                     100e3830     psipred.exp
 0002:000da858       rgpv                       100e3858     psipred.exp
 0002:000da85c       rgszName                   100e385c     psipred.exp
 0002:000da860       rgwOrd                     100e3860     psipred.exp
 0002:000da862       szName                     100e3862     psipred.exp
 0002:000da86e       $N00001                    100e386e     psipred.exp
 0002:000db326       .idata$6                   100e4326     U2Core:U2Core.dll
 0002:000db53e       .idata$6                   100e453e     U2Algorithm:U2Algorithm.dll
 0002:000db5e6       .idata$6                   100e45e6     U2View:U2View.dll
 0002:000db610       .idata$6                   100e4610     Qt5Gui:Qt5Gui.dll
 0002:000dbed0       .idata$6                   100e4ed0     Qt5Core:Qt5Core.dll
 0002:000dbf76       .idata$6                   100e4f76     msvcprt:MSVCP120.dll
 0002:000dc0a8       .idata$6                   100e50a8     MSVCRT:MSVCR120.dll
 0002:000dc2b4       .idata$6                   100e52b4     kernel32:KERNEL32.dll
 0003:0000000c       _Service_PluginViewer      100e600c     PsipredAlgTask.obj
 0003:00000014       _Service_Project           100e6014     PsipredAlgTask.obj
 0003:0000001c       _Service_ProjectView       100e601c     PsipredAlgTask.obj
 0003:00000024       _Service_DNAGraphPack      100e6024     PsipredAlgTask.obj
 0003:0000002c       _Service_DNAExport         100e602c     PsipredAlgTask.obj
 0003:00000034       _Service_TestRunner        100e6034     PsipredAlgTask.obj
 0003:0000003c       _Service_ScriptRegistry    100e603c     PsipredAlgTask.obj
 0003:00000044       _Service_ExternalToolSupport 100e6044     PsipredAlgTask.obj
 0003:0000004c       _Service_GUITesting        100e604c     PsipredAlgTask.obj
 0003:00000054       _Service_WorkflowDesigner  100e6054     PsipredAlgTask.obj
 0003:0000005c       _Service_QueryDesigner     100e605c     PsipredAlgTask.obj
 0003:00000064       _Service_MinCoreServiceId  100e6064     PsipredAlgTask.obj
 0003:0000006c       _Service_MaxCoreServiceId  100e606c     PsipredAlgTask.obj
 0003:00000074       _Service_PluginViewer      100e6074     PsipredPlugin.obj
 0003:0000007c       _Service_Project           100e607c     PsipredPlugin.obj
 0003:00000084       _Service_ProjectView       100e6084     PsipredPlugin.obj
 0003:0000008c       _Service_DNAGraphPack      100e608c     PsipredPlugin.obj
 0003:00000094       _Service_DNAExport         100e6094     PsipredPlugin.obj
 0003:0000009c       _Service_TestRunner        100e609c     PsipredPlugin.obj
 0003:000000a4       _Service_ScriptRegistry    100e60a4     PsipredPlugin.obj
 0003:000000ac       _Service_ExternalToolSupport 100e60ac     PsipredPlugin.obj
 0003:000000b4       _Service_GUITesting        100e60b4     PsipredPlugin.obj
 0003:000000bc       _Service_WorkflowDesigner  100e60bc     PsipredPlugin.obj
 0003:000000c4       _Service_QueryDesigner     100e60c4     PsipredPlugin.obj
 0003:000000cc       _Service_MinCoreServiceId  100e60cc     PsipredPlugin.obj
 0003:000000d4       _Service_MaxCoreServiceId  100e60d4     PsipredPlugin.obj
 0003:0000014c       _Service_PluginViewer      100e614c     moc_PsipredPlugin.obj
 0003:00000154       _Service_Project           100e6154     moc_PsipredPlugin.obj
 0003:0000015c       _Service_ProjectView       100e615c     moc_PsipredPlugin.obj
 0003:00000164       _Service_DNAGraphPack      100e6164     moc_PsipredPlugin.obj
 0003:0000016c       _Service_DNAExport         100e616c     moc_PsipredPlugin.obj
 0003:00000174       _Service_TestRunner        100e6174     moc_PsipredPlugin.obj
 0003:0000017c       _Service_ScriptRegistry    100e617c     moc_PsipredPlugin.obj
 0003:00000184       _Service_ExternalToolSupport 100e6184     moc_PsipredPlugin.obj
 0003:0000018c       _Service_GUITesting        100e618c     moc_PsipredPlugin.obj
 0003:00000194       _Service_WorkflowDesigner  100e6194     moc_PsipredPlugin.obj
 0003:0000019c       _Service_QueryDesigner     100e619c     moc_PsipredPlugin.obj
 0003:000001a4       _Service_MinCoreServiceId  100e61a4     moc_PsipredPlugin.obj
 0003:000001ac       _Service_MaxCoreServiceId  100e61ac     moc_PsipredPlugin.obj
 0003:00000430       __Tuple_alloc              100e6430     PsipredAlgTask.obj
 0003:00000431       _ignore                    100e6431     PsipredAlgTask.obj
 0003:00000432       _allocator_arg             100e6432     PsipredAlgTask.obj
 0003:00000433       _piecewise_construct       100e6433     PsipredAlgTask.obj
 0003:00000434       _taskLog                   100e6434     PsipredAlgTask.obj
 0003:0000043c       _algoLog                   100e643c     PsipredAlgTask.obj
 0003:00000444       _userActLog                100e6444     PsipredAlgTask.obj
 0003:0000044c       _ioLog                     100e644c     PsipredAlgTask.obj
 0003:00000454       _coreLog                   100e6454     PsipredAlgTask.obj
 0003:0000045c       _uiLog                     100e645c     PsipredAlgTask.obj
 0003:00000464       _scriptLog                 100e6464     PsipredAlgTask.obj
 0003:0000046c       _perfLog                   100e646c     PsipredAlgTask.obj
 0003:00000478       _cmdLog                    100e6478     PsipredAlgTask.obj
 0003:00000488       ?cvar@?1???0PsipredAlgTask@U2@@QAE@ABVQByteArray@@@Z@4VGReportableCounter@2@A 100e6488     PsipredAlgTask.obj
 0003:000004b0       ?$S1@?1???0PsipredAlgTask@U2@@QAE@ABVQByteArray@@@Z@4IA 100e64b0     PsipredAlgTask.obj
 0003:000004b4       __Tuple_alloc              100e64b4     PsipredPlugin.obj
 0003:000004b5       _ignore                    100e64b5     PsipredPlugin.obj
 0003:000004b6       _allocator_arg             100e64b6     PsipredPlugin.obj
 0003:000004b7       _piecewise_construct       100e64b7     PsipredPlugin.obj
 0003:000004b8       _taskLog                   100e64b8     PsipredPlugin.obj
 0003:000004c0       _algoLog                   100e64c0     PsipredPlugin.obj
 0003:000004c8       _userActLog                100e64c8     PsipredPlugin.obj
 0003:000004d0       _ioLog                     100e64d0     PsipredPlugin.obj
 0003:000004d8       _coreLog                   100e64d8     PsipredPlugin.obj
 0003:000004e0       _uiLog                     100e64e0     PsipredPlugin.obj
 0003:000004e8       _scriptLog                 100e64e8     PsipredPlugin.obj
 0003:000004f0       _perfLog                   100e64f0     PsipredPlugin.obj
 0003:000004f8       _cmdLog                    100e64f8     PsipredPlugin.obj
 0003:00000500       __Tuple_alloc              100e6500     seq2mtx.obj
 0003:00000501       _ignore                    100e6501     seq2mtx.obj
 0003:00000502       _allocator_arg             100e6502     seq2mtx.obj
 0003:00000503       _piecewise_construct       100e6503     seq2mtx.obj
 0003:00000504       __Tuple_alloc              100e6504     sspred_avpred.obj
 0003:00000505       _ignore                    100e6505     sspred_avpred.obj
 0003:00000506       _allocator_arg             100e6506     sspred_avpred.obj
 0003:00000507       _piecewise_construct       100e6507     sspred_avpred.obj
 0003:00000508       __Tuple_alloc              100e6508     sspred_hmulti.obj
 0003:00000509       _ignore                    100e6509     sspred_hmulti.obj
 0003:0000050a       _allocator_arg             100e650a     sspred_hmulti.obj
 0003:0000050b       _piecewise_construct       100e650b     sspred_hmulti.obj
 0003:0000050c       __Tuple_alloc              100e650c     moc_PsipredAlgTask.obj
 0003:0000050d       _ignore                    100e650d     moc_PsipredAlgTask.obj
 0003:0000050e       _allocator_arg             100e650e     moc_PsipredAlgTask.obj
 0003:0000050f       _piecewise_construct       100e650f     moc_PsipredAlgTask.obj
 0003:00000510       _taskLog                   100e6510     moc_PsipredAlgTask.obj
 0003:00000518       _algoLog                   100e6518     moc_PsipredAlgTask.obj
 0003:00000520       _userActLog                100e6520     moc_PsipredAlgTask.obj
 0003:00000528       _ioLog                     100e6528     moc_PsipredAlgTask.obj
 0003:00000530       _coreLog                   100e6530     moc_PsipredAlgTask.obj
 0003:00000538       _uiLog                     100e6538     moc_PsipredAlgTask.obj
 0003:00000540       _scriptLog                 100e6540     moc_PsipredAlgTask.obj
 0003:00000548       _perfLog                   100e6548     moc_PsipredAlgTask.obj
 0003:00000550       _cmdLog                    100e6550     moc_PsipredAlgTask.obj
 0003:00000558       __Tuple_alloc              100e6558     moc_PsipredPlugin.obj
 0003:00000559       _ignore                    100e6559     moc_PsipredPlugin.obj
 0003:0000055a       _allocator_arg             100e655a     moc_PsipredPlugin.obj
 0003:0000055b       _piecewise_construct       100e655b     moc_PsipredPlugin.obj
 0003:00000560       ___proc_attached           100e6560     MSVCRT:crtdll.obj
 0003:00000568       _GS_ExceptionRecord        100e6568     MSVCRT:gs_report.obj
 0003:000005b8       _GS_ContextRecord          100e65b8     MSVCRT:gs_report.obj
 0003:00000884       _DebuggerWasPresent        100e6884     MSVCRT:gs_report.obj
 0004:00000060       $R000000                   100e7060     * linker generated manifest res *

 Exports

  ordinal    name

        1    _ugene_plugin_init
               exported name: ugene_plugin_init
